:100000000C94F9080C9448090C9448090C9448097C
:100010000C9448090C9448090C9448090C9448091C
:100020000C9448090C94591C0C9448090C944809E8
:100030000C946A360C9448090C9448090C944809AD
:100040000C9448090C9448090C947C180C944809A9
:100050000C94AA0E0C9448090C94740E0C94480944
:100060000C94491F0C9448090C94F0310C944809E5
:100070000C94638F0C9448090C9492860C94480954
:100080000C9448090C9448090C944809701F751F7A
:100090007A1F831F9A1FB11FC11FD11F0C20F5218A
:1000A000B11FB720C820F720152132218C21E7216C
:1000B0000224CF245E25DE251626B926C0282A294B
:1000C000A429ED29372A652A922AF52A3F2B892B64
:1000D000822C0F3243328632F6320E334F330634DF
:1000E000CD34CD34CD34CD34CD34CD34CD34CD3408
:1000F000CD34CD34CD34823484348934A134A33426
:100100000E6ACD6A526B816AA86BD86B426AB06A7C
:1001100095773378B8781A796E79D7793781587AA4
:100120008A7A8A7A8A7A8A7A8A7A8A7A8A7A8A7AAF
:100130008A7AB87A337BC87BED7B307C887C137DF0
:10014000FC7D637E637E637E637E637E637E637E0F
:10015000637E637E9B7EB97EDE7E3A7F767FE57F1F
:100160001280B28037811281128112811281128134
:10017000128112811281B68DB98DB98DB98DC28D62
:10018000C58DC88DDA8DD78D0A0D3D3D3D3D3D3D78
:100190003D3D3D3D3D3D3D3D3D3D3D3D3D3D3D3D8F
:1001A0003D3D3D3D3D3D3D3D3D3D3D3D3D000A0D1F
:1001B000426174743A002025642043656C6C73209E
:1001C00000204C6F77207761726E696E673A202548
:1001D000642E2564000A0D466F756E6420424C2D16
:1001E0004374726C3A20002564000A0D0A0D212127
:1001F000204D495353494E4720424C2D4354524CB5
:100200003A202564202121000A0D43616C69627245
:100210006174696E6720707265737375726520739F
:10022000656E736F722E2E004F4B0A0D000A0D463D
:100230006C696768742D74696D65202575206D691A
:100240006E20546F74616C3A2575206D696E0041A3
:100250006E676C654E69636B202020202020204152
:100260006E676C65526F6C6C20202020202020412E
:1002700063634E69636B20202020202020202041D2
:100280006363526F6C6C2020202020202020205996
:1002900061774779726F202020202020202020487D
:1002A00065696768742056616C756520202020415F
:1002B00063635A2020202020202020202020204757
:1002C0006173202020202020202020202020204377
:1002D0006F6D706173732056616C756520202056B8
:1002E0006F6C74616765205B302E31565D20205243
:1002F00065636569766572204C6576656C2020477C
:1003000079726F20436F6D70617373202020204DD0
:100310006F746F7220312020202020202020204D5B
:100320006F746F7220322020202020202020204D4A
:100330006F746F7220332020202020202020204D39
:100340006F746F7220342020202020202020203144
:100350003620202020202020202020202020203176
:100360003720202020202020202020202020203165
:100370003820202020202020202020202020203154
:100380003920202020202020202020202020205321
:100390006572766F202020202020202020202048F9
:1003A0006F76657267617320202020202020204313
:1003B000757272656E74205B302E31415D20204372
:1003C00061706163697479205B6D41685D202048CC
:1003D000656967687420536574706F696E74203244
:1003E00035202020202020202020202020202032E6
:1003F00036202020202020202020202020202043C4
:100400006F6D7061737320536574706F696E74499A
:1004100032432D4572726F7220202020202020420E
:100420004C204C696D69742020202020202020471A
:1004300050535F4E69636B202020202020202047EE
:1004400050535F526F6C6C202020202020202021F0
:10045000212120494E434F4D50415449424C4520A3
:10046000212121002A002E000A0D20444143206F43
:100470007220493243204552524F52212043686531
:10048000636B204932432C2033567265662C20441E
:10049000414320616E6420424C2D4374726C005BBA
:1004A00025695D005B25695D002B204D696B726FCE
:1004B0004B6F70746572202B0048573A5625642E96
:1004C00025642053573A25642E256425632056342D
:1004D0000053657474696E673A2564202573004D76
:1004E00069786572204572726F72210045525225FB
:1004F00032643A00486172647761726520457272B5
:100500006F7220313A2564202121004D697373698F
:100510006E6720424C2D4374726C3A256421210091
:10052000493243204552524F5221212100486569EA
:100530006768743A202025356900536574706F69C7
:100540006E743A2535690050726573737572653A39
:10055000253569004F66667365743A202025356934
:100560000048656967687420636F6E74726F6C0011
:1005700044495341424C4544006163742E206265F6
:100580006172696E67004E69636B3A2020202020FB
:100590002025356900526F6C6C3A202020202020E5
:1005A00025356900436F6D706173733A20202025F3
:1005B0003569004B25693A25346920204B25693A75
:1005C00025346920004E693A2534692020526F3A5B
:1005D000253469200047733A253469202047693A59
:1005E000253469200050313A253469202050323AB0
:1005F000253469200050333A253469202050343A9C
:1006000025346920004779726F202D2053656E7361
:100610006F72004E69636B25346920282533692E7B
:1006200025692900526F6C6C2534692028253369AF
:100630002E256929004769657225346920282533EC
:100640006929004E69636B202534692028253369A8
:100650002E25782900526F6C6C20253469202825BE
:1006600033692E25782900596177202025346920A7
:100670002825336929004E69636B202534692028B9
:1006800025336929282533692900526F6C6C202590
:1006900034692028253369292825336929005961BF
:1006A00077202025346920282533692928253369B6
:1006B0002900414343202D2053656E736F72004E15
:1006C00069636B2025346920282533692900526F1E
:1006D0006C6C20253469202825336929005A202094
:1006E000202025346920282533692900566F6C7431
:1006F0006167653A2020202533692E25316956002F
:1007000043757272656E743A2020202533692E2558
:1007100031694100506F7765723A202020202025F2
:10072000346957004469736368617267653A2025CC
:1007300035696D416800526563656976657200527E
:10074000432D525353493A2020202025346900522A
:10075000432D5175616C6974793A202534690052D2
:10076000432D4368616E6E656C733A2534690043AE
:100770006F6D70617373004D61676E65743A202010
:1007800020253569004779726F3A202020202025E6
:10079000356900536574706F696E743A2025356948
:1007A00000506F746925693A202025336900506F25
:1007B000746925693A202025336900536572766F84
:1007C000202000536574706F696E74202025336992
:1007D00000506F736974696F6E3A20253369005257
:1007E000616E67653A2533692D25336900424C2DCA
:1007F0004374726C204572726F72732000253364EB
:100800002025336420253364202533642000424CA6
:100810002054656D7065726174757265002533646E
:100820002025336420253364202533642000424C86
:100830002D4374726C20666F756E642000202563F2
:1008400020202025632020202563202020256320D0
:1008500000202563202020256320202025632020E0
:1008600020256320002025632020202D2020202DFE
:100870002020202D2000313000313100313200465F
:100880006C696768742D54696D65202000546F741D
:10089000616C3A2535756D696E004163743A2020AC
:1008A0002535756D696E0028726573657429000AB7
:1008B0000D47656E65726174696E67206465666177
:1008C000756C7420506172616D657465722053653A
:1008D00074202564000A0D5573696E67205061729B
:1008E000616D6574657220536574202564000A0D7E
:1008F00047656E65726174696E67206465666175CF
:100900006C74204D69786572205461626C65000AD0
:100910000D4D697865722D436F6E6669673A2027C1
:1009200025732720282575204D6F746F7273290059
:100930000A0D414343206E6F742063616C696272DB
:1009400061746564210D0A0000008F001E01AD0175
:100950003B02CA025803E603740402058F051B0616
:10096000A7063307BE074808D2085B09E3096B0AEC
:10097000F20A780BFD0B810C040D860D070E870E15
:10098000060F840F00107B10F5106E11E5115B123D
:10099000CF124213B31323149214FE146A15D31505
:1009A0003B16A11605176717C81727188318DE18F6
:1009B00037198E19E319361A871AD61A231B6E1B9C
:1009C000B61BFD1B411C831CC31C001D3C1D751D5B
:1009D000AB1DE01D121E421E6F1E9A1EC31EE91E95
:1009E0000D1F2E1F4D1F691F841F9B1FB01FC31F8C
:1009F000D31FE11FEC1FF51FFB1FFF1F002000008E
:100A000005000500040106010800060102000400BB
:100A100004000700070007000700070007000700A1
:100A200003010301050017010F01060009010A0176
:100A300019010501050119011A010F0100004E6F8E
:100A4000204572726F722020202020202020004E2E
:100A50006F7420636F6D70617469626C6520200033
:100A60004D4B334D6167206E6F7420636F6D706105
:100A7000004E6F20464320636F6D6D756E69636134
:100A80007400436F6D7061737320636F6D6D756E6D
:100A900069630047505320636F6D6D756E696361C4
:100AA00074696F00636F6D706173732076616C752C
:100AB00065202020005243205369676E616C206CD2
:100AC0006F73742020004643207370692072782071
:100AD0006572726F7220004E6F204E4320636F6DFF
:100AE0006D756E69636174004643204E69636B20C7
:100AF0004779726F2020202000464320526F6C6C93
:100B0000204779726F2020202000464320596177CA
:100B1000204779726F2020202020004643204E6914
:100B2000636B204143432020202020004643205275
:100B30006F6C6C204143432020202020004643203E
:100B40005A2D414343202020202020202000507295
:100B50006573737572652073656E736F72200049DB
:100B600032432046432D3E424C2D4374726C20008C
:100B7000426C204D697373696E672020202020200D
:100B8000004D69786572204572726F7220202020B6
:100B900020004361726566726565204572726F72EE
:100BA00020200047505320466978206C6F737420D2
:100BB000202020004D61676E6574204572726F724F
:100BC00020202020004D6F746F7220726573746155
:100BD000727420202000424C204C696D697461744D
:100BE000696F6E202020004750532052616E676568
:100BF00020202020202020004E6F2053442D4361D0
:100C000072642020202020200053442D4C6F676701
:100C1000696E67206572726F7200466C79696E67E3
:100C20002072616E676521202020004D617820418F
:100C30006C74697475646521202020004E6F204714
:100C400050532066697820202020202000636F6D9B
:100C500070617373206E6F742063616C2E002021AD
:100C600021204C69506F20766F6C7461676520217C
:100C70002120200020202020204D696B726F4B6FB7
:100C80007074657220202020200020202020202049
:100C90002020202020202020202020202020200074
:100CA00020202532692E253169562020002020255C
:100CB00032692E25316956202000414C543A2534A2
:100CC000696D20256300414C543A2534696D20201C
:100CD00000414C543A2D2D2D2D2000202025326925
:100CE0003A2530326920200020202532693A25300B
:100CF00032692020004449523A202533642563009C
:100D000043002000202025356920200020202535A3
:100D100069202000493A2532692E25316941200099
:100D20003A003A003A002D2D2D2D2D2D2D2D2D2B55
:100D30002D2D2D2D2D2D2D2D2D2D2D002D2D2D2D10
:100D40002D2D2D2D2D2D2D2D2D2D2D2D2D2D2D2DD3
:100D50002D003A005341543A25326420004449534F
:100D6000543A2533646D00442000334400212100AF
:100D70004D41473A25337525252000484D3A253306
:100D800064256320256300696E636C3A253264250F
:100D900063282532692900202020202532756D2FF7
:100DA000733A2020484D3A2533642563202563009B
:100DB0004552523A202532642021004552523A20B1
:100DC000002121204C69506F20766F6C746167653B
:100DD00020212100207777772E4D696B726F4B6F42
:100DE000707465722E6465202000202532693A25D2
:100DF00030326920202532692E253169562025346C
:100E0000696D416800202532693A25303269202019
:100E10002532692E25316956202534696D416800D7
:100E20004449523A253364256300414C543A2534F1
:100E3000696D00414C543A2534696D00414C543A77
:100E40002D2D2D2D2000256300484D3A2533642596
:100E5000632020444953543A2533646D20256300B0
:100E60005057523A2532692E25316941202825698B
:100E7000572920004346002020004750533A25328E
:100E8000756D2F73205341543A2564200020203380
:100E90004420004E4F4649580044475053200020FC
:100EA00020204E6F204E6176694374726C202020A2
:100EB00020202020002532692E2569202532692E28
:100EC0002569202532692E2569202532692E25695C
:100ED00041002533692025336920253369202533D6
:100EE00069256343002532692E2569202532692E44
:100EF000256941002532692E2569202532692E2574
:100F000069202532692E2569202532692E256941FF
:100F100000253369202533692563432020202020C4
:100F200020202000253369202533692025336920BE
:100F3000253369256343004552523A202532642007
:100F400021004552523A20002121204C69506F2047
:100F5000766F6C7461676520212100207777772E8A
:100F60004D696B726F4B6F707465722E64652020D3
:100F70000053657474696E673A25752025732000E7
:100F80004D696E3A2532692E253169562025732028
:100F900000414C543A00504F54493A2533752000D3
:100FA000284F4E29202000284F46462920004C4932
:100FB0004D495400564152494F0044495341424C17
:100FC00045440043463A0044495341424C4544009D
:100FD00020284F4E29200020284F46462900205423
:100FE00045414348004750533A0044495341424C1D
:100FF0004544002846524545290028484F4D45297B
:10100000002841494429200028484F4C4429002009
:1010100046533A257573656B2000484F4D45204176
:101020004C543A0025756D00484F4C4420004E69E1
:101030003A25346920526F3A25346920433A2533E2
:10104000690047733A2534692059613A253469208B
:101050000050313A2534692050323A253469203322
:101060003A2533690050343A2534692050353A2501
:10107000346920363A25336900434F55504C494E68
:1010800047204F46462120004C4F4F50494E4721A4
:1010900020004848212000434F4D50415353204FDA
:1010A0004646212000004F50515253545356574842
:1010B000005859005A5545464748410049424A4A56
:1010C0000000000000000000000000444C4D000043
:1010D0000000004E0000004B00430A0D7777772E8A
:1010E0004D696B726F4B6F707465722E646520284A
:1010F000632920486953797374656D7320476D6265
:1011000048000A0D74686520757365206F66207449
:1011100068697320736F66747761726520697320E4
:101120006F6E6C79207065726D6974746564200AE5
:101130000D6F6E206F726967696E616C204D696B0F
:10114000726F4B6F707465722D4861726477617253
:1011500065005573657200486F5454205634004141
:1011600043542044534C004A657469005370656BC6
:101170007472756D0050504D000A0D5265636569BB
:101180007665723A2000532E42757300756E6B6E51
:101190006F776E2E205573696E672050504D2E2E3E
:1011A0002E006E6F7420737570706F72746564209A
:1011B000627920686172647761726521000A0D4668
:1011C0006C69676874436F6E74726F6C0A0D486166
:1011D0007264776172653A25642E25640A0D536F37
:1011E0006674776172653A5625642E2564256320FE
:1011F000000011241FBECFEFD0E4DEBFCDBF12E050
:10120000A0E0B1E0E6E9F4E201E00BBF02C0079024
:101210000D92A63DB107D9F71BE0A6EDB2E001C0E3
:101220001D92AE3DB107E1F77AEAE2E0F0E081E23B
:1012300080935700D4907E010894E11CF11C20EFAC
:1012400037EF41E050E087016FE0DA01C9012F5F1D
:101250003F4F4F4F5F4FABBFFC018791F801819328
:101260008F01615067FFF1CFF7016EE08191782720
:101270007095615067FFFACF8889781729F0F7E9F0
:10128000DF1611F40000FECF0E941B0A0C944A9254
:101290000C94000088E891E09F938F9380E695E19D
:1012A0009F938F93E0913D05F0913E0509950F9036
:1012B0000F900F900F90089580918607E82FFF27D9
:1012C000EE0FFF1FE754F74F808191818D5E9F4F96
:1012D00014F010920201808191818A5B9F4FCCF4BF
:1012E000809102018823A9F481E08093020180911A
:1012F00071058F5F80937105853038F088EE93E03B
:1013000090930B0380930A0304C066E970E00E9487
:10131000043A8091710599279093090780930807F3
:1013200008951F93CF93DF93182F882389F08EEAB7
:1013300091E09F938F9380E695E19F938F93E09147
:101340003D05F0913E0509950F900F900F900F907D
:101350008091A907823308F044C084EF91E00E9495
:101360006F19EC01112329F0CE010E94781988230E
:10137000D9F3C2E0D0E026E530E080911F019091E2
:1013800020018217930730F02196255D3F4FC7302B
:10139000D10598F38091A9079927C89F9001C99F0B
:1013A000300DD89F300D1124209300011123D9F066
:1013B00068EC70E08C2F0E94043ADF93CF9386EBA9
:1013C00091E09F938F9380E695E19F938F93E091B7
:1013D0003D05F0913E0509958DB79EB706968DBFE8
:1013E00002C080930001112311F1809100016AE095
:1013F0000E949D91892F99279F938F93809100013F
:101400000E949D9199279F938F9381EC91E09F93E8
:101410008F9380E695E19F938F93E0913D05F09146
:101420003E0509952DB73EB7285F3F4F2DBFDF9191
:10143000CF911F910895CFEFD0E4DEBFCDBF8824B8
:10144000992414B815B8B7EEEB2EB3E0FB2E2EECB2
:101450003FEFE20EF31EF7FEFACF199B02C085E1C3
:1014600001C086E18093010181E887B93E9A8FEF40
:1014700088B98BE184B981E085B98EE38AB987E4C4
:101480008BB9469A84B7877F84BF8091600088615A
:10149000809360001092600084EC99E090930B03BD
:1014A00080930A0310921604109215041092BE083D
:1014B0001092BD08109218041092170410921A048A
:1014C0001092190420910101243128F084EC94E059
:1014D000A0E0B0E004C08BE095E0A0E0B0E0809335
:1014E0003C0190933D01A0933E01B0933F012A300F
:1014F00011F0243110F0289801C0289A2C3010F0F7
:10150000263111F4299A01C029980E94D8190E9405
:10151000A9190E9468150E9441360E94DA1D81E0D7
:101520000E94A4310E94A0680E943A720E942E8EEE
:10153000809101018C3010F0863111F4299A01C09C
:10154000299878940E94C33080914F0382608093E1
:101550004F03109252030E94504584EF91E00E9485
:101560006F197C0180914F0380FD05C0C7010E9467
:1015700078198823B9F385ED91E09F938F93A0E6C6
:10158000AA2EA5E1BA2EBF92AF92E0913D05F0914F
:101590003E05099580EA9FE00E946F197C01C0E03A
:1015A000D0E00F900F900F900F900BE518E0FFE048
:1015B000CF2EF8E0DF2E0E94504580914F0380FD32
:1015C00005C0C7010E9478198823B9F3F60180810C
:1015D0001816ACF40BC00E94504580914F0380FD5B
:1015E00005C0C7010E9478198823B9F3C7010E947A
:1015F0007819882321F4F8018081882364F7F801A1
:10160000808187FF19C02196DF93CF93219787EEC2
:1016100091E09F938F93BF92AF92E0913D05F0913F
:101620003E0509958091D7028F5F8093D7022DB731
:101630003EB72A5F3F4F2DBF219684E090E0C80E51
:10164000D91E085F1F4FCC30D10508F4B4CFC0E0DD
:10165000D0E008E518E0EFE0EE2EE8E0FE2EF8011D
:10166000838187FD1DC0F70180811816CCF4219677
:10167000DF93CF9321978AEE91E09F938F9380E63B
:1016800095E19F938F93E0913D05F0913E0509957B
:1016900082E0809308032DB73EB72A5F3F4F2DBFEE
:1016A000F801838180788383219624E030E0E20E84
:1016B000F31E085F1F4FCC30D10588F20E944A0903
:1016C000909184078091D702981728F4809157054C
:1016D00080618093570588E092E09F938F93C0E6E6
:1016E000D5E1DF93CF93E0913D05F0913E0509955B
:1016F00088EE93E00E946F197C010E94E01D0F901C
:101700000F900F900F90C7010E9478198823D9F38A
:1017100088E292E09F938F93DF93CF93E0913D0512
:10172000F0913E05099580E00E94E83A8091010120
:101730000F900F900F900F908A3011F0843110F0BD
:10174000289801C0289A80ED97E090930B0380932E
:101750000A0385E5809373058EE090E00E94E72EF2
:101760009927182F00278FE090E00E94E72E080F9E
:10177000111D1093DD020093DC028AE090E00E94CC
:10178000E72E9927182F00278BE090E00E94E72E84
:10179000080F111D1093DB020093DA020F5F1F4F39
:1017A00039F08091DC029091DD028F5F9F4F41F410
:1017B0001092DD021092DC021092DB021092DA022B
:1017C0008091DA029091DB029F938F938091DC02EB
:1017D0009091DD029F938F938DE292E09F938F9380
:1017E000DF93CF93E0913D05F0913E0509950E946E
:1017F000742388E893E19093370180933601C1E028
:10180000C09372058C2F0E9491098091AC070E94B1
:101810007A8D0E944A0980ED97E00E946F197C0141
:101820008AEF90E00E946F1983E08093E0061092A7
:10183000D6028091F3072DB73EB7285F3F4F2DBFEB
:1018400084FF02C0C093DE028091E002882311F081
:101850004798FECF80910E03882309F43DC2809102
:101860001101882309F438C210920E03809171058A
:10187000882319F00E945C0902C00E94A9480E94B6
:101880005045209101012A3011F0243110F02898A0
:1018900001C0289A80910904882331F080910904BD
:1018A0008150809309040EC080916F008062809304
:1018B0006F001092BA081092B9088091570588609D
:1018C000809357058091360190913701019790934D
:1018D0003701809336018091360190913701892B31
:1018E00021F0809150038823C9F1809136019091B5
:1018F0003701892BD9F40E94CE3185E090E0909396
:1019000037018093360180911A0790911B07019649
:1019100090931B0780931A078091570581608093ED
:1019200057058091E10682608093E106809109016C
:1019300090910A018F5F9F4FC1F480910804882322
:10194000A1F088EA91E690930B0380930A0380E864
:1019500090E090930A018093090107C02A3011F0AA
:10196000243110F0289801C0289A0E94E68E8091B8
:101970000E03882309F0B0C180911E05882319F059
:101980000E94BB81A9C180910F01882311F00E94A0
:10199000311A0E94AC150E94FA10C7010E947819F2
:1019A000882309F495C184E190E0E80EF91E0E94B5
:1019B000EF198091AC07863019F40E94597704C062
:1019C000843011F40E948B8280915003882349F067
:1019D000809157058260809357058091E10682606F
:1019E0000FC080910A0390910B03892B59F48091C9
:1019F000360190913701079728F08091E1068D7F9D
:101A00008093E1068091DE02882361F080910904D1
:101A1000873940F01092DE0288E893E190930B033F
:101A200080930A0380910401882321F081508093E0
:101A300004012EC080937D051092DD031092DC031B
:101A40001092DB031092DA031092D9031092D8039C
:101A5000809109048823E1F48091090190910A01A1
:101A60008F5F9F4FA9F42091DE02223089F088E930
:101A70009AE390930B0380930A0380E09CE0909399
:101A80000A0180930901222319F082E08093DE028B
:101A900080919901893C48F081508093990180910F
:101AA00057058B7F809357053FC080919A09882303
:101AB000F9F08091570584608093570589E0809301
:101AC000E4048091090190910A018F5F9F4F81F496
:101AD00080910804882361F088E99AE390930B03CE
:101AE00080930A0380E098EA90930A0180930901A9
:101AF0001092D6041092D5041092D4041092D304FC
:101B00001092D20410928D091092CC091092CB0938
:101B10001092CE091092CD098FEF9FEF9093CA09D2
:101B20008093C9091092990180910001282F3327D1
:101B300080911F019091200182179307CCF480912E
:101B4000D10380628093D1038091090190910A01B1
:101B50008F5F9F4FC1F480E797E190930B038093D1
:101B60000A0380E093E090930A01809309010BC07F
:101B700080910A0390910B03892B29F48091D10362
:101B80008F7D8093D1030E94976D84E08093090339
:101B90008091DF028F5F8093DF02813309F04FC0B5
:101BA0001092DF028091D10381FF0AC08091D80298
:101BB0009091D90201969093D9028093D8023FC0A8
:101BC0005AEA852E55E0952E8091290790912A0793
:101BD0009C01442737FD4095542F80911701909127
:101BE0001801A0911901B0911A01281739074A0765
:101BF0005B0734F48091290790912A0701961BC056
:101C00008091290790912A079C01442737FD409530
:101C1000542F8091170190911801A0911901B09152
:101C20001A0182179307A407B5074CF4809129077E
:101C300090912A07019790932A0780932907089487
:101C4000811C911C32E783163BE0930609F040C0EB
:101C5000882499242091DC023091DD022F5F3F4FD0
:101C60003093DD022093DC028091DA029091DB0256
:101C700001969093DB028093DA02832F9927682FD5
:101C80008EE090E00E94EF2E8091DC029091DD02C8
:101C90009070682F8FE090E00E94EF2E8091DA0222
:101CA0009091DB02892F9927682F8AE090E00E94AB
:101CB000EF2E8091DA029091DB029070682F8BE01A
:101CC00090E00E94EF2E84E190E00E946F197C0169
:101CD0000E94E76D0E94517280910903882309F0E8
:101CE000B3CD0E94C168B0CD1F920F920FB60F9274
:101CF00011248F939F93EF93FF9380910601882384
:101D0000E1F48091FA029091FB0201969093FB021C
:101D10008093FA02FC01EF5CF94FE081ED3019F09D
:101D20008F3A910539F41092FB021092FA0281E089
:101D300080930601E093C60004C01092FB0210924B
:101D4000FA02FF91EF919F918F910F900FBE0F902C
:101D50001F9018951F920F920FB60F9211242F9378
:101D60003F934F935F936F937F938F939F93AF9323
:101D7000BF93CF93EF93FF9390E08091E002813087
:101D800029F48091C6008093CE00CCC08091E002FF
:101D9000823029F48091C60080938005C3C0809171
:101DA000C6008093F202509100035F3A10F09093C6
:101DB00001038091F2028D3009F065C0809101032A
:101DC000823009F060C090930103852F99278058D5
:101DD0009A4FFC01329740812091FC023091FD0224
:101DE000241B3109DC0111978C91281B3109C90191
:101DF0009F709093FD028093FC0246E09695879534
:101E00004A95E1F7982F935C9093FE022F73307000
:101E1000235C2093FF028081981729F48C91281766
:101E200011F491E006C090E08091EF028F5F809303
:101E3000EF02C091F102CC2309F074C0992309F498
:101E400071C081E08093F102580F5093EE0251501F
:101E5000E52FFF27E058FA4F8DE0808380918205BF
:101E6000823509F05FC00E94742388E190E02CE085
:101E70000FB6F894A895809360000FBE2093600081
:101E8000C09308034FC020910103822F992781300E
:101E90009105F9F0823091051CF4892B21F040C0A6
:101EA000029711F13DC08091F202833239F48091A2
:101EB000F102882319F481E0809301038091F202FA
:101EC0008093800581E0809300038091F20299273E
:101ED00022C02F5F20930103E52FFF27E058FA4F20
:101EE0008091F202808309C0E52FFF27E058FA4F66
:101EF0008091F20280835F3A20F45F5F5093000389
:101F000002C0109201032091F2028091FC02909194
:101F1000FD02820F911D9093FD028093FC0202C08E
:101F200010920103FF91EF91CF91BF91AF919F91DB
:101F30008F917F916F915F914F913F912F910F9072
:101F40000FBE0F901F901895AC01A0E0B0E09D016E
:101F5000A817B90748F4E1E3F6E08191280F311D95
:101F60001196A417B507C8F33F70FD01EF5CF94F58
:101F7000C90156E0969587955A95E1F7835C808371
:101F80001196FD01EF5CF94F2F733070822F835C47
:101F90008083AE5CB94F8DE08C93109206018091E6
:101FA00031068093C6000895A0E0B0E0EAEDFFE0BE
:101FB0000C9416922C859D850E85BB2483E280931C
:101FC00031069F59909332062093330633E0E32E77
:101FD000F12C002309F49EC0CF84D888BE016D5E29
:101FE0007F4FA989BA890150109709F493C01097BF
:101FF000B9F0F601EB0DF11DB3949081119791F4B6
:10200000002349F1FB016E5F7F4FDB01C080D1806F
:102010006E5F7F4F0D90BC91A02DBB24015002C07C
:1020200090E019C01097B9F0F601EB0DF11DB394D3
:102030004081119791F4002341F1FB016E5F7F4FC6
:10204000DB01C080D1806E5F7F4F0D90BC91A02DD1
:10205000BB24015002C040E018C01097B1F0F60157
:10206000EB0DF11DB3941081119781F4002371F0F1
:10207000FB013296DB01CD90DC90BF016E5F7F4F9C
:10208000A081B181BB24015001C010E0F701EF5CD9
:10209000F94F892F86958695835C80830894E11C8F
:1020A000F11CF701EF5CF94F892F9927837090702D
:1020B00024E0880F991F2A95E1F755279A0194E0AB
:1020C000369527959A95E1F7822B835C8083089457
:1020D000E11CF11CF701EF5CF94F4F705070440F99
:1020E000551F440F551F812F992726E096958795F8
:1020F0002A95E1F7842B835C80830894E11CF11C12
:10210000F701EF5CF94F1F73135C10830894E11C17
:10211000F11C6ACFC7010E94A40FE9E00C9432922F
:10212000A3E07A2F4091EE024650442309F458C0B0
:10213000E72FFF27E058FA4F80818D537F5FE72F0D
:10214000FF27E058FA4F20812D537F5FE72FFF27AD
:10215000E058FA4F30813D537F5FE72FFF27E0586B
:10216000FA4F60816D537F5F9927880F991F880F01
:10217000991F522F52955F70582B822F99278F707D
:102180009070F4E0880F991FFA95E1F7232F2695B8
:102190002695282B832F992783709070E6E0880F6F
:1021A000991FEA95E1F7682B41504F3FC9F0EA2F9C
:1021B000FF27E058FA4F5083AF5F41504F3F81F007
:1021C000EA2FFF27E058FA4F2083AF5F41504F3F7F
:1021D00039F0EA2FFF27E058FA4F6083AF5FA5CFB1
:1021E00083E895E09093ED028093EC02A350A093D6
:1021F000EB020895A2E0B0E0E0E0F1E10C941C9263
:102200008091F102882309F457C40E9490108091B4
:102210008105823609F023C3809182059927803792
:10222000910509F4AFC081379105C4F48A36910550
:1022300009F480C28B36910544F48B34910571F119
:102240008636910509F45FC10AC38D36910509F4FC
:1022500069C08E36910509F44DC001C384379105DC
:1022600041F1853791054CF48137910509F491C00E
:102270008337910509F4DFC0F2C28737910509F46D
:102280001BC2883791052CF48537910509F4D7C115
:10229000E6C28937910509F46DC1E1C2E091EC0213
:1022A000F091ED028081918190938B0180938A015E
:1022B000D6C28091EE02A091EC02B091ED02853180
:1022C00040F080E1EBE5F5E00D9001928A95E1F7B1
:1022D0000DC08D919D910D90BC91A02D80935B05BB
:1022E00090935C05A0935D05B0935E0580EF8093AD
:1022F000E9024BC0809106018823E1F38DE490E070
:102300009F938F9382E098E09F938F9381E08F93C8
:102310008F938EE48F930E94D40F8DB79EB707964C
:102320008DBF9DC2A091EC02B091ED021C911130C5
:1023300081F48DE4E2E0F8E00D9001928A95E1F7F6
:102340000E9400301983809157058F7E8093570536
:1023500001C01982809106018823E1F381E090E0B9
:102360009F938F93CE0101969F938F9381E08F93DC
:102370008F938DE48F930E94D40FADB7BEB717969D
:10238000ADBF6DC281E08093F4028FEF80930401B2
:1023900066C2E091EC02F091ED02E0818E2F8A504E
:1023A0008A3058F48983882311F481E003C0863091
:1023B00010F085E0898361E00EC08E2F84518A3051
:1023C00070F48983882311F481E003C0863010F013
:1023D00085E0898360E089810E94803012C0E983B2
:1023E000EF3F19F40E94633089838981882311F4B7
:1023F00081E003C0863010F085E0898389810E94E6
:10240000052F809106018823E1F38CE790E09F93EC
:102410008F9385E897E09F938F9381E090E09F935F
:102420008F93CE0101969F938F9382E08F9381E0EB
:102430008F9381E577C12091EC023091ED02D901B3
:102440008C918150853008F045C0F90181818D352E
:1024500009F040C0809108048823E1F52F5F3F4FC9
:102460008CE7E5E8F7E0D9010D9001928A95E1F754
:10247000F90182910E94702F8091C6079927AA279F
:10248000BB27BC01CD0124EC39E040E050E00E94C4
:102490007E91DC01CB018093820190938301A09314
:1024A0008401B09385018091C7079927AA27BB278C
:1024B000BC01CD010E947E91DC01CB0180937E01A5
:1024C00090937F01A0938001B09381010E946330BB
:1024D000898301C01982809106018823E1F381E09C
:1024E00090E09F938F93CE0101969F938F9381E00D
:1024F0008F938F9383E58F930E94D40F8DB79EB7F0
:1025000007968DBF26C0E091EC02F091ED02E081CC
:102510008E2F8150853018F48E2F0E94052F0E9437
:1025200063308983809106018823E1F381E090E0A4
:102530009F938F93CE0101969F938F9381E08F930A
:102540008F9386E48F930E94D40FADB7BEB71796D2
:10255000ADBF80910804882329F46EE670E089817C
:102560000E94043A80E00E9491098091AC070E9489
:102570007A8D75C1E091EC02F091ED02808199278E
:1025800087FD90959093D4088093D30881819927F3
:1025900087FD90959093D6088093D50882819927DE
:1025A00087FD90959093D8088093D70883819927C9
:1025B00087FD90959093DA088093D90884819927B4
:1025C00087FD90959093DC088093DB08858199279F
:1025D00087FD90959093DE088093DD08868199278A
:1025E00087FD90959093E0088093DF088781992775
:1025F00087FD90959093E2088093E1088085992764
:1026000087FD90959093E4088093E308818599274E
:1026100087FD90959093E6088093E5088285992739
:1026200087FD90959093E8088093E7088385992724
:1026300087FD90959093EA088093E90810C1E09196
:10264000EC02F091ED0280810E949A358A83882302
:1026500019F481E0898301C01982809106018823E1
:10266000E1F388E090E09F938F9380E598E09F935B
:102670008F9321E030E03F932F938091EC02909173
:10268000ED029F938F933F932F93CE0102969F93DA
:102690008F933F932F93CE01820F931F9F938F931E
:1026A00084E08F9381E08F9385E58F930E94D40F10
:1026B000EDB7FEB773963CC08091EB02893008F409
:1026C000CEC02091EC023091ED022F5F3F4F88E0A9
:1026D000A0E5B8E0F90101900D928A95E1F7D901E2
:1026E0008E910E94F0348A83882319F481E08983D3
:1026F00001C01982809106018823E1F321E030E0D6
:102700003F932F93CE0102969F938F933F932F93E6
:10271000CE01820F931F9F938F9382E08F9381E06E
:102720008F9387E58F930E94D40FEDB7FEB73B964A
:10273000EDBF95C080910804882309F090C00E94E5
:102740002D8D8983823019F0843009F088C020E40F
:1027500030E0F8948091C1008F738093C100809124
:10276000C9008F738093C9008091C100877E8093D8
:10277000C1008091C900877E8093C9008091C80004
:1027800087FF03C08091CE00F9CF8091C00087FF02
:1027900003C08091C600F9CFE091EC02F091ED0208
:1027A000E081E13021F482E08093E0022EC0E43643
:1027B00011F421E830E081E08093E002832F992733
:1027C0008093CD002093CC008091CD008093C500F4
:1027D0008091CC008093C4008091CA008F7D80934B
:1027E000CA008091CA008F7E8093CA008091C90080
:1027F0008B7F8093C9008091CA0084608093CA0057
:102800008091CA0082608093CA008091CA00877F4D
:102810008093CA008091C200877F8093C20080911C
:10282000C9008E7F8093C9008091C1008861809328
:10283000C1008091C90088618093C9008091C10066
:1028400080688093C1008091C90080688093C9002E
:1028500010926E0010926F00109270007894809128
:10286000820599278436910509F4BBC08536910508
:10287000ACF48136910509F46FC0823691052CF4D1
:102880008B34910509F45DC00FC18236910509F4BE
:1028900070C08336910509F47FC006C18C3691055E
:1028A00009F4EDC08D3691054CF48736910509F495
:1028B000F8C08836910509F4B2C0F6C08437910596
:1028C00029F08637910509F4E8C0EEC08091EE0248
:1028D000A091EC02B091ED02803140F080E1EBE597
:1028E000F5E00D9001928A95E1F70DC08D919D91D3
:1028F0000D90BC91A02D80935B0590935C05A093F7
:102900005D05B0935E05809106018823E1F31F9277
:10291000809103018F9384E58F930E94D40F8AEFF7
:102920008093E9028FEF8093040180EA9FE00E9488
:102930006F199093E2028093E1020F900F900F9035
:10294000B3C0E091EC02F091ED028081918190930F
:102950008B0180938A01A8C0E091EC02F091ED0216
:10296000808180930501803298F08FE1809305018A
:102970000FC0A091EC02B091ED028BE0E3E7F5E02F
:102980000D9001928A95E1F780917C058093220752
:102990008FEF8093040188C08091E5029091E60258
:1029A000892B89F4E091EC02F091ED02E081EE23B5
:1029B00051F08AE0E89FC00111240E946F199093A2
:1029C0004E0580934D05E091EC02F091ED0290816F
:1029D0008AE0989FC00111249093E6028093E5025B
:1029E00015C08FEF80930401E091EC02F091ED02AD
:1029F00090818AE0989FC00111249093E80280930F
:102A0000E702892B19F081E08093F60280EA9FE0CB
:102A10000E946F199093E2028093E10245C08FEF0C
:102A200080930401E091EC02F091ED02908197FD1A
:102A300008C082E08093F3021092E4021092E30255
:102A40001AC0909580914803892B80934803918107
:102A50008AE0989FC00111249093E4028093E302DE
:102A600084E08093F30280EA9FE00E946F199093C4
:102A7000E2028093E10281E08093F70215C08FEFBC
:102A800080930401E091EC02F091ED02808180934B
:102A9000490381E08093F80207C081E08093F5024A
:102AA00003C081E08093F9021092F1021092ED02CE
:102AB0001092EC021092EB02E3E0CE5F0C9438929D
:102AC000982F8091C00085FFFCCF9093C600089599
:102AD0000F931F9388E18093C1008091C0008260B2
:102AE0008093C0008091C10080688093C100809174
:102AF000C10080648093C10000E010E00093C50035
:102B00008AE290E08093C4008091E7029091E8020D
:102B10000E946F199093500580934F058CED90E0C3
:102B20000E946F1990937F0580937E051092510546
:102B30008AE58093520584E0809355058BE080936D
:102B40005305109254051093ED020093EC0210927D
:102B5000EB021F910F910895A0E1B0E0E2EBF5E1E7
:102B60000C94199280910601882309F4C1C28091C6
:102B7000E1029091E2020E947819882361F010929C
:102B8000E4021092E3021092E8021092E70210921F
:102B9000E6021092E5028091E3029091E402892B13
:102BA00041F080912F06909130060E947819882379
:102BB00029F48091F702882309F460C0809106010E
:102BC000882309F45BC08091F30204E317E08430AA
:102BD000A8F00E948A2380E590E09F938F931F9333
:102BE0000F9381E08F938F9388E48F930E94D40F8B
:102BF0002DB73EB7295F3F4F2DBF34C010924A0317
:102C00008FE494E09F938F938DE793E29F938F934C
:102C1000E0913D05F0913E05099584E190E09F9398
:102C20008F931F930F9381E090E09F938F9383EF97
:102C300092E09F938F9382E08F9381E08F9388E45B
:102C40008F930E94D40F8091F302982F8F5F80930F
:102C5000F3022DB73EB7215F3F4F2DBF943010F0E8
:102C60001092F3028091E3029091E4020E946F19A6
:102C70009093300680932F061092F7028091F8020D
:102C8000882351F180910601882331F10E948A2323
:102C900080E590E09F938F9384E397E09F938F93D9
:102CA00021E030E03F932F9381E291E09F938F9357
:102CB0003F932F9389E493E09F938F9383E08F93C7
:102CC00081E08F938CE48F930E94D40F1092F802CE
:102CD0008DB79EB70F968DBF8091F5028823D1F0F6
:102CE000809106018823B1F08AE090E09F938F9352
:102CF00081E595E09F938F9381E08F938F9386E595
:102D00008F930E94D40F1092F5022DB73EB7295F22
:102D10003F4F2DBF8091F9028823D9F080910601A1
:102D20008823B9F08BE090E09F938F9383E795E041
:102D30009F938F9381E08F93809103018F9387E41A
:102D40008F930E94D40F1092F9028DB79EB7079609
:102D50008DBF80917E0590917F050E947819882310
:102D600009F461C080910601882309F45CC0809158
:102D7000A1079927880F991F880F991F7C010027A9
:102D8000F7FC0095102F8091630490916404A0914A
:102D90006504B0916604BC01CD01A80197010E94B1
:102DA000F29130936C0520936B0580915B049091B8
:102DB0005C04A0915D04B0915E04BC01CD01A8014A
:102DC00097010E94F29130936E0520936D058091DA
:102DD000E60380936F058091E5038093700588E09A
:102DE00090E09F938F938BE695E09F938F9381E084
:102DF0008F9383E08F938BE68F930E94D40F809103
:102E000071052DB73EB7295F3F4F2DBF853018F0B4
:102E100086E08093710583E690E00E946F1990939D
:102E20007F0580937E058091E7029091E802892BCF
:102E300041F080914F05909150050E9478198823A8
:102E400021F48091F602882339F1809106018823CC
:102E500019F10E94EE3882E490E09F938F9380EE08
:102E600096E09F938F9381E08F938F9384E48F9369
:102E70000E94D40F1092F6028DB79EB707968DBFB1
:102E80008091E7029091E802009731F00E946F195B
:102E90009093500580934F058091E5029091E60252
:102EA000892B09F4B8C080914D0590914E050E9480
:102EB0007819882309F4AFC080910601882309F4AA
:102EC000AAC08091A1079927880F991F880F991F81
:102ED0007C010027F7FC0095102F809163049091EE
:102EE0006404A0916504B0916604BC01CD01A80101
:102EF00097010E94F2913093400520933F05809105
:102F00005B0490915C04A0915D04B0915E04BC01EF
:102F1000CD01A80197010E94F291309342052093C0
:102F20004105209182093091830940918409509193
:102F30008509DA01C90163E0880F991FAA1FBB1F29
:102F40006A95D1F7820F931FA41FB51F820F931F9D
:102F5000A41FB51F20913C0130913D0140913E01DD
:102F600050913F01BC01CD010E94F2913093440584
:102F70002093430580912B0490912C04A0912D0463
:102F8000B0912E0449E0B595A795979587954A95F8
:102F9000D1F7809345058091270490912804A09152
:102FA0002904B0912A0439E0B595A795979587959E
:102FB0003A95D1F78093460580913304909134047B
:102FC000A0913504B091360429E0B595A795979561
:102FD00087952A95D1F7809347058EE090E09F93DF
:102FE0008F938FE395E09F938F9381E08F938F93DF
:102FF00083E48F930E94D40F8091E5029091E602C2
:103000000E946F1990934E0580934D052DB73EB7E2
:10301000295F3F4F2DBF809105018F3F71F19927A7
:1030200004E0880F991F0A95E1F7815B9D4F40E10D
:1030300050E0BC01CE0101960E94C88F80E190E073
:103040009F938F93CE0101969F938F9381E090E0A1
:103050009F938F9385E091E09F938F9382E08F936E
:1030600081E08F9381E48F930E94D40F8FEF809340
:1030700005018DB79EB70B968DBF809122078823DF
:10308000D1F0809106018823B1F081E090E09F9318
:103090008F9382E297E09F938F9381E08F938F933A
:1030A00082E48F930E94D40F109222072DB73EB76F
:1030B000295F3F4F2DBF8091F4028823C9F0809192
:1030C00006018823A9F084E390E09F938F9389EB16
:1030D00098E09F938F9381E08F938F9380E58F93F8
:1030E0000E94D40F1092F4028DB79EB707968DBF41
:1030F000E6E0C05F0C9435921F920F920FB60F92CC
:1031000011242F933F935F936F937F938F939F939C
:10311000AF93BF93EF93FF9320E08091090388233F
:1031200029F0809109038150809309038091F8046C
:10313000882319F081508093F80480911103815005
:10314000809311038F3F09F05BC089E080931103E6
:1031500080910F0390911003019690931003809338
:103160000F03809110018F5F81708093100188237D
:1031700019F481E080930E03349903C081E08093B9
:10318000120380910A0390910B03892B21F1809106
:103190000A0390910B030B9750F080910A039091D2
:1031A0000B030A9790930B0380930A0304C01092B9
:1031B0000B0310920A0380910A0390910B03209154
:1031C000090130910A0182239323892B11F021E018
:1031D00008C020E006C08FEF9FEF90930A01809314
:1031E000090180910101222331F08A3011F45A9AA9
:1031F00007C0479A05C08A3011F45A9801C0479811
:1032000080911203882309F45AC020919901222346
:1032100009F055C08091720983FF51C086B199278A
:10322000FC01E071F07084FF13C080910C03909159
:103230000D03019690930D0380930C0380910C0372
:1032400090910D03895E9340D0F12093120337C013
:1032500080910C0390910D03892B69F180910C03EF
:1032600090910D038A56914030F580910C03909116
:103270000D0369E270E00E94A99180910C03909186
:103280000D03860F971F90930D0380930C0380917D
:103290000C0390910D030B9750F080910C039091CB
:1032A0000D030A9790938B0180938A0104C0F093D9
:1032B0008B01E0938A0110920D0310920C03FF9191
:1032C000EF91BF91AF919F918F917F916F915F919E
:1032D0003F912F910F900FBE0F901F901895209146
:1032E0000F0330911003280F391FC901019608956B
:1032F00020910F0330911003821B930B892F992784
:103300008695807490700895CF93DF930E946F1913
:10331000EC01CE010E9478198823D9F3DF91CF9177
:103320000895CF93DF930E946F19EC0109C080913B
:103330001101882329F0909311018FEC80937A007A
:10334000CE010E947819982F882389F3DF91CF91BD
:1033500008959FB7F8945F983E9A469A8091B0007E
:103360008F708093B0008091B00083608093B00034
:103370008091B1008B738093B1008091B1008B601C
:103380008093B1001092B2008FEF8093B3008091D0
:10339000B00080688093B000809170008A7F809335
:1033A0007000809170008260809370009FBF0895CC
:1033B0008AE090E00E946F1990932407809323077E
:1033C00082E085BD83EA84BD17BC84EB88BD86E0BE
:1033D00086BD80916E00816080936E00089580911B
:1033E000F2072091690182FF30C09091B5078CE30C
:1033F000989FB00111249091B40780E5989FA00197
:103400001124922F905897FD9D5F9595959586E094
:103410009802C00111242091070130910801281B56
:10342000390B3093080120930701421753072CF002
:10343000509308014093070108952617370784F039
:1034400070930801609307010895822F992736E051
:10345000880F991F3A95E1F790930801809307012F
:103460000895A0E0B0E0E7E3FAE10C9418928091AF
:10347000BC07E82FFF27EE5BFE4F9681D08080913E
:103480000F01A92FBB27A7FDB095CB2FDB2F8130D4
:1034900009F017C1209163043091640440916504E0
:1034A00050916604BD01CE010E947E9197FF04C039
:1034B00061587F4F8F4F9F4F7B018C01C7E015955F
:1034C0000795F794E794CA95D1F78D2D992787FD35
:1034D0009095A92FB92F20915B0430915C04409105
:1034E0005D0450915E04BC01CD010E947E9197FF66
:1034F00004C061587F4F8F4F9F4FB7E095958795D8
:1035000077956795BA95D1F7F801E701C61BD70BF8
:10351000E80BF90B2091DD043091DE04C901A3E032
:10352000880F991FAA95E1F7821B930BAA2797FD95
:10353000A095BA2FC81BD90BEA0BFB0B8091670132
:103540009927AA27BB27BC01CD019E01AF010E948C
:103550007E9197FF04C061507E4F8F4F9F4FFC01BB
:10356000EB0179E0F595E795D795C7957A95D1F771
:103570001091F207609107017091080112FF05C0D8
:1035800070930E0160930D0118C040910D01509190
:103590000E018091BB07282F3327CB01841B950B8D
:1035A000B9010E94BD9180910D0190910E01860F8D
:1035B000971F90930E0180930D0110FF14C080910E
:1035C0000D0190910E0197FD0F9664E095958795FA
:1035D0006A95E1F7AA2797FDA095BA2FC80FD91FC2
:1035E000EA1FFB1F15C080910D0190910E0197FD00
:1035F0000F9654E0959587955A95E1F7AA2797FD80
:10360000A095BA2F8C1B9D0BAE0BBF0BFD01EC01DF
:103610002091EF07222321F1332780910403909119
:103620000503829FA001839F500D929F500D11248E
:10363000CA01AA2797FDA095BA2F8C0F9D1FAE1F18
:10364000BF1F2F5F3F4F442737FD4095542FBC01CC
:10365000CD010E94F291309305032093040304C02E
:10366000D0930503C09304038091B407282F332718
:10367000220F331F220F331F809104039091050303
:10368000821793077CF08091B507282F3327220FEC
:10369000331F220F331F80910403909105032817D5
:1036A000390724F43093050320930403809101012A
:1036B000843108F4F7C080910F018F5F80930F0170
:1036C000F3C020915B0430915C0440915D04509103
:1036D0005E04BD01CE010E947E9197FF04C0615837
:1036E0007F4F8F4F9F4F7B018C0187E0159507958A
:1036F000F794E7948A95D1F78D2D992787FD9095BA
:10370000A92FB92F2091630430916404409165047E
:1037100050916604BC01CD010E947E919B01AC01D9
:1037200097FF04C021583F4F4F4F5F4FC7E055955B
:10373000479537952795CA95D1F72E0D3F1D401F08
:10374000511F809166019927AA27BB27BC01CD0193
:103750000E947E9197FF04C061507E4F8F4F9F4F14
:10376000FC01EB01B9E0F595E795D795C795BA95BA
:10377000D1F7809168019927A6E0880F991FAA9533
:10378000E1F740910B0150910C012091BB073327C9
:10379000841B950BB9010E94BD9180910B01909102
:1037A0000C01860F971F90930C0180930B01809161
:1037B000F20781FF14C080910B0190910C0197FDDD
:1037C0000F9674E0959587957A95E1F7AA2797FD6E
:1037D000A095BA2FC80FD91FEA1FFB1F15C08091F3
:1037E0000B0190910C0197FD0F9664E095958795DC
:1037F0006A95E1F7AA2797FDA095BA2F8C1B9D0B20
:10380000AE0BBF0BFD01EC012091F007222321F14B
:1038100033278091020390910303829FA001839F2D
:10382000500D929F500D1124CA01AA2797FDA09513
:10383000BA2F8C0F9D1FAE1FBF1F2F5F3F4F442716
:1038400037FD4095542FBC01CD010E94F291309379
:1038500003032093020304C0D0930303C093020325
:103860008091B807282F3327220F331F220F331FD1
:103870008091020390910303821793077CF080915B
:10388000B907282F3327220F331F220F331F8091B0
:103890000203909103032817390724F4309303039C
:1038A0002093020310920F01E7E0CDB7DEB70C942E
:1038B00034921F920F920FB60F9211242F933F93C1
:1038C0004F935F938F939F93EF93FF9380910101A9
:1038D00090911303843108F04CC0992309F029C159
:1038E0008091B00086FF24C08091B0008F7B8093D0
:1038F000B000809104039091050387559E4F9093EB
:1039000007038093060325E08D3D920718F08CEDA8
:1039100095E005C08757914030F487E791E0909398
:103920000703809306038091060390910703C2C0AA
:103930008091B00080648093B0008091BA07282FF6
:1039400033278DED96E0289FA001299F500D389FC9
:10395000500D1124CA012091140330911503821BCC
:10396000930B909307038093060381E080930F01EC
:10397000DDC0992309F0DDC08091B00086FF9FC0B3
:103980008091B0008F7B8093B000E091160320916E
:10399000BA07EE23D9F433278DED96E0289FA001D6
:1039A000299F500D389F500D1124CA0120911403F6
:1039B00030911503821B930B9093070380930603AA
:1039C0001092150310921403469AB0C02E1738F4C3
:1039D0008AE090E09093070380930603A7C089EAEA
:1039E00093E090930703809306038E2F99278330EB
:1039F0009105D9F08430910534F48130910549F076
:103A0000029761F020C08430910591F0059799F0FC
:103A10001AC0809104039091050304C080910203B1
:103A20009091030387559E4F1DC080914E0905C09C
:103A30008091270902C0809157099927880F991F03
:103A4000880F991FEFCFFF27EE0FFF1FE754F74FA7
:103A500020813181220F331F80910603909107034B
:103A6000820F931F909307038093060380910603B0
:103A70009091070355E08D3D950718F08CED95E08A
:103A800005C08757914030F487E791E09093070392
:103A90008093060320910603309107032C5B30408E
:103AA000309307032093060380911403909115032C
:103AB000820F931F909315038093140337C0809156
:103AC000B00080648093B0008CEB90E0909307038B
:103AD00080930603809114039091150384549F4FA3
:103AE000909315038093140380910803882321F099
:103AF00080910904882321F480910803823011F415
:103B0000469801C0469A809116038F5F80931603F2
:103B1000282F33278091BA07992701968217930798
:103B20002CF481E080930F011092160381E08093C2
:103B30001303209106033091070341E02F37340728
:103B400030F08FEF8093B3002F5F30400FC02F3FD6
:103B50003105C9F0C0F0A9014F5F50404F37510502
:103B600050F480E88093B30020583040309307032E
:103B70002093060312C08FEF8093B3005093070386
:103B8000409306030AC0809106038093B30010920D
:103B900007031092060310921303FF91EF919F9178
:103BA0008F915F914F913F912F910F900FBE0F908A
:103BB0001F90189510927C008FEC80937A000895E6
:103BC000CF93DF9310921B0386E987BD83E090E0DB
:103BD0000E94E72EC82F863E08F4C65FC8BD84E663
:103BE00090E00E94911980911501909116018152E7
:103BF000934010F0C0EF02C0C530F8F0C8BD82E3BA
:103C000090E00E94911984E694E09F938F9380E660
:103C100095E19F938F93E0913D05F0913E050995C5
:103C200080911501909116010F900F900F900F90B9
:103C30008152934010F4C550DFCF6C2F83E090E0A9
:103C40000E94EF2ECF3018F0CCE8D0E002C0C0E0E8
:103C5000D0E0CA3FD105F8F4C7BD82E390E00E94EE
:103C6000911986E694E09F938F9380E695E19F9368
:103C70008F93E0913D05F0913E05099580911501E6
:103C8000909116010F900F900F900F9080529340DB
:103C900010F02196DECFC09331078091920780FF0C
:103CA00009C08C2F8A508B3E28F080915605806485
:103CB00080935605C7BD8CE291E00E949119DF9177
:103CC000CF910895EF92FF921F93CF9310E080ED74
:103CD00097E00E946F197C01CCE8133019F4CB30C7
:103CE00008F0C9E010E080912A0390912B038C5FCB
:103CF000934024F48091140181500AC080912A03DA
:103D000090912B038750944034F0809114018F5F81
:103D10008093140101C011E0809128039091290340
:103D20008C5F934024F48091130181500AC08091EC
:103D30002803909129038750944034F08091130117
:103D40008F5F8093130101C01F5F809126039091C4
:103D500027038C5F934024F48091120181500AC0A4
:103D6000809126039091270387509440C4F080915E
:103D700012018F5F8093120113C088E694E09F9335
:103D80008F9380E695E19F938F93E0913D05F091AD
:103D90003E0509950F900F900F900F905FC01F5F29
:103DA00082E18093550380914F038E7F80934F0370
:103DB00085EA8093BC00809114018A3040F48091A0
:103DC00056058160809356058AE0809314018091A6
:103DD0001401863F40F0809156058160809356051E
:103DE00085EF80931401809113018A3040F4809113
:103DF00056058260809356058AE080931301809176
:103E00001301863F40F080915605826080935605ED
:103E100085EF80931301809112018A3040F48091E4
:103E200056058460809356058AE080931201809144
:103E30001201863F40F080915605846080935605BC
:103E400085EF8093120180915503882339F0C701D3
:103E50000E947819882309F090CFF5CF10921101B4
:103E60008FEC80937A00809111018823E1F3CA30AE
:103E700020F48AE090E00E949119C15009F02DCF02
:103E800086E490E00E949119CF911F91FF90EF90EE
:103E900008951F920F920FB60F921124EF92FF9286
:103EA0000F931F932F933F934F935F936F937F9342
:103EB0008F939F93AF93BF93EF93FF9380913303BF
:103EC000282F3327442755278F5F80933303F90129
:103ED0002231310508F0E3C3EA5BFF4F0C944492B2
:103EE000809178009091790046C0809178009091FF
:103EF000790047C1809178009091790090933603C2
:103F00008093350372C180916C0490916D0420916F
:103F1000780030917900821B930B90932607809351
:103F20002507809125079091260790934003809361
:103F30003F0379C1809178009091790020916E04BF
:103F400030916F04821B930B9093300780932F075F
:103F500080912F0790913007909342038093410303
:103F6000A0C38091390390913A0320917800309159
:103F70007900820F931F90933A038093390381E075
:103F800091C380913703909138032091780030914C
:103F90007900820F931F909338038093370384E056
:103FA00081C38091F30783FF1AC080911F01909114
:103FB00020019C01220F331F280F391F40917800E8
:103FC000509179008BE090E0489FB001499F700DBF
:103FD000589F700D1124CB016EE170E00FC08091ED
:103FE0001F01909120019C01220F331F280F391FC0
:103FF000809178009091790063E070E00E94A9912F
:10400000260F371F36952795369527953093200133
:1040100020931F0185E046C380917800909179003C
:104020004091680450916904841B950B909321037F
:10403000809320038091200390912103029704F143
:1040400072E04E3E570784F4209134032B5F209397
:10405000340325508091D2039091D303845F914023
:1040600018F4215F2093340380913403853684F162
:104070004F5F5F4F5093690440936804845626C095
:1040800080912003909121038F5F9F4F0CF572E088
:1040900047325707ECF02091340325502093340326
:1040A0002B5F8091D2039091D303845F914018F4E9
:1040B0002F5020933403809134038C394CF44150B9
:1040C000504050936904409368048C5980933403A2
:1040D000809178009091790090932807809327072A
:1040E00080912003909121039C01442737FD409546
:1040F000542F8091230490912404A0912504B09121
:104100002604820F931FA41FB51F8093230490934E
:104110002404A0932504B093260420912304309115
:104120002404409125045091260457FF04C02150D7
:104130003C4F4F4F5F4F6AE0559547953795279510
:104140006A95D1F78091230490912404A0912504CD
:10415000B0912604821B930BA40BB50B8093230410
:1041600090932404A0932504B09326042EC180913B
:104170003703909138032091780030917900820FB5
:10418000931F9093380380933703109232038CC2AD
:10419000809101018A3071F48091780090917900CA
:1041A0002091350330913603820F931F0196969527
:1041B000879517C04091350350913603843158F0EC
:1041C0002091780030917900240F351F8FEF97E010
:1041D000821B930B06C08091780090917900840F28
:1041E000951F909327038093260386E05BC28091FE
:1041F0006C0490916D042091780030917900821BBD
:10420000930B909326078093250780912507909123
:10421000260720913F0330914003820F931F909314
:1042200025038093240387E03DC28091780090911C
:10423000790020916E0430916F04821B930B909350
:10424000300780932F0780912F079091300720919E
:10425000410330914203820F931F90932303809375
:1042600022031FC22091390330913A0380917800D4
:1042700090917900280F391F30933A032093390326
:10428000809101018A3019F4220F331F04C0220FDC
:10429000331F220F331F30933A03209339032091A9
:1042A000390330913A03C90137FD079603E095952C
:1042B00087950A95E1F790932B0380932A038091C9
:1042C0003B0390913C03820F931F97FD01969595B8
:1042D000879590933C0380933B0320917804309121
:1042E0007904821B930B90931E0180931D012091F2
:1042F00030033091310380911D0190911E01280FF0
:10430000391F37FF02C02F5F3F4F359527953093F8
:1043100031032093300333CE20913703309138039B
:104320008091780090917900280F391F30933803DD
:1043300020933703809101018A3019F4220F331F33
:1043400004C0220F331F220F331F309338032093F2
:1043500037032091370330913803C90137FD0796A1
:10436000F3E095958795FA95E1F79093290380936B
:10437000280380913D0390913E03820F931F97FD88
:1043800001969595879590933E0380933D032091E8
:10439000760430917704821B930B90931C018093D9
:1043A0001B0120912E0330912F0380911B019091CE
:1043B0001C01280F391F37FF02C02F5F3F4F359573
:1043C000279530932F0320932E0383E06BC1109227
:1043D000330381E0809311018091170390911803BA
:1043E0000196909318038093170380917800909121
:1043F0007900909316018093150180911501909199
:104400001601AA27BB272091430330914403409112
:10441000450350914603280F391F4A1F5B1F209305
:1044200043033093440340934503509346038091E4
:1044300047038F5F80934703803108F432C1809136
:10444000170190911801A0911901B0911A017C01F6
:104450008D0163E0EE0CFF1C001F111F6A95D1F760
:10446000E81AF90A0A0B1B0BE20EF31E041F151FB4
:1044700080911B03992787FD9095A92FB92FBC0127
:10448000CD0120EB30E240E050E00E947E91DC0163
:10449000CB01E81AF90A0A0B1B0BD801C7010496D5
:1044A000A11DB11DB7FF05C0D801C7010B96A11D05
:1044B000B11D23E0B595A795979587952A95D1F7D6
:1044C0008093170190931801A0931901B0931A01DA
:1044D0008091290790912A077C010027F7FC00951D
:1044E000102F8091170190911801A0911901B0919E
:1044F0001A01E81AF90A0A0B1B0BE0920304F09266
:104500000404009305041093060420911C033091C9
:104510001D0340911E0350911F0357FF04C0215FEC
:104520003F4F4F4F5F4F84E05595479537952795FF
:104530008A95D1F780911C0390911D03A0911E03D1
:10454000B0911F03821B930BA40BB50B80931C032C
:1045500090931D03A0931E03B0931F0380911C032F
:1045600090911D03A0911E03B0911F038E0D9F1DFE
:10457000A01FB11F80931C0390931D03A0931E03E3
:10458000B0931F0380911C0390911D03A0911E0303
:10459000B0911F03B7FF03C00F96A11DB11D14E01A
:1045A000B595A795979587951A95D1F7209103040E
:1045B00030910404281B390B64E0213036071CF0CD
:1045C00020E034E006C07CEF2030370714F420E010
:1045D0003CEF8091190390911A03809119039091F7
:1045E0001A0397FF03C0909581959F4FA901F3E0AF
:1045F000440F551FFA95E1F78D5B9240C4F080910E
:10460000190390911A039C01E4E0220F331FEA95ED
:10461000E1F7281B390B240F351F37FF02C0215F3C
:104620003F4F74E0359527957A95E1F717C0809153
:10463000190390911A039C0165E0220F331F6A95BC
:10464000E1F7281B390B240F351F37FF02C0215E0D
:104650003F4F45E0359527954A95E1F730931A038A
:10466000209319038091430390914403A091450343
:10467000B0914603B7FF03C00196A11DB11DB595CA
:10468000A795979587958093430390934403A093B0
:104690004503B093460388E08093470302C010921D
:1046A000330382E0809332038091320380937C0055
:1046B00080913303882319F08FEC80937A00FF9167
:1046C000EF91BF91AF919F918F917F916F915F918A
:1046D0004F913F912F911F910F91FF90EF900F906D
:1046E0000FBE0F901F90189590E2E4E3F7E08FE47F
:1046F0009193815087FFFCCF089590914A039035A4
:1047000040F4E92FFF27EC5CF84F80839F5F909384
:104710004A030895AF92BF92CF92DF92FF920F9318
:104720001F93CF93DF932091480320FF0AC080910D
:104730004903882311F0815002C0809121018093A8
:10474000490321FF0CC090914903809121019817E2
:1047500019F41092490303C09F5F90934903822F7D
:10476000992780FF04C081FF02C0109249030E9474
:10477000742380914903282F33279DE7C92E93E2A4
:10478000D92EC0913D05D0913E058A3098F481E143
:1047900080934A033F932F938FE994E09F938F93E5
:1047A000DF92CF92FE0109952DB73EB72A5F3F4FAA
:1047B0002DBF11C080E180934A033F932F9384EA79
:1047C00094E09F938F93DF92CF92FE0109958DB76E
:1047D0009EB706968DBF20914903822F9927AA275D
:1047E000BB27FC01419710F00C94E22CE85AFF4FD4
:1047F0000DE7C02E03E2D02EC0913D05D0913E05BD
:104800000C94449210924A0389EA94E09F938F9308
:104810000DE713E2DF92CF92FE01099584E18093C8
:104820004A030F900F900F900F9085E690E09F93B2
:104830008F938AE590E09F938F931F921F928091B0
:1048400001016AE00E949D91892F99279F938F9380
:10485000809101010E949D9199279F938F9389EBED
:1048600094E09F938F93DF92CF92E0913D05F0917A
:104870003E05099588E280934A03EDB7FEB73E9660
:10488000EDBF83E098E09F938F930E946330992758
:104890009F938F9381ED94E09F938F93DF92CF92BC
:1048A000E0913D05F0913E050995809157059927C6
:1048B0002DB73EB7285F3F4F2DBFEC01C071D070C0
:1048C00084FF06C08CE380934A038FED94E0F1C02F
:1048D0009091E404992349F18CE380934A03892F52
:1048E00099279F938F938CEE94E09F938F931F93C0
:1048F0000F93E0913D05F0913E050995DF93CF932D
:104900009091E40481E1989FC0011124825C954F4D
:104910009F938F931F930F93E0913D05F0913E0578
:1049200009958DB79EB70C9647C19091560599236E
:10493000B1F08CE380934A03892F99279F938F933B
:1049400084EF94E09F938F931F930F93E0913D0525
:10495000F0913E050995EDB7FEB7369679C4909172
:104960005003992371F08CE380934A03892F992790
:104970009F938F938BE095E09F938F931F930F935B
:10498000D9C48091360190913701069710F00C94AC
:10499000EB2C8CE380934A0380E295E0A5C78091DD
:1049A00072091DE7C12E13E2D12EC0913D05D091B1
:1049B0003E0580FF6BC010924A03809103049091E2
:1049C0000404A0910504B0910604BC01CD0125E0CA
:1049D00030E040E050E00E94F2913F932F938DE24F
:1049E00095E09F938F93DF92CF92FE01099584E12A
:1049F00080934A038DB79EB706968DBF8091FF03C3
:104A000090910004A0910104B0910204BC01CD0179
:104A100025E030E040E050E00E94F2913F932F9378
:104A20008AE395E09F938F93DF92CF92E0913D05CB
:104A3000F0913E05099588E280934A03EDB7FEB7F1
:104A40003696EDBF80911501909116019F938F933B
:104A500087E495E09F938F93DF92CF92E0913D059D
:104A6000F0913E0509958CE380934A032DB73EB73C
:104A70002A5F3F4F2DBF87B599279F938F9384E57A
:104A800095E09F938F93DF92CF928EC010924A034E
:104A900081E695E09F938F93DF92CF92FE01099577
:104AA00084E180934A030F900F900F900F9080E75E
:104AB00095E09F938F93DF92CF921AC710924A038B
:104AC00089E795E09F938F930DE713E2DF92CF92F2
:104AD000FE01099584E180934A030F900F900F9097
:104AE0000F908091630490916404A0916504B0914B
:104AF0006604B7FF04C081509C4FAF4FBF4FCAE060
:104B0000B595A79597958795CA95D1F7BF93AF931C
:104B10009F938F9386E895E09F938F931F930F93B6
:104B2000E0913D05F0913E05099588E280934A03A6
:104B3000EDB7FEB73896EDBF80915B0490915C04B1
:104B4000A0915D04B0915E04B7FF04C081509C4FFA
:104B5000AF4FBF4FFAE0B595A79597958795FA9512
:104B6000D1F7BF93AF939F938F9385E995E09F9380
:104B70008F931F930F93E0913D05F0913E050995AA
:104B80008CE380934A032DB73EB7285F3F4F2DBF7C
:104B900080912F09909130099F938F9384EA95E03B
:104BA0009F938F931F930F93E0913D05F0913E05E6
:104BB00009958DB79EB706968DBF0DC7E1E0FE2E15
:104BC000C1E0D0E00BEB18E09F2D969584E1989F13
:104BD000C001112480934A03F801828193819F933D
:104BE0008F932196DF93CF932197808191819F931B
:104BF0008F93DF93CF9383EB95E09F938F938DE714
:104C000093E29F938F93E0913D05F0913E050995C6
:104C10002DB73EB7245F3F4F2DBF32E0F30E2296F3
:104C20000C5F1F4F88E08F1578F6D5C610924A03A7
:104C300080918707E82FFF27EE0FFF1FE754F74FFC
:104C4000808191819F938F9380918607E82FFF2722
:104C5000EE0FFF1FE754F74F808191819F938F9351
:104C600085EC95E09F938F93DF92CF92FE0109959B
:104C700084E180934A03EDB7FEB73896EDBF80918B
:104C80008907E82FFF27EE0FFF1FE754F74F8081BA
:104C900091819F938F9380918807E82FFF27EE0FD4
:104CA000FF1FE754F74F8081918181589F4F9F9359
:104CB0008F9385ED95E09F938F93DF92CF92E09154
:104CC0003D05F0913E05099588E280934A032DB792
:104CD0003EB7285F3F4F2DBF80918B07E82FFF27FE
:104CE000EE0FFF1FE754F74F8081918181589F4F4E
:104CF0009F938F9380918A07E82FFF27EE0FFF1F66
:104D0000E754F74F8081918181589F4F9F938F93F4
:104D100085EE95E09F938F93DF92CF92E0913D05D2
:104D2000F0913E0509958CE380934A038DB79EB7B9
:104D300008968DBF80918D07E82FFF27EE0FFF1F8C
:104D4000E754F74F8081918181589F4F9F938F93B4
:104D500080918C07E82FFF27EE0FFF1FE754F74FD6
:104D60008081918181589F4F9F938F9385EF95E02C
:104D700063C210924A0385E096E09F938F930DE7FC
:104D800013E2DF92CF92FE010995809101010F900D
:104D90000F900F900F908A3009F09DC084E18093AE
:104DA0004A0380917804909179049C0197FF02C096
:104DB000295F3F4F287F821B930B9F938F93809196
:104DC00078049091790497FD079673E095958795FF
:104DD0007A95E1F79F938F9320917804309179042D
:104DE00037FF02C0295F3F4F63E0359527956A95ED
:104DF000E1F780912A0390912B03821B930B9F93E1
:104E00008F9383E196E09F938F931F930F93E0918D
:104E10003D05F0913E05099588E280934A032DB740
:104E20003EB7265F3F4F2DBF809176049091770467
:104E30009C0197FF02C0295F3F4F287F821B930B85
:104E40009F938F93809176049091770497FD0796B6
:104E500053E0959587955A95E1F79F938F9320910D
:104E600076043091770437FF02C0295F3F4F43E05B
:104E7000359527954A95E1F780912803909129036C
:104E8000821B930B9F938F9384E296E09F938F9363
:104E90001F930F93E0913D05F0913E0509958CE33A
:104EA00080934A038DB79EB70A968DBF8091740494
:104EB000909175049F938F938091740490917504E1
:104EC0002091260330912703821B930B9F938F938E
:104ED00085E396E0ADC08B3019F0843108F4ADC0A5
:104EE00084E180934A0380917804909179049C0135
:104EF00097FF02C0215F3F4F207F821B930B97FDDE
:104F00000196959587959F938F93809178049091C2
:104F1000790497FD0F9624E0959587952A95E1F7FA
:104F20009F938F93209178043091790437FF02C0CA
:104F3000295F3F4FC3E035952795CA95E1F78091EA
:104F40002A0390912B03821B930B9F938F9383E4EF
:104F500096E09F938F931F930F93E0913D05F091FF
:104F60003E05099588E280934A032DB73EB7265F38
:104F70003F4F2DBF80917604909177049C0197FF5D
:104F800002C0215F3F4F207F821B930B97FD01964C
:104F9000959587959F938F93809176049091770450
:104FA00097FD0F96A4E095958795AA95E1F79F93B5
:104FB0008F93209176043091770437FF02C0295FE8
:104FC0003F4FF3E035952795FA95E1F78091280357
:104FD00090912903821B930B9F938F9385E596E015
:104FE0009F938F931F930F93E0913D05F0913E05A2
:104FF00009958CE380934A038DB79EB70A968DBFBF
:10500000809174049091750497FD0196959587950C
:105010009F938F938091740490917504209126033F
:1050200030912703821B930B9F938F9387E696E023
:105030009F938F931F930F9303C18D3009F0CBC4BF
:1050400084E180934A038091140199279F938F9361
:10505000809178049091790497FD0F9674E095956E
:1050600087957A95E1F79F938F93209178043091FB
:10507000790437FF02C0295F3F4F63E035952795DC
:105080006A95E1F780912A0390912B03821B930B81
:105090009F938F9386E796E09F938F931F930F9331
:1050A000E0913D05F0913E05099588E280934A0321
:1050B0002DB73EB7265F3F4F2DBF80911301992733
:1050C0009F938F93809176049091770497FD0F962C
:1050D00054E0959587955A95E1F79F938F9320918A
:1050E00076043091770437FF02C0295F3F4F43E0D9
:1050F000359527954A95E1F78091280390912903EA
:10510000821B930B9F938F938AE896E09F938F93D4
:105110001F930F93E0913D05F0913E0509958CE3B7
:1051200080934A038DB79EB70A968DBF8091120176
:1051300099279F938F93809174049091750497FDA4
:105140000196959587959F938F9380917404909184
:1051500075042091260330912703821B930B9F93A4
:105160008F938EE996E09F938F931F930F93E09117
:105170003D05F0913E050995EDB7FEB73A9668C03A
:1051800010924A0382EB96E09F938F93DF92CF9227
:10519000FE01099584E180934A030F900F900F90D0
:1051A0000F9080916E0490916F049F938F938091E4
:1051B0002203909123039F938F938FEB96E09F930D
:1051C0008F93DF92CF92E0913D05F0913E050995D6
:1051D00088E280934A032DB73EB7285F3F4F2DBF2B
:1051E00080916C0490916D049F938F938091240320
:1051F000909125039F938F938EEC96E09F938F93CE
:10520000DF92CF92E0913D05F0913E0509958CE348
:1052100080934A038DB79EB708968DBF809168042E
:10522000909169049F938F93809120039091210323
:105230009F938F938DED96E09F938F93DF92CF9204
:10524000E0913D05F0913E050995EDB7FEB7389622
:10525000EDBFC1C310924A0380911F0190912001BC
:105260006AE070E00E94BD919F938F9380911F012F
:10527000909120016AE070E00E94BD917F936F934E
:105280008CEE96E09F938F93DF92CF92FE0109956B
:1052900084E180934A032DB73EB7285F3F4F2DBF6F
:1052A0008091120A9091130A6AE070E00E94A9911D
:1052B0009F938F938091120A9091130A6AE070E095
:1052C0000E94A9917F936F9380E097E09F938F93C3
:1052D000DF92CF92E0913D05F0913E05099588E27D
:1052E00080934A038DB79EB708968DBF8091140AAC
:1052F0009091150A9F938F9384E197E09F938F93EA
:10530000DF92CF92E0913D05F0913E0509958CE347
:1053100080934A03EDB7FEB73696EDBF8091160A2B
:105320009091170A9F938F9384E297E09F938F93B6
:10533000DF92CF92E0913D05F0913E0509952DB7A2
:105340003EB72A5F3F4F4FC110924A0386E397E072
:105350009F938F93DF92CF92FE01099584E1809312
:105360004A030F900F900F900F908091B908909181
:10537000BA089F938F938FE397E09F938F93DF9269
:10538000CF92E0913D05F0913E05099588E280932A
:105390004A038DB79EB706968DBF80910904992761
:1053A0009F938F938FE497E09F938F93DF92CF9299
:1053B000E0913D05F0913E0509958CE380934A0309
:1053C000EDB7FEB73696EDBF8091B80899270197E3
:1053D0009F938F938FE597E0A9CF10924A038FE6B2
:1053E00097E09F938F93DF92CF92FE01099584E11E
:1053F00080934A030F900F900F900F9080918A0135
:1054000090918B019F938F9387E797E09F938F9362
:10541000DF92CF92E0913D05F0913E05099588E23B
:1054200080934A038DB79EB706968DBF80912F0952
:10543000909130099F938F9385E897E09F938F9386
:10544000DF92CF92E0913D05F0913E0509958CE306
:1054500080934A03EDB7FEB73696EDBF80912104E5
:10546000909122049F938F9383E997E05FCFCAE0E6
:10547000CC2EC4E0DC2E20E030E0E901B3E0FB2ECE
:10548000C0934A03F60181916F0199279F938F93EF
:1054900089010F5F1F4F1F930F9381EA97E09F933E
:1054A0008F938DE793E29F938F93E0913D05F09169
:1054B0003E0509952DB73EB7285F3F4F2DBFFA94A3
:1054C00064969801F7FEDCCF86C2AEE0CA2EA4E057
:1054D000DA2EC0E0D0E08E01F3E0FF2E00934A0305
:1054E000F60181916F0199279F938F932596DF9302
:1054F000CF938EEA97E09F938F938DE793E29F93EC
:105500008F93E0913D05F0913E0509952DB73EB78B
:10551000285F3F4F2DBFFA940C5E1F4F2497F7FE74
:10552000DDCF59C210924A038BEB97E09F938F9384
:105530000DE713E2DF92CF92FE01099584E180939B
:105540004A030F900F900F900F9080916901992757
:105550009F938F9383EC97E09F938F93DF92CF92EB
:10556000E0913D05F0913E05099588E280934A035C
:105570008DB79EB706968DBF809104039091050369
:1055800097FD039695958795959587959F938F930E
:1055900081ED97E09F938F931F930F93E0913D05CB
:1055A000F0913E0509958CE380934A03EDB7FEB771
:1055B0003696EDBF8091B50799279F938F93809181
:1055C000B40799279F938F938FED97E09F938F93C5
:1055D0001F930F93E0913D05F0913E0509952DB77E
:1055E0003EB7285F3F4F2DBFF6C110924A038DEEA4
:1055F00097E09F938F937DE7A72E73E2B72EDF92FC
:10560000CF92FE0109950F900F900F900F90C8E573
:10561000D8E000E010E062E0F62E802F8C5E8093F0
:105620004A038B8D99278F7790709F938F938B89E7
:1056300099278F7790709F938F938B8599278F777A
:1056400090709F938F938B8199278F7790709F9302
:105650008F938DEF97E09F938F93BF92AF92E091DE
:105660003D05F0913E0509958DB79EB70C968DBF0F
:10567000FA940C5E1F4FA096F7FECFCFACC11092EC
:105680004A038EE098E09F938F935DE7A52E53E247
:10569000B52EDF92CF92FE0109950F900F900F90DB
:1056A0000F90C8E5D8E000E010E042E0F42E802F33
:1056B0008C5E80934A038F8D992787FD90959F93E9
:1056C0008F938F89992787FD90959F938F938F85CF
:1056D000992787FD90959F938F938F81992787FDB9
:1056E00090959F938F938DE198E09F938F93BF92B6
:1056F000AF92E0913D05F0913E050995EDB7FEB7FB
:105700003C96EDBFFA940C5E1F4FA096F7FECFCFEC
:1057100062C110924A038EE298E09F938F930DE747
:1057200013E2DF92CF92FE01099584E180934A0350
:105730000F900F900F900F9080917308881F88270B
:10574000881F97E0899FC00111248D969F938F93A6
:1057500080916B08881F8827881F96E0899FC00169
:1057600011248D969F938F9380916308881F8827BB
:10577000881F95E0899FC00111248D969F938F9378
:1057800080915B08881F8827881F9927880F991F99
:10579000880F991F8D969F938F938DE398E09F9329
:1057A0008F93DF92CF92E0913D05F0913E050995F0
:1057B00088E280934A032DB73EB7245F3F4F2DBF49
:1057C00080919308881F8827881F9BE0899FC001CC
:1057D00011248D969F938F9380918B08881F882723
:1057E000881F9AE0899FC00111248D969F938F9303
:1057F00080918308881F8827881F99E0899FC001AE
:1058000011248D969F938F9380917B08881F882702
:10581000881F992723E0880F991F2A95E1F78D9615
:105820009F938F9381E598E09F938F93DF92CF9220
:10583000E0913D05F0913E0509958CE380934A0384
:105840008DB79EB70C968DBF80919B08881F8827C7
:10585000881F9CE0899FC00111248D969F938F9390
:1058600085E698E09F938F93DF92CF92E0913D057C
:10587000F0913E0509958091A308EDB7FEB73696E5
:10588000EDBF87FF12C080E480934A0386E798E06B
:105890009F938F93DF92CF92E0913D05F0913E056B
:1058A00009950F900F900F900F908091AB0887FF94
:1058B00012C084E480934A0389E798E09F938F9312
:1058C0001F930F93E0913D05F0913E0509950F90D0
:1058D0000F900F900F908091B30887FF7CC088E4F1
:1058E00080934A038CE798E09F938F931F930F93C5
:1058F000E0913D05F0913E0509950F900F900F90B6
:105900000F9069C010924A038FE798E09F938F939E
:10591000DF92CF92FE01099584E180934A030F90B4
:105920000F900F900F908091DA029091DB029F937D
:105930008F938DE898E09F938F93DF92CF92E091C1
:105940003D05F0913E05099588E280934A032DB705
:105950003EB72A5F3F4F2DBF8091DC029091DD0260
:105960009F938F938AE998E09F938F93DF92CF92D2
:10597000E0913D05F0913E05099589E480934A0345
:105980008DB79EB706968DBF87EA98E09F938F9359
:10599000DF92CF92E0913D05F0913E05099580910F
:1059A00048030F900F900F900F9083FF14C0109238
:1059B000DD021092DC0260E070E08EE090E00E9478
:1059C000002F09C080912101281719F4215020933C
:1059D00021011092490310924803DF91CF911F914A
:1059E0000F91FF90DF90CF90BF90AF900895F999FD
:1059F000FECF92BD81BDF89A80B599270895F99997
:105A0000FECF1FBA92BD81BD60BD0FB6F894FA9A61
:105A1000F99A0FBE08954AEA20E030E026173707CA
:105A200040F4FC018191480F2F5F3F4F2617370745
:105A3000C8F3842F99270895EAEA40E050E046171A
:105A4000570778F49C01F999FECF32BD21BDF89A31
:105A500080B5E80F4F5F5F4F2F5F3F4F46175707E7
:105A600090F38E2F9927089581E08093880782E034
:105A70008093870783E08093860784E0809389077B
:105A800085E080938A0786E080938B0787E0809388
:105A90008C0788E080938D0789E080938E078AE0E9
:105AA00080938F078BE0809390078CE08093910721
:105AB00008958DE5809385078CE0E5EFF7E011927E
:105AC0008A95E9F780910101843150F08AE0809352
:105AD000A5071092C9078BE18093A1078EE40AC045
:105AE00083E08093A50780E28093C9078EE18093CD
:105AF000A10785E58093C6078093C70780E280935E
:105B0000C8071092F1078AE68093920782E2809399
:105B1000F30780E48093F40766E06093AC0710928B
:105B2000E9071092E60748E040939F0756EE50932E
:105B3000A0078093A2079EE1909393078FEF809335
:105B400095072FE02093960790939407109298075B
:105B50004093990784E180939A0710929B072093C2
:105B600097071092AE071092AF071092B0071092ED
:105B7000B1071092CB071092CC071092CD0710926C
:105B8000CE0790E89093B20732E33093B30782E0F8
:105B90008093F2072093B4075093B50784E0809375
:105BA000BA072DE72093BD072093BE072093BF07B8
:105BB0009093B60755E55093B70786E48093B807EE
:105BC0008CED8093B9078CE38093BB071092BC07E0
:105BD0008FE58093CF0783EF8093D1078AEA809384
:105BE000D3078093D40788E28093D0078093D207AD
:105BF0001092D5073093C0079AE59093C107309370
:105C0000C2078EEF8093D60784E68093D7079093E0
:105C1000D8079093D9079093DA078BE48093DB073A
:105C20005093DC078093DD071092DE076093DF0757
:105C30004093E0079093E1078AE28093E20785EFC3
:105C40008093E3078CE88093E40785E08093E50781
:105C50001092E7071092E80781E28093A90781E498
:105C60008093AA079093AB071092EA071092EB0774
:105C70001092EC0786E98093ED072093C30784E335
:105C80008093C4071092EE071092EF071092F0076E
:105C900008950E94592D8AE080939C0780E18093AB
:105CA0009D0726E020939E079AE59093A30788E737
:105CB0008093A4079093A6078093A7072093A80733
:105CC00080E28093AD078CE38093C5078BE48093DB
:105CD000CA0786E491E6A3E7B4E78093F5079093BB
:105CE000F607A093F707B093F8076CE770E085E834
:105CF00097E00E940B2D809301080895CF93DF93C6
:105D00000E94592D88E080939C0730E130939D07D5
:105D100026E020939E0794E69093A30788E780935C
:105D2000A4079093A6078093A7072093A807309312
:105D3000AD0786E48093C5078093CA07A5EFB7E057
:105D4000E2E2F1E0ED01019009922A95E1F76CE7BA
:105D500070E0CD01805790400E940B2D8093010888
:105D6000DF91CF9108950E94592D26E020939C0742
:105D70008AE080939D0784E080939E0794E6909349
:105D8000A30788E78093A4079093A6078093A707AB
:105D90002093A80780E18093AD0786E48093C50730
:105DA0008093CA0785E491E6A3E7B9E78093F507F6
:105DB0009093F607A093F707B093F8076CE770E0AD
:105DC00085E897E00E940B2D809301080895F999CA
:105DD000FECF92BD81BDF89A80B599270895F999B3
:105DE000FECF1FBA92BD81BD60BD0FB6F894FA9A7E
:105DF000F99A0FBE089567EF7CE20E940C90089517
:105E00004FEF5CE20E9446900895EF92FF920F934D
:105E10001F93CF93C82F8150853008F0C3E08DE7E2
:105E2000C89F8001112487EEE82E8FEFF82EE00E38
:105E3000F11E6CE770E0C7010E941C2D682F9801CD
:105E40002D593F4F8FB39927AC014270507081FD9F
:105E5000F9CF32BD21BDF89A80B5861711F0CA017D
:105E600023C08FB399279C012270307081FDF9CF38
:105E7000F2BCE1BCF89A80B58D3511F0C90114C0AF
:105E80008DE7C89FC0011124499727EF3CE24DE7F9
:105E900050E0BC0185E897E00E94E78F0E94D86D32
:105EA0000E94C48B81E090E0CF911F910F91FF90F1
:105EB000EF900895282F863010F025E003C0882346
:105EC00009F421E0F999FECF1FBA82E090E092BD7B
:105ED00081BD20BD0FB6F894FA9AF99A0FBE0895C5
:105EE000CF93C82F809185078D3509F051C0C630FA
:105EF00010F0C5E003C0CC2309F44AC00E94D08E44
:105F00008091F40782FF07C08091AA07843618F0B9
:105F100080E58093AA076CE770E085E897E00E942F
:105F20000B2D809301088DE7C89FC00111242FEF2E
:105F30003CE24DE750E065E877E049970E94249005
:105F40002FEF3CE24CE050E066E877E080E590E03F
:105F50000E9424906CE070E086E897E00E940B2D90
:105F6000282FF999FECF1FBA8CE590E092BD81BD34
:105F700020BD0FB6F894FA9AF99A0FBE8C2F0E94A2
:105F80005A2F0E94D86D0E94C48B81E090E002C01D
:105F900080E090E0CF9108956DE470E088EE93E0AA
:105FA0000E941C2D482F8FB399279C0122703070BE
:105FB00081FDF9CF85E394E092BD81BDF89A80B56B
:105FC000841779F48FB399279C012270307081FD7A
:105FD000F9CF88EE93E092BD81BDF89A80B581300B
:105FE00011F0C901089527EF3CE24EE450E068EE5D
:105FF00073E082E098E00E94E78F81E090E00895EE
:10600000809102088130A9F46DE470E082E098E0AC
:106010000E940B2D80934F082FEF3CE24EE450E09E
:1060200062E078E088EE93E00E94249081E090E0C6
:10603000089580E090E00895CF93DF9381E080930E
:106040000208E2E0F8E08FE0158616861786108ACF
:106050008150349687FFF8CF80E480930F088093B7
:10606000100810921108809312088093130890EC86
:1060700090931408109215088093160880931708BF
:10608000109218089093190890931A0880931B088F
:1060900010921C0880931D0890931E08A3E0B8E09E
:1060A0008CE0E9E2F1E0ED01019009928A95E1F7D7
:1060B0006DE470E0CD0101970E940B2D80934F0895
:1060C000DF91CF910895F999FECF82E090E092BDE3
:1060D00081BDF89A80B5282F863078F023E0322FE2
:1060E000F999FECF1FBA82E090E092BD81BD30BD2C
:1060F0000FB6F894FA9AF99A0FBE822F992708954D
:106100001F93CF93C82F162F863010F0C5E003C021
:10611000882309F4C1E08C2F99278230910541F042
:106120008330910544F4019731F40E94492E05C053
:106130000E947E2E02C00E94B32E1123E1F06CE07B
:1061400070E080E590E00E941C2D282FF999FECF89
:106150008CE590E092BD81BDF89A80B5821759F424
:1061600027EF3CE24CE050E060E570E086E897E025
:106170000E94E78F02C00E94342D8C2F0E94702F46
:10618000CF911F910895DF92EF92FF920F931F938B
:10619000CF93FF24DF2CEF2C81E090E00E94E72ECC
:1061A0008D3511F031E0E32E6CE070E080E590E099
:1061B0000E941C2DC82FF999FECF8CE590E092BD6E
:1061C00081BDF89A80B58C1711F421E0D22EC1E080
:1061D00001E010E0EE2029F48C2F0E94052F882387
:1061E000C9F591E0F92E1F930F938FEA98E09F93E2
:1061F0008F9380E695E19F938F93E0913D05F09119
:106200003E0509952DB73EB72A5F3F4F2DBF02309F
:10621000110549F0033011054CF40130110531F43A
:106220000E94492E05C00E947E2E02C00E94B32EFD
:10623000DD2059F027EF3CE24CE050E060E570E0F3
:1062400086E897E00E94E78F02C00E94342D8C2FD1
:106250000E94702FCF5F0F5F1F4FC63008F4BACF78
:10626000FF2019F083E00E945A2F0E946330C82F4C
:106270000E94052F8C2F99279F938F9385ED98E08F
:106280009F938F9300E615E11F930F93E0913D05D7
:10629000F0913E05099581E090E00E94E72E2DB730
:1062A0003EB72A5F3F4F2DBF8F3F21F00E94CC2F7A
:1062B000882399F48EEE98E09F938F931F930F930A
:1062C000E0913D05F0913E0509950E941C300E9429
:1062D00000300F900F900F900F90EE2029F06DE599
:1062E00081E090E00E94EF2E1092840790E0EFE0B2
:1062F000F8E0CFE08081349618160CF49F5FC1500F
:10630000C7FFF8CF90938407892F99279F938F9386
:1063100083E098E09F938F938FE099E09F938F9312
:106320001F930F93E0913D05F0913E0509950E9462
:106330004A098DB79EB708968DBFCF911F910F91D7
:10634000FF90EF90DF900895982F2FB7F894399829
:10635000389A88B1836088B98091B9008C7F809326
:10636000B9008AE28093B80010925503109253034B
:1063700010925203992379F0E8E5F8E08BE010825F
:106380001182128213821482158216821782815022
:10639000389687FFF4CF78942FBF08951092550355
:1063A00084E98093BC0080E88093BC001092BD001B
:1063B0001092BA001092BB001092B9001092B8006F
:1063C0001092510380E00E94A4311092BB0085E836
:1063D0008093BC0080914F03826080934F030895A7
:1063E0001F920F920FB60F9211242F933F934F934A
:1063F0005F938F939F93EF93FF9380915503282F83
:106400003327442755278F5F80935503F9012731A0
:10641000310508F0C2C2E759FF4F0C94449281E065
:106420008093510309C0809153038C3090F4809184
:1064300053038F5F8093530380915303E82FFF270B
:10644000EE0FFF1FEE0FFF1FEE5FF74F858518164B
:1064500054F7809153038C3070F010924E031092D9
:106460004D031092530385E08093550380915203AE
:10647000880F8D5A04C080915303880F8E5A8093E1
:10648000BB0085E87FC280915303E82FFF2783E09C
:10649000EE0FFF1F8A95E1F7E85AF74F818180934D
:1064A000BB0085E88093BC0080915303E82FFF2751
:1064B000EE0FFF1FEE0FFF1FEE0FFF1FE85AF74F03
:1064C000808180FF91C080915303E82FFF27EE0F5A
:1064D000FF1FEE0FFF1FEE0FFF1FE85AF74F8281DD
:1064E000882329F080918407873008F46CC280915A
:1064F0004D0390914E03892B09F065C280914B03A7
:1065000090914C03892B09F05EC26EC080915303B9
:1065100021E030E002C0220F331F8A95E2F780911C
:106520004B0390914C0328233923232B79F080913E
:106530005303E82FFF27EE0FFF1FEE0FFF1FEE0F95
:10654000FF1FE85AF74F80E184830DC08091530309
:10655000E82FFF27EE0FFF1FEE0FFF1FEE0FFF1FAD
:10656000E85AF74F148280915303E82FFF2753E036
:10657000EE0FFF1F5A95E1F7E85AF74F8481282F55
:10658000332743E0220F331F4A95E1F780915303ED
:10659000E82FFF2793E0EE0FFF1F9A95E1F7E85AE7
:1065A000F74F82818770822B8093BB0085E88093B0
:1065B000BC002091530381E090E002C0880F991F36
:1065C0002A95E2F720914D0330914E0382239323C5
:1065D000892B51F080E598E09093590380935803FC
:1065E00088E080935A03EFC184E089C1E0915803A9
:1065F000F091590381918093BB0085E88093BC00A2
:10660000F0935903E093580380915A03815080938B
:106610005A03882309F4D7C183E071C18091B9007E
:10662000803351F580915603882329F480915303D8
:106630008F5F8093560380915303E82FFF2783E0F9
:10664000EE0FFF1F8A95E1F7E85AF74F83819927EC
:106650008F7790708F3791057CF480915303E82FEA
:10666000FF27EE0FFF1FEE0FFF1FEE0FFF1FE85A71
:10667000F74F83818F5F83831092550384E9809362
:10668000BC008AE090E090933701809336018091BE
:1066900053038F5F80935303109255036DC1809114
:1066A000B9008034C9F180915203E82FFF27EE0F23
:1066B000FF1FEE0FFF1FEE0FFF1FE85AF74F8381FA
:1066C0008F778383809152038F5F809352038091F1
:1066D00052038C30A0F01092520310924C0310928F
:1066E0004B03809157038F5F809357038C3038F0B2
:1066F0001092570380914F038D7F80934F038091B9
:106700004F03816080934F031092550384E9809377
:10671000BC001092510373C080915203E82FFF27F1
:10672000EE0FFF1FEE0FFF1FEE0FFF1FE85AF74F90
:1067300083818068838380915203E82FFF27EE0FC7
:10674000FF1FEE0FFF1FEE0FFF1FE85AF74F80816C
:1067500080FF2FC080915203E82FFF2753E0EE0FF8
:10676000FF1F5A95E1F7E85AF74F84819927009760
:1067700051F04097D9F580E598E0909359038093C4
:10678000580388E031C080915203992743E0880F75
:10679000991F4A95E1F7835A974F90935903809335
:1067A000580390915203809157039817E1F483E0C6
:1067B0001BC080915203992733E0880F991F3A95A7
:1067C000E1F7835A974F9093590380935803809130
:1067D0004F0381FD06C09091520380915703981793
:1067E00011F482E001C081E080935A0380915A0342
:1067F000813011F485E801C085EC8093BC00809164
:1068000056038093500310925603DDC0E091580365
:10681000F09159038091BB0080838091580390913F
:1068200059030196909359038093580380915A031A
:10683000815080935A03823010F085EC5DC0813026
:1068400011F485E859C080914F0381FF2DC08091DC
:10685000D10380FD1DC080915203E82FFF2723E064
:10686000EE0FFF1F2A95E1F7E85AF74F86818A3F1E
:1068700079F480915203E82FFF2793E0EE0FFF1F7A
:106880009A95E1F7E85AF74F8081816080830CC0C8
:1068900080915203E82FFF2783E0EE0FFF1F8A95B8
:1068A000E1F7E85AF74F1082809152038F5F80938F
:1068B0005203809152038C30A0F010925203109238
:1068C0004C0310924B03809157038F5F80935703C3
:1068D0008C3038F01092570380914F038D7F809356
:1068E0004F031092550384E98093BC0080914F03BD
:1068F000816080934F0365C08093BC0086E08093E5
:10690000550361C088E9BBCD80915403880F805F37
:10691000B6CD8091540399278130910561F0823082
:1069200091051CF4892B21F04EC0029739F04BC021
:1069300080911401A4CD80911301A1CD8091120109
:106940009ECD80E89CCD1092550384E98093BC00D5
:10695000109251038AE090E09093370180933601C2
:1069600080915403823088F4809154038F5F809328
:10697000540382E18093550380914F038E7F80936F
:106980004F0385EA8093BC001EC01092540380918F
:106990004F03816080934F0316C01092550384E922
:1069A0008093BC0080914F03816080934F038AE005
:1069B00090E0909337018093360110925303109228
:1069C000520310925103FF91EF919F918F915F912C
:1069D0004F913F912F910F900FBE0F901F901895E0
:1069E0001F93CF93DF93182F80910804882321F4FD
:1069F0008091E902882319F081E090E097C01D3072
:106A000008F092C01123B1F0E12FFF2723E0EE0F31
:106A1000FF1F2A95E1F7E85AF74F359780813596A1
:106A200088230CF081C03897808180FD03C083E00B
:106A300090E07CC080915008823019F084E090E0B2
:106A400075C067E070E080E598E00E940B2D9091A2
:106A50005708891719F085E090E068C080ED97E04D
:106A60000E946F19EC0180914F0380FD05C0CE019B
:106A70000E9478198823B9F3112319F48FEF90E05D
:106A80000BC0212F33272150304081E090E002C01D
:106A9000880F991F2A95E2F790934E0380934D0338
:106AA000A1E0B0E0E8E5F8E040E050E06BE0CD01C7
:106AB000042E02C0880F991F0A94E2F720914D031B
:106AC00030914E0382239323892B11F0118212827D
:106AD00061504F5F5F4F389667FFE9CF10925303C5
:106AE0001092550380914F038E7F80934F0385EA68
:106AF0008093BC0080914F0380FD05C0CE010E94B1
:106B000078198823B9F380914D0390914E03892B16
:106B100029F0CE010E947819882311F380914D034A
:106B200090914E03009711F082E090E0DF91CF91B9
:106B30001F9108950F931F93CF93DF93982F809108
:106B40000804882321F48091E902882319F081E068
:106B500090E092C09D30A0F4992319F486E090E073
:106B60008BC0C92FDD27FE0133E0EE0FFF1F3A95E2
:106B7000E1F7E85AF74F35978081359687FD03C0D6
:106B800082E090E079C03897808180FD03C083E087
:106B900090E072C080ED97E00E946F198C018091A7
:106BA0004F0380FD05C0C8010E9478198823B9F3FE
:106BB000219721E030E0C90102C0880F991FCA95D2
:106BC000E2F790934C0380934B03D901E8E5F8E09A
:106BD00040E050E06BE0CD01042E02C0880F991F09
:106BE0000A94E2F720914B0330914C0382239323C4
:106BF000892B11F01182128261504F5F5F4F3896DE
:106C000067FFE9CF10925203109250081092570874
:106C10001092550380914F038E7F80934F0385EA36
:106C20008093BC0080914F0380FD05C0C8010E9485
:106C300078198823B9F380914B0390914C03892BE9
:106C400029F0C8010E947819882311F38091500817
:106C5000823019F084E090E00FC067E070E080E5DA
:106C600098E00E940B2D90915708891719F085E044
:106C700090E002C080E090E0DF91CF911F910F91F2
:106C80000895CF93DF9380E021E83FEFCDEED8E089
:106C9000E9EBF8E0DF01853020F411961C921E929A
:106CA00002C0318320831982188222968F5F129648
:106CB00032968A3180F31092750410927404109207
:106CC0007704109276041092790410927804DF9180
:106CD000CF9108951F920F920FB60F9211240F9328
:106CE0001F932F933F934F935F936F937F938F9354
:106CF0009F93AF93BF93CF93DF93EF93FF938091D5
:106D0000F30782FDE1C04091860050918700809199
:106D10005C0390915D03481B590B80918600909114
:106D2000870090935D0380935C03CA018D54944067
:106D3000A0915E03B0915F03835F9A4178F48091E4
:106D40005E038093B808149714F010923A0181E022
:106D500090E090935F0380935E032BC2AD30B1054A
:106D60000CF027C2CA018B5F9040845B914008F011
:106D700086C08091380190913901481B590BE091F0
:106D8000EE07EE2351F0FF27EE0FFF1FE754F74FFA
:106D90008081918184369105ECF4FD01EA0FFB1F9F
:106DA000E754F74F80819181FA01E81BF90BCF017D
:106DB000F7FF03C0909581959F4F06975CF48091F3
:106DC0000904883C20F480910904865F01C088ECA6
:106DD00080930904FD01EA0FFB1FE754F74F808100
:106DE00091819C01220F331F280F391F240F351F5B
:106DF00037FF02C02D5F3F4FE901D595C795D59567
:106E0000C795CA0101968C179D0714F4219706C0F7
:106E100041505040C417D5070CF4219680910904C5
:106E2000833CE0F08D010A0F1B1FF801E754F74F78
:106E3000808191819E01281B390BC90163E070E0BC
:106E40000E94BD91CB01880F991F860F971F035198
:106E5000174FD80111969C938E9307C0AA0FBB1FA2
:106E6000A351B74F11961C921E92E0915E03F091D0
:106E70005F03EE0FFF1FE754F74FD183C0832091CC
:106E80005E0330915F032F5F3F4F30935F0320938A
:106E90005E0380910101843108F08BC125303105FA
:106EA00011F45D9A01C05D9880915E0390915F033B
:106EB0008630910511F45C9A01C05C98079711F433
:106EC0005B9A77C15B9875C14091860050918700AD
:106ED0008091600390916103481B590B809186005B
:106EE000909187009093610380936003CA018D5451
:106EF00094406091CA03835F9A4108F07AC060931E
:106F00005B0380915B03843008F453C09091B80810
:106F100080915B03981709F04CC05091CB035B3014
:106F200008F43FC010923A011092CA0340E05F316A
:106F3000C0F0E42FFF27EE0FFF1F9F012A563C4FA2
:106F4000DF01A754B74F8D919C91D9018D939C93EC
:106F5000DF01A351B74F8D919C91E055FC4F918378
:106F60008083E42FFF27EE0FFF1F9F012754374F29
:106F7000DF01AE59BC4F8D919C91D90111969C9324
:106F80008E93DF01A458BC4F8D919C91E351F74F34
:106F900091838083842F8F5F482F8D3040F28093C0
:106FA000CA038091CB038F3FB9F08F5F8093CB03EF
:106FB00013C08091CB03853620F08AE08093CB0309
:106FC00002C01092CB03809101018A3011F084310C
:106FD00010F0289A01C0289881E08093CA0380911C
:106FE0000804882309F0E5C080915B038093B8080A
:106FF000E0C06D3008F0B5C0CA018B5F9040845B83
:10700000914008F090C08091380190913901481B5F
:10701000590BE62FFF27EE0FFF1FEE59FC4F808123
:107020009181FA01E81BF90BCF0105960B9720F52A
:10703000E091EE07EE2351F0FF27EE0FFF1FE7541C
:10704000F74F8081918184369105B4F48091CB0310
:107050008A3120F080910904865F05C08B3028F0CA
:10706000809109048E5F8093090480910904893C12
:1070700018F088EC80930904E62FFF27EE0FFF1F1E
:10708000EE59FC4F808191819C01220F331F280F04
:10709000391F240F351F37FF02C02D5F3F4FE90115
:1070A000D595C795D595C795CA0101968C179D07AB
:1070B00014F4219706C041505040C417D5070CF472
:1070C0002196809109048E3BD8F0E62FFF27EE0F22
:1070D000FF1FDF01AE59BC4F8D919C919E01281B73
:1070E000390BC90163E070E00E94BD91CB01880FAC
:1070F000991F860F971FE458FC4F9183808308C027
:10710000E62FFF27EE0FFF1FE458FC4F118210827D
:107110008091CA03E82FFF27EE0FFF1FEE59FC4FA7
:10712000D183C08309C0809101018A3011F084317C
:1071300010F0289A01C0289880910101843188F4C8
:107140008091CA03853011F45D9A05C05D98863040
:1071500011F45C9A05C05C98873011F45B9A01C009
:107160005B988091CA03843120F48F5F8093CA03B7
:1071700020C08431F1F4809101018A3011F0843112
:1071800010F0289A01C028988EE18093CA032CE061
:10719000CDEED8E0A6E9B3E0E9EBF8E08D919D9162
:1071A000918380833296198218822296215027FF7C
:1071B000F5CFFF91EF91DF91CF91BF91AF919F916B
:1071C0008F917F916F915F914F913F912F911F917F
:1071D0000F910F900FBE0F901F901895EF92FF9296
:1071E0000F931F938091A1079927880F991F880FEC
:1071F000991F7C010027F7FC0095102F80916304F4
:1072000090916404A0916504B0916604BC01CD0125
:10721000A80197010E94F2913093E3062093E206C1
:1072200080915B0490915C04A0915D04B0915E0438
:10723000BC01CD01A80197010E94F2913093E506AF
:107240002093E406809176099091770997FD039643
:1072500095958795959587959093E7068093E60693
:10726000809186099091870997FD0396959587955A
:10727000959587959093E9068093E806809174042C
:10728000909175042091260330912703821B930B64
:107290009093EB068093EA06809103049091040496
:1072A000A0910504B0910604BC01CD0125E030E0B9
:1072B00040E050E00E94F2913093ED062093EC06FE
:1072C00080912003909121039093EF068093EE0626
:1072D00080918A0190918B019093F3068093F2063E
:1072E00080911F01909120019093F5068093F40600
:1072F0008091090499279093F7068093F606809170
:107300002F09909130099093F9068093F8068091A7
:10731000590899279093FB068093FA06809161089B
:1073200099279093FD068093FC0680916908992720
:107330009093FF068093FE068091710899279093A1
:1073400001078093000780910403909105039093B7
:107350000B0780930A078091120A9091130A909369
:107360000F0780930E078091160A9091170A909349
:107370001107809310078091FF0390910004A09162
:107380000104B0910204BC01CD0125E030E040E0F1
:1073900050E00E94F29130931307209312078091DE
:1073A00021049091220490931907809318078091EB
:1073B000180A992790931D0780931C078091D50484
:1073C0009091D60490931F0780931E078091D30459
:1073D0009091D404909321078093200780915605C3
:1073E000882321F480915705882321F08091E106BC
:1073F000816003C08091E1068E7F8093E1061F913A
:107400000F91FF90EF900895EF92FF921F93CF930B
:10741000DF93182F7B0180910804882391F58091D8
:1074200001018C3010F0863111F4299801C0299A9D
:1074300011501F3FE9F0F0920B03E0920A03E701BD
:1074400080910A0390910B03892B11F4209781F30B
:1074500080910E038823A1F310920E0380910A03FA
:1074600090910B03892B09F421970E94E68EE8CFB7
:10747000809101018C3010F0863111F4299A01C0FD
:107480002998DF91CF911F91FF90EF900895CF93AE
:10749000DF93809101018D3011F40E94621E1092E1
:1074A0007A0080912A0390912B0390933B0980935B
:1074B0003A09809128039091290390932B09809396
:1074C0002A09809126039091270390937C09809349
:1074D0007B092091220330912303C901880F991F52
:1074E000880F991F820F931F820F931F9093770924
:1074F000809376092091240330912503C901880FD8
:10750000991F880F991F820F931F820F931F9093CB
:107510008709809386098FEC80937A00AAE0B4E013
:10752000CAE8D7E097E08991E82FFF27EE0FFF1F09
:10753000E754F74F0190F081E02DE158FF4F1E1600
:107540001F061CF0E0E0F0E005C0EF3FF10514F08D
:10755000EFEFF0E08C91282F3327E217F30714F4B4
:10756000815004C02E173F0714F48F5F8C93915005
:10757000119697FFD8CF8091C6079927AA27BB27D6
:10758000BC01CD0124EC39E040E050E00E947E9146
:10759000DC01CB018093820190938301A09384014D
:1075A000B09385018091C7079927AA27BB27BC0103
:1075B000CD010E947E91DC01CB0180937E019093EE
:1075C0007F01A0938001B0938101DF91CF91089555
:1075D000A0E0B0E0EEEEFAE30C941392882EC0E047
:1075E000D0E07E016E0110925605D0936F04C093D7
:1075F0006E04D0936D04C0936C04D0936904C0935F
:107600006804D0937904C0937804D0937704C0932E
:107610007604D0937504C0937404109264011092A0
:10762000630110921B030E94473A84E690E00E9497
:1076300091190E94473A8091920780FF10C0809173
:10764000150190911601875B934038F480911501E4
:10765000909116018E5E924010F40E94E01D0FE1A1
:107660008AE090E00E94911980912603909127036F
:10767000C80FD91F80912A0390912B03E80EF91EA1
:107680008091280390912903C80ED91E015007FF4D
:10769000E7CF9701205F3F4F369527953695279581
:1076A0003093790420937804C60140969695879587
:1076B0009695879590937704809376046096F5E08D
:1076C000D695C795FA95E1F7D0937504C0937404E5
:1076D0009093730480937204309371042093700428
:1076E000882009F441C0809176099091770997FF2D
:1076F00003C0909581959F4F6CE070E00E94BD9112
:107700009B0170936F0460936E0480918609909141
:10771000870997FF03C0909581959F4F6CE070E0BB
:107720000E94BD9170936D0460936C048091270753
:10773000909128079093690480936804B90184E0CC
:1077400090E00E94002F60916C0470916D0486E0BF
:1077500090E00E94002F609168047091690488E0B5
:1077600090E00E94002F65C084E090E00E94FB2E14
:1077700090936F0480936E0486E090E00E94FB2E4D
:1077800090936D0480936C0488E090E00E94FB2E3F
:107790009C01909369048093680480916E04909199
:1077A0006F048150984050F480916C0490916D0466
:1077B0008150984018F421503440D8F180E399E08A
:1077C0009F938F9380E695E19F938F93E0913D0582
:1077D000F0913E050995809176099091770997FF80
:1077E00003C0909581959F4F6CE070E00E94BD9121
:1077F00070936F0460936E0480918609909187095D
:1078000097FF03C0909581959F4F6CE070E00E94B8
:10781000BD9170936D0460936C04809127079091E3
:10782000280790936904809368040F900F900F903D
:107830000F9010923B0910923A0910922B09109266
:107840002A0910927C0910927B0984E690E00E943C
:10785000911980912203909123039C01220F331FE1
:10786000220F331F280F391F280F391F3093770934
:107870002093760980912403909125038C01000FB9
:10788000111F000F111F080F191F080F191F109348
:107890008709009386098091A107C82EDD24EE2474
:1078A000FF24442737FD4095542FC701B6010E949D
:1078B0007E914B015C016093630470936404809338
:1078C0006504909366049801442737FD4095542F32
:1078D000C701B6010E947E91DC01CB0180935B045D
:1078E00090935C04A0935D04B0935E048092430483
:1078F00090924404A0924504B092460480933B04C5
:1079000090933C04A0933D04B0933E041092330442
:1079100010923404109235041092360480911701AD
:1079200090911801A0911901B0911A0190932A0722
:107930008093290710921A031092190310922304BE
:1079400010922404109225041092260400918A01BA
:1079500010918B01109322040093210484E690E09F
:10796000909387018093860182E390E090930B03CC
:1079700080930A038091C6079927AA27BB27BC01D9
:10798000CD0124EC39E040E050E00E947E91DC0122
:10799000CB018856954CAF4FBF4F80938201909397
:1079A0008301A0938401B09385018091C707992733
:1079B000AA27BB27BC01CD010E947E91DC01CB012F
:1079C0008856954CAF4FBF4F80937E0190937F01B7
:1079D000A0938001B0938101109241011092400167
:1079E000C801AA2797FDA095BA2F20913C0130919C
:1079F0003D0140913E0150913F01BC01CD010E94EB
:107A00007E91DC01CB018093820990938309A0933E
:107A10008409B093850910921E0410921D040E94DF
:107A2000D86D8091D10384608093D1038FEF8093D0
:107A3000020A1092030A80E28093040ACAE0D4E0AA
:107A4000AAE8B7E007E08D91E82FFF27EE0FFF1FB0
:107A5000E754F74F8081918181588993015007FF46
:107A6000F2CF84E68093090480910803882311F003
:107A7000579A06C080E091E1909308018093070136
:107A8000809178049091790480569940815C9B4262
:107A900028F0809156058160809356058091760488
:107AA0009091770480569940815C9B4228F08091A8
:107AB00056058260809356058091740490917504F8
:107AC0008C5291408957954028F0809156058460EA
:107AD0008093560580916E0490916F048C52914072
:107AE000835C914028F0809156058860809356050C
:107AF00080916C0490916D048C529140835C914014
:107B000028F0809156058061809356058091680425
:107B100090916904805092408355914028F0809163
:107B2000560580628093560586E4809379010E9411
:107B3000C48BECE0CDB7DEB70C942F92A3E1B0E09C
:107B4000E4EAFDE30C940D92809174049091750425
:107B50002091260330912703821B930B90937C097D
:107B600080937B09809130039091310397FD0796B4
:107B70009C0113E0359527951A95E1F730933B0961
:107B800020933A0980912E0390912F0397FD079639
:107B9000B3E095958795BA95E1F790932B0980937B
:107BA0002A09309346092093450990933E09809312
:107BB0003D098091760990917709AC01440F551FDA
:107BC000480F591F2091220330912303C901880FC8
:107BD000991F880F991F820F931F820F931F480FC1
:107BE000591F57FF02C04D5F5F4F559547955595FB
:107BF0004795509377094093760980918609909133
:107C00008709AC01440F551F480F591F20912403C9
:107C100030912503C901880F991F880F991F820F82
:107C2000931F820F931F480F591F57FF02C04D5FCC
:107C30005F4F5595479555954795509387094093C4
:107C400086092091220330912303C901880F991FCF
:107C5000880F991F820F931F820F931F9C01442747
:107C600037FD4095542F8091530490915404A09176
:107C70005504B0915604820F931FA41FB51F809323
:107C8000530490935404A0935504B0935604209148
:107C9000240330912503C901880F991F880F991F6C
:107CA000820F931F820F931F9C01442737FD40953D
:107CB000542F80914F0490915004A0915104B091A1
:107CC0005204820F931FA41FB51F80934F049093FB
:107CD0005004A0935104B093520480914F099091A5
:107CE00050092091220330912303820F931F909318
:107CF000500980934F0980917E0990917F092091CE
:107D0000240330912503820F931F90937F09809362
:107D10007E0980916A0490916B04019690936B04A4
:107D200080936A0480912707909128072091680426
:107D300030916904821B930B9C01442737FD4095C9
:107D4000542F80914B0490914C04A0914D04B0911C
:107D50004E04820F931FA41FB51F80934B04909372
:107D60004C04A0934D04B0934E048FEC80937A00A2
:107D70001092110120913B0430913C0440913D044C
:107D800050913E0429873A874B875C8729543B46AC
:107D9000414050402CF028E43BE641E050E00DC06B
:107DA00089859A85AB85BC85885B9449AE4FBF4F6A
:107DB0004CF428EB34E94EEF5FEF2D833E834F8385
:107DC000588708C089859A85AB85BC858D839E833D
:107DD000AF83B88720914304309144044091450417
:107DE000509146042D873E874F87588B29543B4638
:107DF000414050402CF028E43BE641E050E00DC00B
:107E00008D859E85AF85B889885B9449AE4FBF4FFD
:107E10004CF428EB34E94EEF5FEF29833A834B8330
:107E20005C8308C08D859E85AF85B88989839A83D8
:107E3000AB83BC83A0917B09B0917C09BB8BAA8BDF
:107E4000FD01CF01AA2797FDA095BA2FA09033047A
:107E5000B0903404C0903504D0903604A80EB91EFA
:107E6000CA1EDB1EA0923304B0923404C0923504C3
:107E7000D0923604E0908209F09083090091840941
:107E800010918509E80EF91E0A1F1B1FE092820956
:107E9000F09283090093840910938509F091EC0313
:107EA000F98BFF2309F098C18091EB03882309F037
:107EB00093C18091720986FF8FC180912A099091A8
:107EC0002B09AA2797FDA095BA2FBC01CD012981C6
:107ED0003A814B815C810E947E919B01AC0197FFAE
:107EE00004C02150384F4F4F5F4FBBE05595479529
:107EF00037952795BA95D1F780916301682E77243D
:107F000088249924CA01B901A40193010E947E9199
:107F1000DC01CB018093840490938504A0938604B4
:107F2000B0938704B7FF04C08150904FAF4FBF4F4D
:107F30001C012D01ACE05594479437942794AA95E1
:107F4000D1F72092840430928504409286045092A6
:107F5000870480913A0990913B09AA2797FDA09543
:107F6000BA2FBC01CD012D813E814F8158850E94E1
:107F70007E9197FF04C06150784F8F4F9F4FFBE079
:107F80009595879577956795FA95D1F7A401930113
:107F90000E947E91DC01CB01809388049093890438
:107FA000A0938A04B0938B04B7FF04C08150904F14
:107FB000AF4FBF4F9C01AD01ECE05595479537950C
:107FC0002795EA95D1F7209388043093890440934C
:107FD0008A0450938B04809184049091850490933B
:107FE00022098093210980918804909189049093BB
:107FF000260980932509221933094409550920933C
:1080000088043093890440938A0450938B04E20ED1
:10801000F31E041F151FE0928209F092830900935A
:10802000840910938509809162018823B1F457FF78
:1080300004C02F5F3F4F4F4F5F4F55954795379582
:108040002795A21AB30AC40AD50AA0923304B092A3
:108050003404C0923504D09236042A893B897901D0
:108060000027F7FC0095102F8091880490918904D7
:10807000A0918A04B0918B04E80EF91E0A1F1B1F01
:10808000C801B70129813A814B815C810E947E91B0
:108090009B01AC0197FF04C02150384F4F4F5F4FF9
:1080A0006BE055954795379527956A95D1F780915F
:1080B0006401A82EBB24CC24DD24CA01B901A60189
:1080C00095010E947E91DC01CB0180937C0490930A
:1080D0007D04A0937E04B0937F04B7FF04C0815059
:1080E000904FAF4FBF4F3C014D013CE095948794BA
:1080F000779467943A95D1F760927C0470927D04EE
:1081000080927E0490927F04C801B7012D813E8148
:108110004F8158850E947E9197FF04C06150784F2F
:108120008F4F9F4F2BE095958795779567952A956B
:10813000D1F7A60195010E947E91DC01CB018093CD
:10814000800490938104A0938204B0938304B7FFCA
:1081500004C08150904FAF4FBF4FAC01BD018CE0C8
:1081600075956795579547958A95D1F74093800403
:108170005093810460938204709383042A893B891D
:1081800037FF03C0309521953F4F21343105E4F18D
:10819000D401C30197FE07C0B095A0959095819535
:1081A0009F4FAF4FBF4F81389105A105B10584F4B2
:1081B000DB01CA0177FF07C0B095A0959095819526
:1081C0009F4FAF4FBF4F81389105A105B105E4F036
:1081D00081E080931F0418C010922609109225098F
:1081E00010922209109221091092800410928104A9
:1081F000109282041092830410927C0410927D04E9
:1082000010927E0410927F048091800490918104EA
:10821000A0918204B0918304BC01CD0124E630E03A
:1082200040E050E00E94F291E0907C04F0907D04E8
:10823000E21AF30AF0923909E092380980917C043D
:1082400090917D04A0917E04B0917F04BC01CD018A
:1082500024E630E040E050E00E94F291DA01C901EA
:1082600020918004309181048C01021B130B109328
:108270002D0900932C0980913C0190913D01A09122
:108280003E01B0913F01BC01CD0128E631E040E064
:1082900050E00E947E9120918209309183094091A3
:1082A000840950918509261737074807590764F054
:1082B000261B370B480B590B2093820930938309F7
:1082C0004093840950938509209182093091830954
:1082D000409184095091850957FF0CC0260F371F24
:1082E000481F591F209382093093830940938409C2
:1082F0005093850960912A0970912B096E0D7F1D9D
:108300009B01442737FD4095542F8091370490916D
:108310003804A0913904B0913A04820F931FA41F2E
:10832000B51F8093370490933804A0933904B09319
:108330003A048091F1039091F203681B790BCB0111
:10834000AA2797FDA095BA2F29853A854B855C858C
:10835000820F931FA41FB51F80933B0490933C048E
:10836000A0933D04B0933E04C0907E01D0907F0165
:10837000E0908001F0908101C816D906EA06FB065C
:10838000C4F488EA91E6A0E0B0E08C199D09AE093A
:10839000BF0980933B0490933C04A0933D04B093A9
:1083A0003E048093370490933804A0933904B0932B
:1083B0003A0422273327A9012C193D094E095F09E8
:1083C00080913B0490913C04A0913D04B0913E0407
:1083D00082179307A407B507B4F4D701C601885ADA
:1083E0009146A040B04080933B0490933C04A093FE
:1083F0003D04B0933E048093370490933804A093D7
:108400003904B0933A0460913A0970913B09600FC6
:10841000711F9B01442737FD4095542F80913F04E5
:1084200090914004A0914104B0914204820F931FA7
:10843000A41FB51F80933F0490934004A093410470
:10844000B09342048091EF039091F003681B790B85
:10845000CB01AA2797FDA095BA2F2D853E854F8584
:108460005889820F931FA41FB51F809343049093D4
:108470004404A0934504B0934604E0908201F09038
:1084800083010091840110918501E816F9060A071D
:108490001B07C4F488EA91E6A0E0B0E08E199F09BA
:1084A000A00BB10B8093430490934404A093450424
:1084B000B093460480933F0490934004A0934104FA
:1084C000B093420422273327A9012E193F09400BFC
:1084D000510B8091430490914404A0914504B091C4
:1084E000460482179307A407B507B4F4D801C7015F
:1084F000885A9146A040B04080934304909344042E
:10850000A0934504B093460480933F0490934004A5
:10851000A0934104B09342048091330490913404B9
:10852000A0913504B0913604809347049093480499
:10853000A0934904B0934A04809143049091440469
:10854000A0914504B0914604809363049093640421
:10855000A0936504B093660480913B0490913C0421
:10856000A0913D04B0913E0480935B0490935C0421
:10857000A0935D04B0935E0480913F049091400409
:10858000A0914104B091420480935F0490936004F1
:10859000A0936104B09362048091370490913804F1
:1085A000A0913904B0913A048093570490935804F1
:1085B000A0935904B0935A0480911D0190911E011B
:1085C00097FD079603E0959587950A95E1F79093B7
:1085D0003B0980933A0980911B0190911C0197FD02
:1085E000079613E0959587951A95E1F790932B09D7
:1085F00080932A0980912A0390912B030F9734F4DA
:1086000088E19CEF90933B0980933A0980912A037B
:1086100090912B03079734F480E398EF90933B09F4
:1086200080933A09209101012A30A9F480912A030C
:1086300090912B03835F934034F088EE93E0909306
:108640003B0980933A0980912A0390912B038A5F1A
:108650009340DCF014C080912A0390912B03815D3C
:10866000974034F088EE93E090933B0980933A0969
:1086700080912A0390912B03805E974034F080ED27
:1086800097E090933B0980933A0980912803909159
:1086900029030F9734F488E19CEF90932B09809382
:1086A0002A098091280390912903079734F480E3E5
:1086B00098EF90932B0980932A092A30A9F480918E
:1086C000280390912903835F934034F088EE93E070
:1086D00090932B0980932A09809128039091290374
:1086E0008A5F9340DCF014C08091280390912903A5
:1086F000815D974034F088EE93E090932B0980934E
:108700002A098091280390912903805E974034F0D4
:1087100080ED97E090932B0980932A096091700176
:10872000662309F4AFC040911D0150911E01809154
:108730008C0490918D04481B590B509393044093E3
:10874000920420911D0130911E01280F391F37FF1F
:1087500002C02F5F3F4F3595279530938D042093AE
:108760008C04413851051CF080E890E005C0405869
:108770005F4F34F480E89FEF9093930480939204CA
:1087800040911B0150911C0180918E0490918F04A7
:10879000481B590B509391044093900420911B0166
:1087A00030911C01280F391F37FF02C02F5F3F4F48
:1087B0003595279530938F0420938E0441385105C9
:1087C0001CF080E890E005C040585F4F34F480E82A
:1087D0009FEF9093910480939004462F55278091AA
:1087E000920490919304849FB001859F700D949F93
:1087F000700D11249B0177FF02C0215F3F4FF4E011
:1088000035952795FA95E1F780913A0990913B09C2
:10881000820F931F90933B0980933A0980919004B3
:1088200090919104849FD001859FB00D949FB00DCD
:108830001124AD019D01B7FF02C0215F3F4FE4E06D
:1088400035952795EA95E1F780912A0990912B09B2
:10885000820F931F90932B0980932A0980911D0109
:1088600090911E01860F971F90931E0180931D010A
:1088700080911B0190911C01840F951F90931C0106
:1088800080931B0100913D0910913E0980912109BF
:1088900090912209101611065CF59C0197FF04C007
:1088A00022273327281B390BC901AA2797FDA0953A
:1088B000BA2F20916201332744275527BC01CD01EF
:1088C0000E947E919B01AC0197FF04C0215C3F4F49
:1088D0004F4F5F4F76E055954795379527957A9599
:1088E000D1F78091380990913909820F931F27C0E1
:1088F00097FF03C0909581959F4FAA2797FDA0955C
:10890000BA2F20916201332744275527BC01CD019E
:108910000E947E919B01AC0197FF04C0215C3F4FF8
:108920004F4F5F4F66E055954795379527956A9568
:10893000D1F78091380990913909821B930B90935C
:10894000390980933809E0904509F09046098091F3
:108950002509909126091E141F045CF59C0197FFC0
:1089600004C022273327281B390BC901AA2797FDEA
:10897000A095BA2F20916201332744275527BC01C7
:10898000CD010E947E919B01AC0197FF04C0215C48
:108990003F4F4F4F5F4F96E0559547953795279539
:1089A0009A95D1F780912C0990912D09820F931FF0
:1089B00027C097FF03C0909581959F4FAA2797FDE9
:1089C000A095BA2F20916201332744275527BC0177
:1089D000CD010E947E919B01AC0197FF04C0215CF8
:1089E0003F4F4F4F5F4F86E05595479537952795F9
:1089F0008A95D1F780912C0990912D09821B930BB8
:108A000090932D0980932C098091720987FF44C0AF
:108A1000B989BB2309F040C08091EB038823E1F5BD
:108A2000E1E0EE16E1E0FE064CF080913A0990910B
:108A30003B098E0D9F1D805091400DC0F0E0EF1658
:108A4000FFEFFF0664F480913A0990913B098E0D87
:108A50009F1D80509F4F90933B0980933A0921E0DE
:108A6000013012074CF080912A0990912B09800F58
:108A7000911F805091400CC03FEF0030130764F409
:108A800080912A0990912B09800F911F80509F4F50
:108A900090932B0980932A09E2E1CD5E0C942992F0
:108AA00080910804882301F58091D1038C7F809305
:108AB000D103ABE5B5E0E8E5F8E09BE08091E902A1
:108AC000882309F48C938D9181831282915038967A
:108AD00097FFF4CF8091E902882359F08091E90251
:108AE00081508093E90205C08091D1038160809319
:108AF000D10380915103882319F0109251030895F6
:108B0000809353038093550380914F038E7F80930E
:108B10004F0385EA8093BC000895CF93DF93AAE0CA
:108B2000B4E0CAE8D7E057E09991E92FFF27EE0FAC
:108B3000FF1FE754F74F0190F081E02DE158FF4F00
:108B4000EF3FF10521F01CF0EFEFF0E004C0F7FF7C
:108B500002C0E0E0F0E0993111F4EC931BC04C91BD
:108B6000242F3327E217F307A9F0CF01821B930BC1
:108B700097FD03969595879595958795242F280FB2
:108B80002C93822F9927E817F90714F4215001C07C
:108B90002F5F2C935150119657FFC6CF80919407A9
:108BA000883F38F0EFEFF0E0E81BF109E65FFB4F9C
:108BB00080818093760180917601882329F0843624
:108BC00018F084E68093760180919607883F38F00C
:108BD000EFEFF0E0E81BF109E65FFB4F8081809347
:108BE000740180917401882329F0843618F084E69A
:108BF000809374018091A307883F38F0EFEFF0E095
:108C0000E81BF109E65FFB4F808180936F01809143
:108C10006F018B3010F48AE002C08F3F11F4809313
:108C20006F018091D007883F38F0EFEFF0E0E81B4C
:108C3000F109E65FFB4F80818093510980915109D2
:108C4000863010F485E002C08F3F11F48093510903
:108C50008091D207883F38F0EFEFF0E0E81BF10990
:108C6000E65FFB4F80818093790980917909863096
:108C700010F485E002C08F3F11F480937909809150
:108C8000BD07873F19F4429905C006C0863F31F4FD
:108C9000439B02C08CE80BC086E409C0883F38F0D3
:108CA000EFEFF0E0E81BF109E65FFB4F8081809376
:108CB0004E098091BE07873F19F4429905C006C04E
:108CC000863F31F4439B02C08CE80BC086E409C0A8
:108CD000883F38F0EFEFF0E0E81BF109E65FFB4F6B
:108CE0008081809327098091BF07883F38F0EFEF9C
:108CF000F0E0E81BF109E65FFB4F808180935709A4
:108D000080919507883F38F0EFEFF0E0E81BF1091C
:108D1000E65FFB4F80818093750180919807883FC3
:108D200038F0EFEFF0E0E81BF109E65FFB4F8081E0
:108D30008093730180919A07883F38F0EFEFF0E05D
:108D4000E81BF109E65FFB4F808180937101809100
:108D5000A207883F38F0EFEFF0E0E81BF109E65F8B
:108D6000FB4F8081809372018091A407883F38F087
:108D7000EFEFF0E0E81BF109E65FFB4F80818093A5
:108D80006E018091A507883F38F0EFEFF0E0E81B17
:108D9000F109E65FFB4F8081809370018091A60707
:108DA000883F38F0EFEFF0E0E81BF109E65FFB4F9A
:108DB000808180936D018091A707883F38F0EFEFA5
:108DC000F0E0E81BF109E65FFB4F808180936C01C6
:108DD0008091AD07883F38F0EFEFF0E0E81BF10934
:108DE000E65FFB4F808180936A018091AE07883FE8
:108DF00038F0EFEFF0E0E81BF109E65FFB4F808110
:108E00008093E6038091AF07883F38F0EFEFF0E002
:108E1000E81BF109E65FFB4F80818093E5038091B9
:108E2000B007883F38F0EFEFF0E0E81BF109E65FAC
:108E3000FB4F80818093E4038091B107883F38F035
:108E4000EFEFF0E0E81BF109E65FFB4F80818093D4
:108E5000E3038091CB07883F38F0EFEFF0E0E81BA9
:108E6000F109E65FFB4F80818093E2038091CC079C
:108E7000883F38F0EFEFF0E0E81BF109E65FFB4FC9
:108E800080818093E1038091CD07883F38F0EFEF38
:108E9000F0E0E81BF109E65FFB4F80818093E0037F
:108EA0008091CE07883F38F0EFEFF0E0E81BF10942
:108EB000E65FFB4F80818093DF038091B207883F9C
:108EC00038F0EFEFF0E0E81BF109E65FFB4F80813F
:108ED000809369018091B607883F38F0EFEFF0E0AA
:108EE000E81BF109E65FFB4F808180936801809168
:108EF000B307883F38F0EFEFF0E0E81BF109E65FD9
:108F0000FB4F8081809367018091B707883F38F0DD
:108F1000EFEFF0E0E81BF109E65FFB4F8081809303
:108F200066018091C007883F38F0EFEFF0E0E81B62
:108F3000F109E65FFB4F8081809365018091C30753
:108F4000883F38F0EFEFF0E0E81BF109E65FFB4FF8
:108F50008081809364018091C407883F38F0EFEFEF
:108F6000F0E0E81BF109E65FFB4F8081809363012D
:108F70008091C507883F38F0EFEFF0E0E81BF1097A
:108F8000E65FFB4F8081809362018091ED07883F0F
:108F900038F0EFEFF0E0E81BF109E65FFB4F80816E
:108FA000809336099091DF04992321F0809136094E
:108FB000981720F080913609882311F49093360990
:108FC00080919207809372098091F30780935609EC
:108FD0008091CA07883F38F0EFEFF0E0E81BF10915
:108FE000E65FFB4F8081809361018091E607883FB7
:108FF00038F0EFEFF0E0E81BF109E65FFB4F80810E
:109000008093890980916A01282F33272F5F3F4F72
:109010008CE398E2B9010E94BD917093780160934E
:1090200077018091A00780937A0980919F078093B0
:109030003F099091E807933308F44AC081E0809398
:10904000DE03983F58F0EFEFF0E0E91BF109E65F2F
:10905000FB4F8081823310F41092DE0380917901FE
:109060002091DE03821721F18330F8F430919F01C3
:10907000222351F08CED95E090930B0380930A032B
:10908000332369F48EE209C088EC90E090930B03DF
:1090900080930A03332319F487E180939F0185E0CD
:1090A0008093F3032093790103C081508093790169
:1090B0008091C9099091CA0997FF0FC08091DE0382
:1090C000882359F08091560580688093560505C025
:1090D0001092DE038AE0809379018091C909909112
:1090E000CA0997FF1DC0809108048823C9F08091A8
:1090F000DE038823A9F08091090190910A018F5F16
:109100009F4F71F488E99AE390930B0380930A03CD
:1091100080E094EA90930A01809309011092DE03A3
:109120008091DE03882369F08091D0038160809371
:10913000D00380916401823D48F4825E8093640193
:1091400005C08091D0038E7F8093D003DF91CF91B3
:109150000895A7E1B0E0EFEAF8E40C940D920E94C4
:109160009E3D8091D103992784719070892B91F550
:109170008091F40782FF27C08091ED039091EE0368
:109180000097F1F002E088359007D4F49C0197FF36
:1091900002C02D5F3F4F35952795359527958091D6
:1091A000AA079927289FA001299F500D389F500D8D
:1091B0001124CA0164E670E00E94BD91CB0106C093
:1091C0008DE290E003C08091AA0799279093CF0386
:1091D0008093CE032091CC033091CD0355E720330B
:1091E000350759F4109214041092130480913F092A
:1091F00099279093CF038093CE03609113047091CD
:1092000014047A83698380913F0999270A96681725
:10921000790714F49A83898380910904843608F0CD
:109220006AC08091D00382FD66C08091A8049091AD
:10923000A904009731F001979093A9048093A804A2
:109240000BC0109208049093D3038093D2038091B3
:10925000D1038D7E8093D103809101018A3011F07A
:10926000843110F0289A01C028988091D2039091FF
:10927000D303895E9340E0F18091180A8536C0F1EE
:109280008091CE039091CF039A8389838091D103FB
:1092900080618093D10380918607A82FBB27AA0FF6
:1092A000BB1FFD01E351F74F1182108280918707A8
:1092B000282F3327220F331FC9018351974FFC01F9
:1092C00011821082A754B74F11961C921E922754F8
:1092D000374FD90111961C921E9280918907E82F71
:1092E000FF27EE0FFF1FE754F74F118210823FC395
:1092F000109208043CC3809109048D3808F40DC312
:109300008091D1038F7E8093D1039091AB0782E34C
:10931000989FC00111249093A9048093A804E98127
:10932000FA81B9978CF080910804882369F08091C4
:10933000D2039091D303FFEF8F3F9F0729F001964F
:109340009093D3038093D2038091D2039091D3035F
:109350008F3F910509F008F510922B0410922C0410
:1093600010922D0410922E041092270410922804BB
:109370001092290410922A041092940410929504D9
:1093800010929604109297041092330410923404B1
:10939000109235041092360405C08091D10382608A
:1093A0008093D10380918807E82FFF27EE0FFF1FDE
:1093B000E754F74F80819181813591050CF438C1D4
:1093C00020910804222309F033C180918907E82FF6
:1093D000FF27EE0FFF1FE754F74F808191818C34F8
:1093E00091050CF4FFC08091AA048F5F8093AA04BA
:1093F000893C08F41DC12093AA041092D303109253
:10940000D20330918607E32FFF27EE0FFF1FE754AB
:10941000F74F8081918187349105B4F4809187075B
:10942000E82FFF27EE0FFF1FE754F74F8081918150
:109430000190F081E02DF7FF03C0F095E195FF4F1B
:10944000E734F1050CF478C041E020918707A22FA2
:10945000BB27AA0FBB1FA754B74F8D919C911197A3
:109460008734910544F0E32FFF27EE0FFF1FE754E9
:10947000F74F808191818D919C918734910574F093
:1094800080918607E82FFF27EE0FFF1FE754F74F65
:1094900080819181873491050CF042E0E22FFF2713
:1094A000EE0FFF1FE754F74F8081918186349105BD
:1094B00074F480918607E82FFF27EE0FFF1FE75413
:1094C000F74F80819181873491050CF043E0E22FC2
:1094D000FF27EE0FFF1FE754F74F808191818A5BD2
:1094E0009F4F74F480918607E82FFF27EE0FFF1F30
:1094F000E754F74F80819181873491050CF044E067
:10950000E22FFF27EE0FFF1FE754F74F8081918175
:109510008A5B9F4F74F480918607E82FFF27EE0F38
:10952000FF1FE754F74F80819181863491050CF439
:1095300045E0842F0E945A2F80918707E82FFF274C
:10954000EE0FFF1FE754F74F808191810190F0816A
:10955000E02DF7FF03C0F095E195FF4F7E97CCF427
:1095600080918607E82FFF27EE0FFF1FE754F74F84
:10957000808191818A5B9F4F64F481E080937105C3
:109580001092F40388EE93E090930B0380930A0308
:109590004FC00E9463300E94052F80E00E94910915
:1095A0008091AC070E947A8D8091720980FF10C073
:1095B0008091150190911601875B934038F480915A
:1095C0001501909116018E5E924010F40E94E01DEC
:1095D00080E00E94E83A81E08093F40380930803DE
:1095E000579A1AC080819181855B9F4FFCF48091CE
:1095F000AA048F5F8093AA04893CD0F020930804CA
:109600002093AA041092D3031092D20381E00E9407
:10961000E83A81E08093F40388E180939F010E94FF
:10962000633068E770E00E94043A02C02093AA0405
:1096300080918807E82FFF27EE0FFF1FE754F74FB1
:10964000808191818B5A9F4F0CF060C12091E90776
:10965000E22FFF27EF77F070EE0FFF1FE351F74F78
:1096600080819181069714F084E606C08081918103
:109670008B5F9F4F1CF48CE98093AD0480910804AC
:10968000E0918907882309F0ECC0FF27EE0FFF1F48
:10969000E754F74F80819181855B9F4F9CF48091C7
:1096A000F40783FD0BC0E22FFF27EE0FFF1FE754E7
:1096B000F74F80819181855B9F4FDCF08091E907B6
:1096C0008823B9F08091F40783FFC8C08091E9072F
:1096D000E82FFF27EE0FFF1FE754F74F808191819E
:1096E000875F9F4F0CF4BAC08091AD04843609F0B7
:1096F000B5C02091F403222329F08091D103886022
:109700008093D1038091AB048F5F8093AB048E3F35
:1097100008F4EEC01092AB0480915605882309F03E
:1097200092C0222309F48FC08091E404882309F0B9
:109730008AC081E090E09093D3038093D20381E0CC
:109740008093080410929404109295041092960449
:10975000109297041092330410923404109235043E
:109760001092360410922F0410923004109231049B
:10977000109232048091A107E82EFF2400271127C0
:1097800080917609909177099C01442737FD409597
:10979000542FC801B7010E947E91DC01CB01809358
:1097A000430490934404A0934504B09346048091ED
:1097B0008609909187099C01442737FD4095542FD5
:1097C000C801B7010E947E91DC01CB0180933B046C
:1097D00090933C04A0933D04B0933E0480916304B5
:1097E00090916404A0916504B091660480933F0455
:1097F00090934004A0934104B093420480915B0491
:1098000090915C04A0915D04B0915E048093370454
:1098100090933804A0933904B0933A0410922B0427
:1098200010922C0410922D0410922E0410922704F2
:10983000109228041092290410922A0484E680933E
:10984000F30384E350C08CED95E090930B03809379
:109850000A03222309F04CC081E045C01092AB04FA
:1098600047C0FF27EE0FFF1FE754F74F808191811C
:109870008C3491059CF08091F40783FD0BC0E22F9E
:10988000FF27EE0FFF1FE754F74F80819181855B23
:109890009F4FCCF08091E9078823A9F08091F407CD
:1098A00083FF24C08091E907E82FFF27EE0FFF1FF9
:1098B000E754F74F808191818E5C9F4FBCF480917B
:1098C000AD048C3999F48091AC048F5F8093AC0423
:1098D0008B3F70F0109208041092AC041092D303E6
:1098E0001092D20386E280939F0102C01092AC04D2
:1098F0008091CC039091CD0313E0883E9107B8F599
:1099000001969093CD038093CC0331C01092AD04A7
:109910001092CD031092CC032AC02E5E324038F153
:1099200080919109909192098059914000F5809120
:10993000030490910404A0910504B09106048C5D89
:109940009540A040B0409CF480E395E79093CD0310
:109950008093CC038091D2039091D3038A5E93408D
:1099600030F089EE93E09093D3038093D2038091FB
:109970003A01815080933A0180913A018F3F21F062
:109980008091D10384FFA9C30E948D45B0909C07AC
:109990008091B6049091B7049C01220F331F280FC9
:1099A000391FC0908607AC2DBB27AA0FBB1FFD0136
:1099B000E754F74F4B2D552780819181849FF0010B
:1099C000859FF00D949FF00D11242E0F3F1F37FF40
:1099D00002C02D5F3F4FB9017595679575956795E5
:1099E000A351B74F80919D07082F11278D919C910E
:1099F000809F7001819FF00C909FF00C11246E0DE0
:109A00007F1D7093B7046093B6048091B804909161
:109A1000B9049C01220F331F280F391FD0908707EC
:109A2000AD2DBB27AA0FBB1FFD01E754F74F808167
:109A30009181849FF001859FF00D949FF00D11247A
:109A40002E0F3F1F37FF02C02D5F3F4FA9015595D5
:109A5000479555954795A351B74F8D919C91809F00
:109A60007001819FF00C909FF00C11244E0D5F1D32
:109A70005093B9044093B8048091DE03882309F41D
:109A800048C0CB0177FD0396DC01B595A795B59548
:109A9000A795CA0157FD0396FC01F595E795F59545
:109AA000E79580919A01682F772767FD70956A9FE7
:109AB00090016B9F300D7A9F300D11248091E60448
:109AC000482F552747FD50954E9FC0014F9F900D41
:109AD0005E9F900D1124280F391F37FF02C0295FA8
:109AE0003F4F93E0359527959A95E1F730931A0407
:109AF000209319046E9F90016F9F300D7E9F300D53
:109B000011244A9FC0014B9F900D5A9F900D112424
:109B10003FC08091E707E82FFF27EE5BFE4F86816D
:109B200080939A0190819093E604A82FBB27A7FD0C
:109B3000B095A69F9001A79F300DB69F300D1124C0
:109B4000E92FFF27E7FDF095E49FC001E59F900D09
:109B5000F49F900D1124280F391F37FF02C0295F91
:109B60003F4F83E0359527958A95E1F730931A04A6
:109B700020931904A49F9001A59F300DB49F300D30
:109B80001124E69FC001E79F900DF69F900D1124D0
:109B9000281B390B37FF02C0295F3F4F03E0359583
:109BA00027950A95E1F730931804209317048091C4
:109BB0008907E82FFF27EE0FFF1FE754F74F80813B
:109BC0009181909581959F4F9093160480931504F1
:109BD0008530910514F0049705C00FEF8C3F900776
:109BE00034F40496909316048093150404C01092E4
:109BF0001604109215048091D204882309F43EC003
:109C0000282F33278091190490911A0497FD079605
:109C100013E0959587951A95E1F7289FA001299F54
:109C2000500D389F500D1124CA0157FD0F96B4E016
:109C300095958795BA95E1F790931A048093190446
:109C4000809117049091180497FD0796A3E09595CD
:109C50008795AA95E1F7289FB001299F700D389F3D
:109C6000700D1124CB0177FD0F96F4E09595879543
:109C7000FA95E1F7909318048093170480901904E3
:109C800090901A048091D5049091D604881A990A6C
:109C900090921A04809219040091170410911804EC
:109CA0008091D3049091D404081B190B10931804CD
:109CB0000093170480918807E82FFF27EE0FFF1FFE
:109CC000E754F74FE080F1808FE790E0E80EF91E4F
:109CD000F0921404E092130480916F019927AA274F
:109CE00097FDA095BA2FBC01CD010E94F290DC0136
:109CF000CB0120E030E040E251E4BC01CD010E9404
:109D00006090DC01CB01BC01CD010E94C490DC015C
:109D1000CB018093800980916E01809358098091D6
:109D20006D019927AA2797FDA095BA2FBC01CD01F7
:109D30000E94F290DC01CB0120E030E040E251E4EF
:109D4000BC01CD010E946090DC01CB01BC01CD01C2
:109D50000E94C490DC01CB018093310980916C0199
:109D60008093470980917D0580FF59C080918909C2
:109D7000813808F454C080917605992787FD909525
:109D80002B2D3327829FD001839FB00D929FB00D62
:109D900011248A0E9B1E90921A04809219048091BD
:109DA0007705992787FD9095829FF001839FF00D9D
:109DB000929FF00D11240E0F1F1F10931804009393
:109DC000170480917805282F332727FD309580913F
:109DD000150490911604820F931F9093160480939C
:109DE000150480917A05282F332727FD309580911F
:109DF00097079927289F8001299F100D389F100DE4
:109E00001124109341010093400180917905992715
:109E10008E159F0524F4909314048093130480916D
:109E200013049091140497FF04C01092140410922C
:109E300013048091720982FF02C010925809409168
:109E4000190450911A04CA0157FD03969C013595D7
:109E500027953595279537FF03C0309521953F4FBE
:109E60008091D6039091D70382179307B4F4CA0167
:109E700057FF03C0909581959F4F97FD0396959549
:109E80008795959587959093D7038093D6038536CC
:109E9000910544F084E690E001C001979093D703C8
:109EA0008093D6034091170450911804CA0157FDBE
:109EB00003969C01359527953595279537FF03C067
:109EC000309521953F4F8091D4039091D50382170F
:109ED0009307B4F4CA0157FF03C0909581959F4F33
:109EE00097FD039695958795959587959093D503BE
:109EF0008093D4038536910544F084E690E001C058
:109F000001979093D5038093D4038091D10384FF6C
:109F100008C01092D7031092D6031092D503109266
:109F2000D403ED2DFF27EE0FFF1FE754F74F4091AD
:109F3000C107242F3327808191812817390744F4E2
:109F40008091F10782FF04C081E08093EA0313C08F
:109F5000ED2DFF27EE0FFF1FE754F74F842F9927B2
:109F60002091C207821B910920813181281739076E
:109F700014F41092EA0340918707E42FFF27EE0FB5
:109F8000FF1FE754F74F5091C107852F99272227CC
:109F90003327281B390B808191818217930744F462
:109FA0008091F10783FF04C081E08093E90316C02C
:109FB0008091E903882391F0E42FFF27EE0FFF1F24
:109FC000E754F74F8091C2079927851B910920819B
:109FD00031818217930714F41092E903EC2DFF27C7
:109FE000EE0FFF1FE754F74F4091C107242F33278F
:109FF000808191812817390744F48091F10780FF0F
:10A0000004C081E08093E70317C08091E7038823B1
:10A0100099F0EC2DFF27EE0FFF1FE754F74F842F29
:10A0200099272091C207821B91092081318128172D
:10A03000390714F41092E70340918607E42FFF27B5
:10A04000EE0FFF1FE754F74F5091C107852F992757
:10A0500022273327281B390B808191818217930790
:10A0600044F48091F10781FF04C081E08093E8030C
:10A0700016C08091E803882391F0E42FFF27EE0FAC
:10A08000FF1FE754F74F8091C2079927851B91095D
:10A09000208131818217930714F41092E803809194
:10A0A000EA03882319F48091E903811181E0809308
:10A0B000EB038091E703882321F48091E803882350
:10A0C00051F081E08093EC031092EB031092EA03CD
:10A0D0001092E90302C08093EC038091EB03882384
:10A0E00021F48091EC03882369F08091C0079927BF
:10A0F00029813A818217930714F49A83898381E036
:10A1000080931F048091D00399279C0124703070A4
:10A1100082FF2DC08091D5049091D60490958195B1
:10A120009F4F90931A04809319048091D3049091C7
:10A13000D404909581959F4F9093180480931704B1
:10A1400080917C0190917D0190931404809313047D
:10A15000809172098B778B66809372098091560982
:10A160008C7B8093560988EC809375011EC080918A
:10A17000D10384FF1AC03093160420931504309342
:10A180001A042093190430931804209317049AE5B5
:10A190009093800988E780935809909331098093C0
:10A1A00047091092EB031092EC0380914A099091B9
:10A1B0004B09A0914C09B0914D0920916304309155
:10A1C00064044091650450916604820F931FA41F9C
:10A1D000B51F80934A0990934B09A0934C09B09303
:10A1E0004D098091520990915309A0915409B09161
:10A1F0005509E0905B04F0905C0400915D041091BF
:10A200005E04EB82FC820D831E838E0D9F1DA01FBA
:10A21000B11F8093520990935309A0935409B093AE
:10A2200055098091410990914209A0914309B0914B
:10A230004409E0905F04F090600400916104109183
:10A240006204EF82F88609871A878E0D9F1DA01F72
:10A25000B11F8093410990934209A0934309B093A1
:10A2600044098091320990913309A0913409B09149
:10A270003509E0905704F09058040091590410916A
:10A280005A04EB86FC860D871E878E0D9F1DA01F2E
:10A29000B11F8093320990933309A0933409B0938E
:10A2A0003509F090EC03FF86FF2029F48091EB0341
:10A2B000882309F460C01092530410925404109241
:10A2C00055041092560410924F04109250041092AC
:10A2D00051041092520410924A0910924B091092A4
:10A2E0004C0910924D091092520910925309109284
:10A2F0005409109255091092410910924209109286
:10A3000043091092440910923209109233091092B5
:10A310003409109235098091430490914404A0912E
:10A320004504B091460480933F0490934004A09369
:10A330004104B093420480913B0490913C04A0916D
:10A340003D04B0913E048093370490933804A09369
:10A350003904B0933A041092180310921703109224
:10A36000F0031092EF031092F2031092F1030F85A5
:10A37000002309F0D0C18091EB03882309F0CBC101
:10A380008091270790912807815092402CF480916A
:10A390000804882309F4BFC19090020AA090A10785
:10A3A000209076093090770940908609509087096F
:10A3B00019140CF0BBC0BB24CC24DD24CA01B901A4
:10A3C000A60195010E94F29179018A018091CB0941
:10A3D0009091CC09281A390AC101AA2797FDA095A6
:10A3E000BA2FE81AF90A0A0B1B0B6B817C818D814D
:10A3F0009E81A60195010E94F29159016A01809106
:10A40000CD099091CE09481A590AC201AA2797FD91
:10A41000A095BA2FA81AB90ACA0ADB0A292C332434
:10A4200027FC3094432C532CC801B701A2019101A1
:10A430000E947E9197FF04C061507E4F8F4F9F4FC7
:10A440003B014C0109E095948794779467940A95B1
:10A45000D1F7C601B501A20191010E947E9197FF3B
:10A4600004C061507E4F8F4F9F4F5B016C0119E01C
:10A47000D594C794B794A7941A95D1F78091D60331
:10A480009091D703813491053CF48091D40390914D
:10A49000D50381349105D4F0D401C30197FE03C0E4
:10A4A0000196A11DB11D3C014D01959487947794AF
:10A4B0006794D601C501D7FE03C00196A11DB11D49
:10A4C0005C016D01D594C794B794A7948091040A58
:10A4D000282F332727FD3095432F532F2615370577
:10A4E0004805590514F439014A01992787FD9095CB
:10A4F000909581959F4FAA2797FDA095BA2F681632
:10A5000079068A069B0614F43C014D012A153B0589
:10A510004C055D0514F459016A01A816B906CA066E
:10A52000DB060CF0D0C05C016D01CDC0EA2CFF242D
:10A5300000271127CA01B901A80197010E94F291D1
:10A5400039014A01C101AA2797FDA095BA2F681ABF
:10A55000790A8A0A9B0A6B817C818D819E81A80180
:10A5600097010E94F29159016A01C201AA2797FD41
:10A57000A095BA2FA81AB90ACA0ADB0AD401C301E6
:10A5800097FE03C00F96A11DB11D3C014D01F4E0E3
:10A590009594879477946794FA95D1F7D601C5017D
:10A5A000D7FE03C00F96A11DB11D5C016D01E4E053
:10A5B000D594C794B794A794EA95D1F78091D60320
:10A5C0009091D703813491053CF48091D40390910C
:10A5D000D50381349105A4F0C401B30123E030E038
:10A5E00040E050E00E94F29139014A01C601B501F4
:10A5F00023E030E040E050E00E94F29159016A010E
:10A6000080918907E82FFF27EE0FFF1FE754F74FD0
:10A61000808191810190F081E02DF7FF03C0F095DA
:10A62000E195FF4F7A97A4F0C401B30123E030E035
:10A6300040E050E00E94F29139014A01C601B501A3
:10A6400023E030E040E050E00E94F29159016A01BD
:10A6500089E18093880121E26216710481049104EA
:10A660002CF070E2672E712C812C912C30EE631649
:10A670003FEF73063FEF83063FEF930644F460EE2F
:10A68000662E6FEF762E6FEF862E6FEF962E41E2DD
:10A69000A416B104C104D1042CF050E2A52EB12CB3
:10A6A000C12CD12C50EEA5165FEFB5065FEFC506A5
:10A6B0005FEFD50644F440EEA42E4FEFB42E4FEFDB
:10A6C000C42E4FEFD42E8091430490914404A09166
:10A6D0004504B091460486199709A809B9098093E1
:10A6E000430490934404A0934504B093460480919E
:10A6F0003B0490913C04A0913D04B0913E048A1922
:10A700009B09AC09BD0980933B0490933C04A09342
:10A710003D04B0933E0480911703909118038F3F3E
:10A72000910509F008F4C4C56F85662309F04EC58C
:10A730008091EB03882309F049C580911F04882389
:10A7400009F044C57091C907788B772309F43EC599
:10A7500080914A0990914B09A0914C09B0914D0903
:10A76000B7FF04C081509F4FAF4FBF4FE92EFA2E65
:10A770000B2F112707FD1A95E0924A09F0924B0919
:10A7800000934C0910934D098091520990915309FF
:10A79000A0915409B0915509B7FF04C081509F4F53
:10A7A000AF4FBF4F892F9A2FAB2FBB27A7FDBA956D
:10A7B000898B9A8BAB8BBC8B8093520990935309F6
:10A7C000A0935409B09355098091A107A82EBB24EA
:10A7D000CC24DD242091530430915404409155043D
:10A7E00050915604C601B5010E947E9197FF04C0A6
:10A7F00061507F4F8F4F9F4F672E782E892E99245F
:10A8000087FC9A9460925304709254048092550489
:10A810009092560420914F0430915004409151047D
:10A8200050915204C601B5010E947E9197FF04C069
:10A8300061507F4F8F4F9F4F272E382E492E552422
:10A8400047FC5A9420924F04309250044092510495
:10A850005092520480914B0490914C04A0914D046D
:10A86000B0914E04B7FF04C081509F4FAF4FBF4F10
:10A87000892F9A2FAB2FBB27A7FDBA9580934B0446
:10A8800090934C04A0934D04B0934E04D801C7019B
:10A8900086199709A809B9098093A0049093A10487
:10A8A000A093A204B093A3042091C807E22EFF2432
:10A8B00000271127BC01CD01A80197010E94F29148
:10A8C00059016A012093AE043093AF044093B00461
:10A8D0005093B10489899A89AB89BC8982199309FB
:10A8E000A409B5098093A4049093A504A093A60499
:10A8F000B093A704BC01CD01A80197010E94F29179
:10A900002093B2043093B3044093B4045093B5043D
:10A91000D601C501D7FE04C081509F4FAF4FBF4F36
:10A92000892F9A2FAB2FBB27A7FDBA959093F003E1
:10A930008093EF0357FF04C021503F4F4F4F5F4FAD
:10A94000BB2757FDBA95A52F942F832F9093F20321
:10A950008093F1038091D6039091D70381349105C0
:10A96000DCF48091D4039091D50381349105A4F453
:10A9700080918907E82FFF27EE0FFF1FE754F74F5D
:10A98000808191810190F081E02DF7FF03C0F09567
:10A99000E195FF4F7A97E4F08091020A8F3FC1F46E
:10A9A0008091EF039091F00397FD0196959587951F
:10A9B0009093F0038093EF038091F1039091F20361
:10A9C00097FD0196959587959093F2038093F103F7
:10A9D0008091410990914209A0914309B0914409A5
:10A9E000B7FF04C081509F4FAF4FBF4F892F9A2FA1
:10A9F000AB2FBB27A7FDBA958093410990934209DD
:10AA0000A0934309B093440980913209909133098E
:10AA1000A0913409B0913509B7FF04C081509F4F10
:10AA2000AF4FBF4F892F9A2FAB2FBB27A7FDBA95EA
:10AA30008093320990933309A0933409B093350978
:10AA40008091630490916404A0916504B0916604C0
:10AA50002F81388549855A85281B390B4A0B5B0B9A
:10AA6000209398043093990440939A0450939B0444
:10AA700080915B0490915C04A0915D04B0915E04B0
:10AA8000EB84FC840D851E85E81AF90A0A0B1B0B62
:10AA9000E0929C04F0929D0400939E0410939F0406
:10AAA0002093A0043093A1044093A2045093A304E4
:10AAB000E092A404F092A5040093A6041093A704C6
:10AAC00080913F0490914004A0914104B0914204D0
:10AAD000821B930BA40BB50B80933F04909340040F
:10AAE000A0934104B09342048091370490913804BC
:10AAF000A0913904B0913A048E199F09A00BB10BB3
:10AB00008093370490933804A0933904B0933A04A7
:10AB100088898823E1F020911D0430911E0421389A
:10AB200031054CF0809174049091750401969093D6
:10AB300075048093740420583F4F4CF48091740442
:10AB4000909175040197909375048093740410920A
:10AB50001E0410921D0481E090E09093BB0480934A
:10AB6000BA04E090A004F090A1040091A204109116
:10AB7000A304D801C70117FF07C088279927DC0164
:10AB80008E199F09A00BB10B81509240A040B0409C
:10AB900034F084E090E09093BB048093BA048091F9
:10ABA000C0049091C104A091C204B091C30420914B
:10ABB0004A0930914B0940914C0950914D09821B33
:10ABC000930BA40BB50B815E914BAF4FBF4F8F53CF
:10ABD0009C49A040B04028F08091030A89310CF4D0
:10ABE000FFC021E0E21620E1F20620E0020720E0AB
:10ABF00012070CF473C08091BC04882309F46AC066
:10AC0000D801C70117FF07C088279927DC018E19D3
:10AC10009F09A00BB10B9C01AD01B7FF04C02150EF
:10AC20003E4F4F4F5F4FF9E0559547953795279524
:10AC3000FA95D1F78091BA049091BB04820F931FCB
:10AC40009093BB048093BA04D801C70117FF03C0D7
:10AC50000796A11DB11DE3E0B595A795979587953A
:10AC6000EA95D1F78093AE049093AF04A093B0041B
:10AC7000B093B10489589341A040B04064F088E893
:10AC800093E1A0E0B0E08093AE049093AF04A09372
:10AC9000B004B093B1042091AE043091AF04409160
:10ACA000B0045091B10457FF04C021503F4F4F4FA3
:10ACB0005F4F232F342F452F552747FD5A958091FD
:10ACC000EF039091F003820F931F9093F003809312
:10ACD000EF0306C081E08093BC0402C01092BC0464
:10ACE00040E0E41640EFF4064FEF04074FEF14077F
:10ACF0000CF073C08091BD04882309F46AC0D801A8
:10AD0000C70117FF07C088279927DC018E199F0903
:10AD1000A00BB10B9C01AD01B7FF04C021503E4F09
:10AD20004F4F5F4F69E055954795379527956A9541
:10AD3000D1F78091BA049091BB04820F931F909336
:10AD4000BB048093BA04D801C70117FF03C007965C
:10AD5000A11DB11D23E0B595A795979587952A95D7
:10AD6000D1F78093AE049093AF04A093B004B09356
:10AD7000B10488579C4EAF4FBF4F64F488E79CEEF8
:10AD8000AFEFBFEF8093AE049093AF04A093B004F5
:10AD9000B093B1042091AE043091AF044091B0045F
:10ADA0005091B10457FF04C021503F4F4F4F5F4FA8
:10ADB000232F342F452F552747FD5A958091EF03B8
:10ADC0009091F003820F931F9093F0038093EF0311
:10ADD00011C081E08093BD040DC01092BD040AC073
:10ADE0001092BB041092BA0484E690E0909387011D
:10ADF000809386016889262F33278091BA04909129
:10AE0000BB042817390724F43093BB042093BA04F9
:10AE10001091030A112379F0212F332727FD309554
:10AE20008091BA049091BB042817390724F4309319
:10AE3000BB042093BA044091A0045091A1046091F6
:10AE4000A2047091A304413851056105710574F0A5
:10AE500080917804909179042091BA043091BB04D8
:10AE6000820F931F909379048093780440585F4F2A
:10AE70006F4F7F4F74F48091780490917904209102
:10AE8000BA043091BB04821B930B90937904809396
:10AE9000780481E090E09093BB048093BA04C09062
:10AEA000A404D090A504E090A604F090A704D701D4
:10AEB000C601F7FE07C088279927DC018C199D0978
:10AEC000AE09BF0981509240A040B04034F084E008
:10AED00090E09093BB048093BA048091C404909155
:10AEE000C504A091C604B091C704209152093091C5
:10AEF00053094091540950915509821B930BA40B9F
:10AF0000B50B815E914BAF4FBF4F8F539C49A04013
:10AF1000B04018F019310CF4FFC001E0C01600E198
:10AF2000D00600E0E00600E0F0060CF473C080916B
:10AF3000BE04882309F46AC0D701C601F7FE07C022
:10AF400088279927DC018C199D09AE09BF099C014E
:10AF5000AD01B7FF04C021503E4F4F4F5F4F09E096
:10AF600055954795379527950A95D1F78091BA045D
:10AF70009091BB04820F931F9093BB048093BA04FB
:10AF8000D701C601F7FE03C00796A11DB11D13E04E
:10AF9000B595A795979587951A95D1F78093B204A3
:10AFA0009093B304A093B404B093B504895893412B
:10AFB000A040B04064F088E893E1A0E0B0E0809366
:10AFC000B2049093B304A093B404B093B504209159
:10AFD000B2043091B3044091B4045091B50457FFCA
:10AFE00004C021503F4F4F4F5F4F232F342F452F29
:10AFF000552747FD5A958091F1039091F203820FF6
:10B00000931F9093F2038093F10306C081E0809335
:10B01000BE0402C01092BE0420E0C21620EFD20689
:10B020002FEFE2062FEFF2060CF073C08091BF0401
:10B03000882309F46AC0D701C601F7FE07C0882734
:10B040009927DC018C199D09AE09BF099C01AD014E
:10B05000B7FF04C021503E4F4F4F5F4FE9E0559579
:10B06000479537952795EA95D1F78091BA04909145
:10B07000BB04820F931F9093BB048093BA04D70143
:10B08000C601F7FE03C00796A11DB11D73E0B5957B
:10B09000A795979587957A95D1F78093B204909369
:10B0A000B304A093B404B093B50488579C4EAF4F3B
:10B0B000BF4F64F488E79CEEAFEFBFEF8093B2041C
:10B0C0009093B304A093B404B093B5042091B20458
:10B0D0003091B3044091B4045091B50457FF04C0BB
:10B0E00021503F4F4F4F5F4F232F342F452F552770
:10B0F00047FD5A958091F1039091F203820F931FBF
:10B100009093F2038093F10311C081E08093BF0418
:10B110000DC01092BF040AC01092BB041092BA0472
:10B1200084E690E090938701809386014889242FDC
:10B1300033278091BA049091BB042817390724F46F
:10B140003093BB042093BA048091030A882379F0DA
:10B15000282F332727FD30958091BA049091BB04A6
:10B160002817390724F43093BB042093BA04409184
:10B17000A4045091A5046091A6047091A7044138DD
:10B1800051056105710574F0809176049091770402
:10B190002091BA043091BB04820F931F90937704DF
:10B1A0008093760440585F4F6F4F7F4FCCF480916F
:10B1B0007604909177042091BA043091BB04821BED
:10B1C000930B90937704809376040AC01092F20355
:10B1D0001092F1031092F0031092EF0310921F04EB
:10B1E00080915809882341F41092F2031092F103E0
:10B1F0001092F0031092EF0380914A0990914B094D
:10B20000A0914C09B0914D098093C0049093C10462
:10B21000A093C204B093C304809152099091530942
:10B22000A0915409B09155098093C4049093C5042A
:10B23000A093C604B093C704109253041092540410
:10B24000109255041092560410924F04109250041C
:10B25000109251041092520410924B0410924C041C
:10B2600010924D0410924E0410924A0910924B090C
:10B2700010924C0910924D091092520910925309E4
:10B2800010925409109255091092410910924209E6
:10B290001092430910924409109232091092330916
:10B2A0001092340910923509109218031092170366
:10B2B000E0901504F0901604C701F7FE04C088273B
:10B2C00099278E199F0904973CF08091720984FD9B
:10B2D00003C082E38093F30310919E07A12EBB2449
:10B2E000CC24DD24B701882777FD8095982F97011E
:10B2F000F7FE04C0222733272E193F09442737FDC4
:10B300004095542F0E947E919B01AC01C601B5016E
:10B310000E947E9197FF04C061507E4F8F4F9F4FD8
:10B3200059E095958795779567955A95D1F79B0143
:10B33000812F99278E9DD0018F9DB00D9E9DB00DC0
:10B340001124CD01B7FD0396959587959595879521
:10B35000280F391F8091F5039091F603280F391FAC
:10B36000442737FD4095542F20939404309395043F
:10B370004093960450939704809133049091340441
:10B38000A0913504B0913604821B930BA40BB50B2E
:10B390008093330490933404A0933504B09336041F
:10B3A0008155934CA040B04064F080E593ECA0E060
:10B3B000B0E08093330490933404A0933504B093A9
:10B3C00036048091330490913404A0913504B091F7
:10B3D0003604805B9C43AF4FBF4F64F480EB9CE32B
:10B3E000AFEFBFEF8093330490933404A093350400
:10B3F000B093360400918A0110918B0117FDFCC0B7
:10B400008091720983FFF8C08091890181508093F7
:10B410008901882309F0F4C08DE08093890180912F
:10B42000630490916404A0916504B0916604B7FF31
:10B4300004C081509E4FAF4FBF4F39E0B595A795DF
:10B44000979587953A95D1F77C0197FF04C0F094C2
:10B45000E194F108F39480915B0490915C04A091D5
:10B460005D04B0915E04B7FF04C081509E4FAF4FA2
:10B47000BF4F29E0B595A795979587952A95D1F760
:10B480009C0197FF03C0309521953F4FE216F306CC
:10B490000CF47901B701F7FE02C0695F7F4F2B0101
:10B4A000A3E055944794AA95E1F722E030E0420EDC
:10B4B000531E609082097090830980908409909057
:10B4C000850920913C0130913D0140913E01509110
:10B4D0003F01C401B3010E94F29159016A01309306
:10B4E000300920932F09021B130BC801845E9D4F66
:10B4F00068E671E00E94BD919C01245B3040809120
:10B50000860190918701009731F001979093870110
:10B51000809386011BC049E1E416F104BCF48091DC
:10B520001D0490911E04820F931F90931E0480931C
:10B530001D048091F303882349F081508093F30325
:10B54000882321F4B0922204A092210480918601E4
:10B5500090918701892BF9F4809188019927289F80
:10B56000B001299F700D389F700D1124CB01B201DD
:10B570000E94BD91CB01AA2797FDA095BA2F680E16
:10B58000791E8A1E9B1E60928209709283098092A6
:10B590008409909285098091F303882369F580914D
:10B5A00021049091220420912F0930913009821BAF
:10B5B000930B845E9D4F68E671E00E94BD919C01F3
:10B5C000245B30408091720186959927289FD00195
:10B5D000299FB00D389FB00D11249D01B7FF02C007
:10B5E000215F3F4FF4E035952795FA95E1F73093C9
:10B5F000F6032093F50304C01092F6031092F503AE
:10B6000080911F04882381F010922704109228044F
:10B610001092290410922A0410922B0410922C04E8
:10B6200010922D0410922E04F090EC03FF20F1F400
:10B6300080915809282F3327442755278091630488
:10B6400090916404A0916504B0916604BC01CD01A1
:10B650000E947E91DC01CB01BC01CD0128EF3AE2D2
:10B6600040E050E00E94F291390102C06624772444
:10B67000E090EB03EE20F1F480915809282F332756
:10B680004427552780915B0490915C04A0915D0450
:10B69000B0915E04BC01CD010E947E91DC01CB0122
:10B6A000BC01CD0128EF3AE240E050E00E94F29167
:10B6B000290102C04424552480912C0990912D0920
:10B6C000893C91051CF088EC90E005C088539F4FA1
:10B6D00034F488E39FEF90932D0980932C09809197
:10B6E000380990913909893C91051CF088EC90E06B
:10B6F00005C088539F4F34F488E39FEF9093390936
:10B700008093380980913A0990913B09AA2797FDC7
:10B71000A095BA2F20918009A22EBB24CC24DD2431
:10B72000BC01CD01A60195010E947E919B01AC0157
:10B7300080912C0990912D09AA2797FDA095BA2FE9
:10B74000E7E0880F991FAA1FBB1FEA95D1F7280FC2
:10B75000391F4A1F5B1F57FF04C0215C3F4F4F4FEB
:10B760005F4F76E055954795379527957A95D1F7B0
:10B770008301020F131F10933B0900933A09809134
:10B780002A0990912B09AA2797FDA095BA2FBC01F1
:10B79000CD01A60195010E947E919B01AC01809193
:10B7A000380990913909AA2797FDA095BA2F67E02B
:10B7B000880F991FAA1FBB1F6A95D1F7280F391F41
:10B7C0004A1F5B1F57FF04C0215C3F4F4F4F5F4F25
:10B7D000F6E05595479537952795FA95D1F74201AB
:10B7E000820E931E90922B0980922A0980917B09E8
:10B7F00090917C09880F991FAA2797FDA095BA2FD1
:10B8000020913109332744275527BC01CD010E94DF
:10B810007E915B016C0197FF08C02FE330E040E0B0
:10B8200050E0A20EB31EC41ED51EE6E0D594C79408
:10B83000B794A794EA95D1F780914709282F332729
:10B84000442755278091470490914804A0914904CA
:10B85000B0914A04BC01CD010E947E91DC01CB0174
:10B86000BC01CD0120EF35E540E050E00E94F291AF
:10B87000B501620F731F70937C0960937B090150BF
:10B88000104134F080E090E190933B0980933A09B5
:10B8900080913A0990913B098050904F34F480E0B8
:10B8A00090EF90933B0980933A0951E0851650E15F
:10B8B000950634F080E090E190932B0980932A095B
:10B8C00080912A0990912B098050904F34F480E0A8
:10B8D00090EF90932B0980932A096150704134F0C6
:10B8E00080E090E190937C0980937B0980917B09B3
:10B8F00090917C098050904F34F480E090EF9093C9
:10B900007C0980937B0980910001482F5527809105
:10B910001F01909120014817590794F420911F01AD
:10B920003091200109811A81049FC001059F900D6B
:10B93000149F900D1124B9010E94A9917A83698303
:10B9400029813A81220F331F220F331F3A83298323
:10B950004091720940FD02C00C94B664EE2011F0D3
:10B960000C94B664FF2011F00C94B66400E010E073
:10B9700048018091ED039091EE0390930D07809321
:10B980000C0720917A0430917B042115310509F0D0
:10B990003FC080911501909116018959934058F04C
:10B9A00087B5803F20F480911B03815011C081E056
:10B9B0008093D1044EC08091150190911601843678
:10B9C000910508F587B58031D0F080911B038F5F1A
:10B9D00080931B039FE0890290011124809131071D
:10B9E000821B87BD8CE291E090930B0380930A0346
:10B9F0008EE591E090937B0480937A042AC081E0E5
:10BA00008093D00426C0F092D004F092D10421C0DB
:10BA10008091030490910404A0910504B091060460
:10BA200064E0880F991FAA1FBB1F6A95D1F7809306
:10BA30001C0390931D03A0931E03B0931F03109348
:10BA40001A03009319032150304030937B04209354
:10BA50007A042091750141FF3CC0223348F5809162
:10BA60008C01815080938C018F3F09F052C08091EE
:10BA70009F01882339F480912004882319F088E2FB
:10BA800080939F01109220048091030490910404FC
:10BA9000A0910504B09106048093FF0390930004E5
:10BAA000A0930104B093020481E080938C0131C023
:10BAB000273478F180919F01882339F48091200404
:10BAC000882319F487E280939F0188EC80938C018E
:10BAD0001DC08091400190914101820F911D2091E4
:10BAE00097073327829FA001839F500D929F500D8F
:10BAF0001124CA01AA2797FDA095BA2F8093FF03AE
:10BB000090930004A0930104B093020481E0809319
:10BB100020048091630490916404A0916504B09125
:10BB20006604E0903C01F0903D0100913E011091CF
:10BB30003F01BC01CD01A80197010E94F29159017A
:10BB40006A0180915B0490915C04A0915D04B091C6
:10BB50005E04BC01CD01A80197010E94F291B901D8
:10BB6000C5010E942C845C01CC971CF05CE3A52EDF
:10BB7000B12CC5010E942A725C0180E280933B01D6
:10BB80001092FE031092FD0380912004882309F493
:10BB90005FC58091D10399279C012071307084FD8D
:10BBA00057C58091D00382608093D003709156096D
:10BBB000872F992741E0C42ED12CC822D92280FD9D
:10BBC00004C08091720981FD10C0C980DA80309371
:10BBD000C9042093C8043093FE032093FD03809191
:10BBE000D103806C8093D103ABC28091D10381FFDC
:10BBF0007AC200917C0110917D01C8010F962090BE
:10BC0000130430901404821593050CF058C08091F1
:10BC1000D004882309F053C08091D10387FF15C059
:10BC20008091D1038F778093D10380910304909109
:10BC30000404A0910504B09106048093FF0390933F
:10BC40000004A0930104B09302048091D1038064A6
:10BC50008093D103E0903609EE20F1F08091FF034C
:10BC600090910004A0910104B0910204BC01CD01A7
:10BC700024E630E040E050E00E94F2918E2D9927BA
:10BC8000AA27BB2782179307A407B5072CF4D092E5
:10BC9000FE03C092FD0310C0C101801B910B0F97E2
:10BCA00097FF03C0909581959F4F9093FE038093DB
:10BCB000FD038BE280933B011092F70316C1C8018C
:10BCC0000F9728163906C4F52091D1042223A1F537
:10BCD0008091D10386FF15C08091D1038F7B809323
:10BCE000D1038091030490910404A0910504B091C4
:10BCF00006048093FF0390930004A0930104B09383
:10BD000002048091D10380688093D103C101801B1C
:10BD1000910B0F9697FF03C0909581959F4F90953B
:10BD200081959F4F9093FE038093FD038DE2809356
:10BD30003B012093F703D9C08DE380933B016091D1
:10BD4000F803662371F12091F9033091FA034091D1
:10BD5000FB035091FC038091FF0390910004A0919C
:10BD60000104B091020482179307A407B507CCF42D
:10BD70008091D10380648093D103862F992790937B
:10BD8000FE038093FD038AE08093F7038EE58093A2
:10BD90003B018091D10387FFA8C08091D1038F77A9
:10BDA00033C0662309F443C02091F9033091FA03AC
:10BDB0004091FB035091FC038091FF03909100049C
:10BDC000A0910104B0910204281739074A075B07C4
:10BDD00074F58091D10380688093D103862F9927D1
:10BDE000909581959F4F9093FE038093FD0386EF7E
:10BDF0008093F70386E780933B018091D10386FF10
:10BE000074C08091D1038F7B8093D1038091030410
:10BE100090910404A0910504B09106048093FF035F
:10BE200090930004A0930104B09302045EC080913B
:10BE3000D103807C09F459C08091F703882379F5F8
:10BE4000E0900304F09004040091050410910604AE
:10BE5000D801C70180589040A040B0402091FF0316
:10BE6000309100044091010450910204821793071D
:10BE7000A407B5075CF4D801C70180589F4FAF4FA6
:10BE8000BF4F281739074A075B075CF08093FF0311
:10BE900090930004A0930104B093020402C0109296
:10BEA000F7038091D1038F738093D1031092C9045B
:10BEB0001092C80471FF06C084EF91E090930B03C9
:10BEC00080930A0380910704882379F48091030406
:10BED00090910404A0910504B0910604C397A105B4
:10BEE000B1051CF081E0809307046091C804709153
:10BEF000C9048091FD039091FE03680F791F709330
:10BF0000C9046093C804CB0177FF04C08827992730
:10BF1000861B970B855F91400CF4CEC04091F703D0
:10BF2000442389F18091F9039091FA032091FF0352
:10BF300030910004821B930B0996439748F480913B
:10BF4000F9039091FA03A091FB03B091FC0312C096
:10BF5000242F332727FD3095432F532F8091FF0344
:10BF600090910004A0910104B0910204820F931FEC
:10BF7000A41FB51F8093FF0390930004A0930104B6
:10BF8000B093020424C0809197072091FF03309161
:10BF9000000440910104509102041616170644F45F
:10BFA00063E00E949D91280F311D411D511D07C066
:10BFB00063E00E949D91281B31094109510920939A
:10BFC000FF03309300044093010450930204109245
:10BFD000C9041092C804E0900304F0900404009196
:10BFE000050410910604D801C70180509440A04078
:10BFF000B0402091FF033091000440910104509122
:10C00000020482179307A407B5075CF4D801C7019F
:10C0100080509C4FAF4FBF4F281739074A075B0727
:10C0200044F08093FF0390930004A0930104B09325
:10C0300002048091560981FF06C084E690E0909347
:10C040000B0380930A0380919B078823A9F58091B5
:10C05000F803882389F54091ED035091EE0357FFD3
:10C0600002C04D5F5F4F5595479555954795809117
:10C070001F0190912001209100013327489FF0017A
:10C08000499FF00D589FF00D1124CF01B9010E9476
:10C09000BD9170937D0160937C01663471051CF441
:10C0A00086E490E005C06739710534F086E990E0D8
:10C0B00090937D0180937C0180917A0490917B0420
:10C0C000892BD1F18091030490910404A09105047F
:10C0D000B09106048093FF0390930004A0930104A1
:10C0E000B093020429C08091030490910404A091AC
:10C0F0000504B091060480599140A040B04080935F
:10C10000FF0390930004A0930104B0930204809174
:10C110009B07882311F0992702C088E790E090934D
:10C120007D0180937C01E980FA80F092EE03E09239
:10C13000ED038EE280933B01C090ED03D090EE03BF
:10C14000E0900304F09004040091050410910604AB
:10C150002091FF03309100044091010450910204AA
:10C160002E153F054007510724F08091560980FDA8
:10C17000BBC280917A0490917B04892B39F0C090E6
:10C18000ED03D090EE0300E010E0D7C0D801C70166
:10C19000821B930BA40BB50B809398049093990486
:10C1A000A0939A04B0939B04823000E890070FEFAD
:10C1B000A0070FEFB0072CF481E090E8AFEFBFEFDE
:10C1C00009C08F5F9F47A040B04064F08FEF9FE7AA
:10C1D000A0E0B0E08093980490939904A0939A040F
:10C1E000B0939B040091980410919904809174017C
:10C1F000282F33274427552780919804909199043C
:10C20000A0919A04B0919B04BC01CD010E947E9143
:10C2100097FF04C0615E7F4F8F4F9F4F25E095953C
:10C220008795779567952A95D1F7609398047093D1
:10C23000990480939A0490939B0465302EEF7207C3
:10C240002FEF82072FEF92072CF484E09EEFAFEFE1
:10C25000BFEF09C0605074408040904064F080E0BF
:10C2600094E0A0E0B0E08093980490939904A093A8
:10C270009A04B0939B048090980490909904209124
:10C28000190330911A0337FF02C0295F3F4F83E043
:10C29000359527958A95E1F74FEF223834071CF43E
:10C2A00021E83FEF05C02038310514F020E830E0E8
:10C2B000C901AA2797FDA095BA2F209176013327AF
:10C2C00044275527BC01CD010E947E9197FF04C0F1
:10C2D0006D5F7F4F8F4F9F4FB2E095958795779514
:10C2E0006795BA95D1F79B015FEF613075071CF434
:10C2F00020E03FEF06C06F3F710519F014F020E019
:10C3000031E08091D103807C49F0C90137FD03966B
:10C310009C0135952795359527950DC08091560937
:10C3200080FF09C0C90137FD07969C01F3E03595F0
:10C330002795FA95E1F7820E931E2091730122232F
:10C3400009F454C060912304709124048091250461
:10C350009091260497FF04C061587F4F8F4F9F4FE5
:10C36000E7E09595879577956795EA95D1F7332717
:10C37000442755270E947E9197FF04C0615E7F4F3E
:10C380008F4F9F4F55E095958795779567955A956F
:10C39000D1F7609398047093990480939A049093D2
:10C3A0009B046138AFEF7A07AFEF8A07AFEF9A07C8
:10C3B0002CF480E89FEFAFEFBFEF0AC06F3F71052D
:10C3C0008105910569F064F080E091E0A0E0B0E0C3
:10C3D0008093980490939904A0939A04B0939B043B
:10C3E0008091980490919904880E991E8091710112
:10C3F000282F33278091060A992787FD9095289F3B
:10C40000F001299FF00D389FF00D11249F01F7FFD7
:10C4100002C021583F4F220F232F221F330BFFEF63
:10C4200021383F071CF420E83FEF06C02F3F3105BD
:10C4300019F014F020E031E0820E931EC401AA2707
:10C4400097FDA095BA2FE090ED03F090EE039701D1
:10C45000442737FD4095542FBC01CD010E947E91A9
:10C4600097FF04C061507E4F8F4F9F4F29E09595F5
:10C470008795779567952A95D1F7C61AD70A80913F
:10C48000FD039091FE03892B09F060C01E141F0468
:10C490000CF05CC0980117FF03C0309521953F4F09
:10C4A0002D33310540F480911B0490911C048C15B0
:10C4B0009D0574F526C02C53304085E036952795B0
:10C4C0008A95E1F72031310510F02FE030E04091FE
:10C4D0001B0450911C0410161106E4F480E190E056
:10C4E000821B930B489F9001499F300D589F300D40
:10C4F0001124B4E036952795BA95E1F72C153D0542
:10C5000020F580917A0190917B01C816D906F4F04C
:10C510006C011CC0205F3F4F80917A0190917B019C
:10C52000829F8001839F100D929F100D112498010E
:10C53000A4E036952795AA95E1F74C155D0514F012
:10C540006A0104C0C216D30608F06901C601AA2711
:10C5500097FDA095BA2FFDE0880F991FAA1FBB1F5A
:10C56000FA95D1F79501442737FD4095542FBC012A
:10C57000CD010E94F29120939C0430939D0440933E
:10C580009E0450939F04C0909C04D0909D04809181
:10C59000CA049091CB049C01220F331F280F391F2E
:10C5A0002C0D3D1D37FF02C02D5F3F4FA901559552
:10C5B0004795559547955093CB044093CA04809175
:10C5C0009307282F3327220F331F220F331F2417DF
:10C5D00035076CF480917A09282F3327220F331FF7
:10C5E000220F331F205530404217530724F0309359
:10C5F000CB042093CA048091560980FF14C0809117
:10C60000CA049091CB0429813A818217930724F0C0
:10C610003093CB042093CA044091CA045091CB04B8
:10C620005A83498361C029813A812E193F0937FF16
:10C6300002C02D5F3F4F3595279535952795609121
:10C64000CA047091CB04620F731F7A8369834CC054
:10C6500080919B07882301F56091ED037091EE03B3
:10C6600077FF02C06D5F7F4F7595679575956795EC
:10C6700040911F015091200180910001282F332704
:10C68000649FC001659F900D749F900D1124B901A6
:10C690000E94BD91CB0101C0992790937D018093A9
:10C6A0007C0180917C0190917D01873491051CF47F
:10C6B00086E490E005C08639910534F086E990E083
:10C6C00090937D0180937C0189819A819093CB0422
:10C6D0008093CA048091D103806C8093D1038091B0
:10C6E000D0038D7F8093D0038091D10399279C0143
:10C6F0002270307081FF2BC18091CC049091CD04C9
:10C70000A091CE04B091CF040097A105B10521F00E
:10C71000809107048130B1F4E981FA81CF01AA2721
:10C7200097FDA095BA2F1EE0880F991FAA1FBB1F67
:10C730001A95D1F78093CC049093CD04A093CE04A6
:10C74000B093CF0480910704813019F482E0809384
:10C750000704E980FA80C701AA2797FDA095BA2FA0
:10C760009501442737FD4095542FBC01CD010E940F
:10C770007E91DC01CB0180939C0490939D04A09357
:10C780009E04B0939F04B7FF04C08150904EAF4FFA
:10C79000BF4F7C018D01ADE015950795F794E794A7
:10C7A000AA95D1F7E0929C04F0929D0400939E0418
:10C7B00010939F046091D2037091D3032FE0603AED
:10C7C000720750F58091CC049091CD04A091CE04D5
:10C7D000B091CF049C01AD01FAE05695479537958D
:10C7E0002795FA95D1F7821B930BA40BB50BA801E3
:10C7F0009701E4E0220F331F441F551FEA95D1F73C
:10C80000820F931FA41FB51F8093CC049093CD0477
:10C81000A093CE04B093CF0460547F4118F580916B
:10C82000CC049091CD04A091CE04B091CF049C0192
:10C83000AD016CE056954795379527956A95D1F7E8
:10C84000821B930BA40BB50BA8019701F2E0220FFA
:10C85000331F441F551FFA95D1F7820F931FA41F52
:10C86000B51F38C08091190390911A038091190364
:10C8700090911A0397FF03C0909581959F4F84363E
:10C88000910584F580910304909104042091FF03A5
:10C8900030910004821B930B81509F4F8F5F91401A
:10C8A00008F58091CC049091CD04A091CE04B09174
:10C8B000CF049C01AD01EEE056954795379527953D
:10C8C000EA95D1F7821B930BA40BB50B8E0D9F1D20
:10C8D000A01FB11F8093CC049093CD04A093CE04ED
:10C8E000B093CF048091CC049091CD04A091CE045C
:10C8F000B091CF047EE0B695A795979587957A95E8
:10C90000D1F79093EE038093ED0340919907442370
:10C9100099F055279C01BA010E94BD91C901861B5F
:10C92000970B90931C0480931B04260F371F3093A2
:10C930007B0120937A011FC010921C0410921B04EB
:10C940008FEF93E090937B0180937A0114C0109253
:10C9500007041092CC041092CD041092CE041092D1
:10C96000CF043093EE032093ED0305C08091D103F3
:10C97000806C8093D1038091E00481FF37C089816E
:10C980009A8197FD03969595879595958795209122
:10C99000CE033091CF032817390760F48091ED035F
:10C9A0009091EE03892B31F0220F331F220F331F9A
:10C9B0003A8329838091030490910404A091050493
:10C9C000B09106048093FF0390930004A0930104A8
:10C9D000B093020488E99AE390930B0380930A03CF
:10C9E00080E09EE090930A018093090120913F0925
:10C9F000822F9927880F991F880F991F8896698120
:10CA00007A818617970714F09A83898370917A093F
:10CA10007D8B872F9927880F991F880F991F805525
:10CA20009040A981BA818A179B0714F49A8389835D
:10CA300080915003882341F48091180A8F3F21F49C
:10CA40008091E4048823E9F08091D2039091D3038C
:10CA50000297C097B0F4E981FA811E161F068CF484
:10CA600081E090E09093D3038093D203E22EFF24E1
:10CA7000EE0CFF1CEE0CFF1C8701085D1F4F1A8394
:10CA8000098329813A813093F1062093F006809141
:10CA9000940490919504A0919604B091970412E0AB
:10CAA000880F991FAA1FBB1F1A95D1F700917B0908
:10CAB00010917C09081B190B213A31058CF0C90132
:10CAC00037FD019695958795801791070CF48C0199
:10CAD000909581959F4F081719076CF48C010BC036
:10CAE0000135110514F000E510E03FEF003B13079E
:10CAF00014F400EB1FEF4D89242F3327220F331F2F
:10CB0000220F331FC90169817A81861B970B801719
:10CB100091070CF48C0189819A81821B930B081771
:10CB200019070CF48C0180913A0990913B096091AE
:10CB3000190470911A04861B970B909349098093EE
:10CB40004809D090580920912B0430912C04409131
:10CB50002D0450912E04DD2041F0661A770AC3019E
:10CB6000AA2797FDA095BA2F04C0AA2797FDA095E4
:10CB7000BA2F280F391F4A1F5B1F20932B043093B5
:10CB80002C0440932D0450932E0480912B049091FB
:10CB90002C04A0912D04B0912E0481509A4FA040F6
:10CBA000B04064F080E09AEFA0E0B0E080932B0406
:10CBB00090932C04A0932D04B0932E0480912B0409
:10CBC00090912C04A0912D04B0912E048050964099
:10CBD000AF4FBF4F64F480E096E0AFEFBFEF8093BC
:10CBE0002B0490932C04A0932D04B0932E04C0909A
:10CBF000A807209148093091490978E0E72EEC1404
:10CC000098F08C2D9927829FA001839F500D929FB1
:10CC1000500D1124CA0157FD07967C0163E0F5947D
:10CC2000E7946A95E1F712C08C2D86959927829F2B
:10CC3000B001839F700D929F700D1124CB0177FD81
:10CC400003967C01F594E794F594E794A09077011E
:10CC5000B09078019501442737FD4095542F80917D
:10CC60002B0490912C04A0912D04B0912E04BC01B2
:10CC7000CD010E94F291E20EF31E90906101692DA8
:10CC8000772788279927980117FF04C02227332781
:10CC9000201B310B37FF02C02F5F3F4F3595279583
:10CCA000A981BA812A0F3B1F442737FD4095542F95
:10CCB0000E947E9197FF04C0615C7F4F8F4F9F4F12
:10CCC00026E095958795779567952A95D1F79B01ED
:10CCD0006E157F050CF47B01309521953F4FE216D0
:10CCE000F3060CF4790180912A0990912B09609147
:10CCF000170470911804861B970B90932909809351
:10CD0000280920912704309128044091290450914A
:10CD10002A04DD2041F0461A570AC201AA2797FDCE
:10CD2000A095BA2F04C0AA2797FDA095BA2F280F67
:10CD3000391F4A1F5B1F2093270430932804409318
:10CD4000290450932A048091270490912804A091EB
:10CD50002904B0912A0481509A4FA040B04064F059
:10CD600080E09AEFA0E0B0E080932704909328043D
:10CD7000A0932904B0932A04809127049091280459
:10CD8000A0912904B0912A0480509640AF4FBF4F24
:10CD900064F480E096E0AFEFBFEF809327049093B8
:10CDA0002804A0932904B0932A04209128093091E3
:10CDB000290948E04C1598F08C2D9927829FB001E5
:10CDC000839F700D929F700D1124CB0177FD079604
:10CDD0006C01B3E0D594C794BA95E1F712C0C6943C
:10CDE0008C2D9927829FD001839FB00D929FB00D0B
:10CDF0001124CD01B7FD03966C01D594C794D59449
:10CE0000C7949501442737FD4095542F80912704FE
:10CE100090912804A0912904B0912A04BC01CD016D
:10CE20000E94F291C20ED31E692D77278827992779
:10CE3000980117FF04C022273327201B310B37FF2F
:10CE400002C02F5F3F4F35952795E981FA812E0F5C
:10CE50003F1F442737FD4095542F0E947E9197FF36
:10CE600004C0615C7F4F8F4F9F4FE6E0959587959B
:10CE700077956795EA95D1F79B016C157D050CF4C4
:10CE80006B01309521953F4FC216D3060CF4690112
:10CE900080913F09282E33245090EA0768E5862EBA
:10CEA00068E0962E5FE0A52E58E0B52E4BE0442EAC
:10CEB00039E5632E39E0732ED5012C9112160CF052
:10CEC00029C1203429F4E981FA81FF8BEE8B1FC040
:10CED00049815A81CA01AA2797FDA095BA2F332705
:10CEE00027FD3095432F532FBC01CD010E947E9129
:10CEF00097FF04C0615C7F4F8F4F9F4F26E0959551
:10CF00008795779567952A95D1F77F8B6E8BF5017D
:10CF10002181203439F42E893F892E0D3F1D3F8B0E
:10CF20002E8B2AC0203C39F44E895F894E195F0947
:10CF30005F8B4E8B21C0C701AA2797FDA095BA2F02
:10CF4000332727FD3095432F532FBC01CD010E947D
:10CF50007E9197FF04C0615C7F4F8F4F9F4FB6E07B
:10CF60009595879577956795BA95D1F7AE89BF89DD
:10CF7000A60FB71FBF8BAE8BF5012281203439F489
:10CF80002E893F892C0D3D1D3F8B2E8B2AC0203CC6
:10CF900039F44E895F894C195D095F8B4E8B21C036
:10CFA000C601AA2797FDA095BA2F332727FD3095F4
:10CFB000432F532FBC01CD010E947E9197FF04C0E7
:10CFC000615C7F4F8F4F9F4FA6E095958795779532
:10CFD0006795AA95D1F7AE89BF89A60FB71FBF8BFA
:10CFE000AE8BF5012381203439F42E893F89200F3F
:10CFF000311F3F8B2E8B2AC0203C39F44E895F892C
:10D00000401B510B5F8B4E8B21C0C801AA2797FD97
:10D01000A095BA2F332727FD3095432F532FBC01FE
:10D02000CD010E947E9197FF04C0615C7F4F8F4FBE
:10D030009F4FF6E09595879577956795FA95D1F787
:10D04000AE89BF89A60FB71FBF8BAE8BF30180815E
:10D0500091812E893F898217930764F4B901680F83
:10D06000791F77FF02C06F5F7F4F759567957F8B44
:10D070006E8B1DC0552049F44E895F89440F551FA2
:10D08000481B590B5F8B4E8B12C051E0551578F43D
:10D09000252D33276E897F89861B970BB9010E9446
:10D0A000BD91AE89BF89A60FB71FBF8BAE8BC101E3
:10D0B000880F991F880F991FEE89FF898E179F0788
:10D0C00064F4FD898F2F9927880F991F880F991F66
:10D0D0002E893F892817390714F09F8B8E8B8E89F4
:10D0E0009F8997FD03969595879595958795F4016A
:10D0F0008183880F991F880F991F2E893F89281BCC
:10D10000390BC901880F8283EE89FF89D301ED9322
:10D11000FC9303C0F401118212824A9422E030E0B1
:10D12000620E731E44E050E0A40EB51E68E070E08D
:10D13000860E971E47FEC0CEE2E1C95E0C9429928E
:10D1400084B1806A84B93D9A82E58CBD1DBC459A44
:10D1500081E080938C098AEA80939D0983E880931B
:10D160009E098AE080939F091092A1091092A0095C
:10D170001092A3091092A2091092050A1092C109F7
:10D18000089530918C09332309F085C00DB407FE52
:10D1900082C084E080930903459A2EB58091E7040C
:10D1A00099278130910589F0823091051CF4892BF3
:10D1B00021F03EC00297B9F03BC03093C0092093E4
:10D1C000E8042138A9F581E008C0253549F48091AB
:10D1D000E804820F8093E80482E08093E70428C08B
:10D1E0003093E70425C08091C009E82FFF27EE5156
:10D1F000F64F20838F5F8093C0099091E8048032BE
:10D20000A0F0291769F480E2A2EEB9E0E2ECF9E0BF
:10D210000D9001928A95E1F781E08093C10902C0E7
:10D220003093C1091092E70403C0920F9093E80471
:10D2300020919C09223208F028C045980000000087
:10D2400000000000000000000000000000000000DE
:10D2500000000000000000000000000000000000CE
:10D26000000000000000000000000000E0919509AF
:10D27000F0919609E20FF11D80818EBD8091BE096B
:10D280009081890F8093BE0903C081E080938C094F
:10D290002F5F20939C090895EF92FF920F931F93A5
:10D2A0008091A1079927880F991F880F991F7C01EA
:10D2B0000027F7FC0095102F80916304909164047F
:10D2C000A0916504B0916604BC01CD01A80197014D
:10D2D0000E94F2913093A1092093A00980915B04F0
:10D2E00090915C04A0915D04B0915E04BC01CD01FD
:10D2F000A80197010E94F2913093A3092093A209FB
:10D3000020918209309183094091840950918509C7
:10D31000DA01C90163E0880F991FAA1FBB1F6A9534
:10D32000D1F7820F931FA41FB51F820F931FA41F55
:10D33000B51F20913C0130913D0140913E0150913B
:10D340003F01BC01CD010E94F2913093A9092093C5
:10D35000A80980917404909175042091260330915E
:10D360002703821B930B9093AF098093AE09E09142
:10D370006A04F0916B0480914F0990915009BF01AC
:10D380000E94BD919B01220F331F220F331F260FD6
:10D39000371F260F371F37FF02C02D5F3F4F3595D0
:10D3A0002795359527953093A5092093A409809159
:10D3B0007E0990917F09BF010E94BD919B01220FC0
:10D3C000331F220F331F260F371F260F371F37FF3C
:10D3D00002C02D5F3F4F35952795359527953093A2
:10D3E000A7092093A60910926B0410926A04109268
:10D3F000500910924F0910927F0910927E09809176
:10D400009F099927AA27BB27FC013A97E830F10525
:10D4100008F0FEC1E058FF4F0C9444928091E6035F
:10D420008093B2098091E5038093B3098091E4036E
:10D430008093B4098091E3038093B5098091E2035E
:10D440008093B6098091E1038093B7098091E0034E
:10D450008093B8098091DF038093B9098091D1034B
:10D460008093BA098091D103837F8093D1030E9476
:10D4700063308093BB098091EB078093BC09809156
:10D48000D003C4C18091120A9091130A9093B309FA
:10D490008093B2098091160A9091170A9093B5096A
:10D4A0008093B40980911F01909120018093B60967
:10D4B000809100018093B70980913B018093B80966
:10D4C0009091E9049093B909E92FFF27A3E0EE0FAB
:10D4D000FF1FAA95E1F7E85AF74F86818093BA09B2
:10D4E00083818093BB0987818093BC098581809368
:10D4F000BD09892F8F5F6CE00E949D919093E90494
:10D5000087C18091D6078093B2098091D707809315
:10D51000B3098091D8078093B4098091D90780938B
:10D52000B5098091DA078093B6098091DE07809370
:10D53000B7098091DF078093B8098091E007809355
:10D54000B9098091E3078093BA098091E10780933C
:10D55000BB098091E2078093BC098091E40756C122
:10D560008091D5078093B2098091AC07863081F015
:10D570008091D602823451F00E946C73E82FFF270D
:10D58000EB55FF4E84918093D60202C00E946C73CB
:10D5900080910C058093B3093BC1F8948091880772
:10D5A000E82FFF27EE0FFF1FE754F74F0190F081A0
:10D5B000E02DE038F1051CF0EFE7F0E006C02FEFBA
:10D5C000E138F20714F4E1E8FFEFE093B20980914B
:10D5D0008907E82FFF27EE0FFF1FE754F74F019051
:10D5E000F081E02DE038F1051CF0EFE7F0E006C037
:10D5F0007FEFE138F70714F4E1E8FFEFE093B309B8
:10D6000080918707E82FFF27EE0FFF1FE754F74FA2
:10D610000190F081E02DE038F1051CF0EFE7F0E03B
:10D6200006C08FEFE138F80714F4E1E8FFEFE0936C
:10D63000B40980918607E82FFF27EE0FFF1FE754FC
:10D64000F74F0190F081E02DE038F1051CF0EFE795
:10D65000F0E006C02FEFE138F20714F4E1E8FFEF45
:10D660007894E093B50980910A048093B60980917B
:10D670000B048093B70980910C048093B8098091C2
:10D680000D048093B90980910E048093BA098091AA
:10D690000F048093BB09809110048093BC09809192
:10D6A0001104B4C080917105863018F01092710594
:10D6B00085E08093B2098091E5078093B30980915A
:10D6C000030490910404A0910504B0910604BC01E8
:10D6D000CD0125E030E040E050E00E94F29130932F
:10D6E000B5092093B4098091FF0390910004A091A3
:10D6F0000104B0910204BC01CD0125E030E040E01E
:10D7000050E00E94F2913093B7092093B6098091BE
:10D71000DB078093B8098091DC078093B909809179
:10D72000DD078093BA09809109048093BB09809139
:10D73000B9089091BA088093BC098091F006909145
:10D74000F10697FD039695958795959587955EC00B
:10D750001092B2098AE58093B30984E08093B409FA
:10D7600084E38093B509809101018093B60980918B
:10D7700056058093B709909157059093B8098F7714
:10D78000809356059071909357058091580580932A
:10D79000B909809172098093BA09809156098093E2
:10D7A000BB098091E7078093BC098091F4072EC0E4
:10D7B0008091BA078093B2098091F2078093B309F0
:10D7C000809169018093B4098091B3078093B50972
:10D7D0008091B4078093B6098091B5078093B7090B
:10D7E000809168018093B8098091B7078093B90947
:10D7F0008091B8078093BA098091B9078093BB09DB
:10D800008091180A8093BC0980911A078093BD0902
:10D810008091C109882309F47DC16091C20980917A
:10D820009B01681719F08AEF8093990160939B011F
:10D8300081E0809389014091C3095091C409CA01D4
:10D8400081509E4F8F5F9340B0F42091C509309175
:10D85000C609C90181509E4F8F5F934060F480914B
:10D86000920785FF08C05093D6044093D5043093A7
:10D87000D4042093D3048091C9099091CA0921E06E
:10D880008936920724F490938B0180938A0120912A
:10D89000D3093091D40980910A0390910B03821728
:10D8A000930740F48091DE02882321F430930B0328
:10D8B00020930A03862F99278936910509F4A5C07C
:10D8C0008A36910544F48736910571F088369105C2
:10D8D00009F462C027C18A36910509F414C18B3658
:10D8E000910509F4E2C01EC18091D5098093020A16
:10D8F0008091D6098093040A8091D7098093030A06
:10D900008091D809809388018091D9098093060A73
:10D910008091DA0980939A018091DB098093E60473
:10D920008091DC098093D2048091DE038823F9F092
:10D930002091DD093091DE0937FD19C030932204B2
:10D94000209321049091BC07992389F08FE0989F40
:10D95000C0011124281B390BC90188599E4F68E664
:10D9600071E00E94BD919093220480932104209144
:10D97000DD043091DE048091DF099091E009280FE9
:10D98000391F37FF02C02F5F3F4F359527953093E2
:10D99000DE042093DD04C6C08091D50980939709E9
:10D9A0008091D609809398098091D709809399092D
:10D9B0008091D80980939A098091D90980939B0915
:10D9C0008091E0069091DA09892B8093E00690918E
:10D9D000E10693708091DB098C70982B9093E1069F
:10D9E0008091DC098093E4048091DD0980938D01AE
:10D9F0008091DE098093050A8091DF098093E0041D
:10DA00008091E0098093DF048DC08091D5098093D7
:10DA10008D098091D60980938E098091D7098093D2
:10DA20008F098091D809809390098091D9099091AC
:10DA3000DA0990939209809391098091DB09909182
:10DA4000DC0990939409809393098091DD099927CB
:10DA500087FD90959093EC088093EB088091DE0908
:10DA60008093F8038091DF099091E0099C0144279D
:10DA700037FD4095542FDA01C90163E0880F991FE3
:10DA8000AA1FBB1F6A95D1F7820F931FA41FB51F52
:10DA9000820F931FA41FB51F8093F9039093FA037D
:10DAA000A093FB03B093FC033DC08091D509809304
:10DAB000E3048091D6098093E2048091D709809392
:10DAC000E1049091D809992349F080919F0188231E
:10DAD00019F08151833010F490939F018091D909FE
:10DAE000809311058091DA09809310058091DB09FC
:10DAF0009091DC0990930E0580930D058091DD09CE
:10DB000080930F050FC08091AC07863059F40E94B6
:10DB1000C57308C01092D6041092D5041092D40494
:10DB20001092D3041F910F91FF90EF900895809170
:10DB30008C09882309F43BC045988DE999E09093BE
:10DB40009609809395099091E504E92FFF27E25704
:10DB5000FE4F9F5F9093E504808180939F099B30E7
:10DB600010F01092E50410928C090E944C6981E03B
:10DB700080939C09000000000000000000000000ED
:10DB80000000000000000000000000000000000095
:10DB90000000000000000000000000000000000085
:10DBA0000000000080919D098093BE098EBD0895FC
:10DBB00087B18C6087B9429843981092EB0480E853
:10DBC00080939D011092EA0480939C0108958091B6
:10DBD000F00481508093F0048F3F09F055C189E033
:10DBE0008093F0048091EB089091EC0881589F4F4E
:10DBF00039F08091EB089091EC0881588093F504FE
:10DC00008091D103992780739070892B21F48091A2
:10DC1000570580FF1DC08091D307882351F0809164
:10DC2000F304882319F484E08093EB0481E080936B
:10DC3000F3048091D4078823B9F08091F4048823F9
:10DC400019F484E08093EA0481E08093F4040CC02A
:10DC50001092F3041092F4048091CF078093F104A2
:10DC60008091D1078093F2048091F304882309F016
:10DC700073C08091F107282F332724FF07C08091BC
:10DC80000804882319F425FD80C081C09091D00735
:10DC9000983F48F0809151098D3D28F08091F10422
:10DCA00088236CF00AC0983F68F080915109853054
:10DCB00049F48091F10487FF02C0429801C0429A62
:10DCC00081E032C08091EB0481508093EB048F3F60
:10DCD00009F05EC08091F40785FF29C09091F5049A
:10DCE000892F86958093EB04992351F48091F10458
:10DCF00087FF02C0429801C0429A10929D0148C01D
:10DD000080919D019091F104882341F48093F50462
:10DD100080E880939D019923D4F137C0982311F0B6
:10DD2000429A01C04298869580939D0131C08091AE
:10DD3000510986958093EB0480919D01813021F4F7
:10DD40001092F50480E801C0869580939D01809132
:10DD50009D019091F10417C08091EB048150809354
:10DD6000EB048F3FA9F489E08093EB0480919D013F
:10DD7000813011F480E801C0869580939D018091E7
:10DD80009D019091D307892311F0429A01C04298D6
:10DD90008091F404882309F043C09091F10797FF24
:10DDA00007C080910804882319F496FD52C053C01F
:10DDB0009091D207983F48F0809179098D3D28F0E5
:10DDC0008091F20488236CF00AC0983F78F080912B
:10DDD0007909853059F48091F20487FF02C0439895
:10DDE00001C0439A81E080939C0136C08091EA048F
:10DDF00081508093EA048F3F79F580917909869567
:10DE00008093EA0480919C01813011F480E801C084
:10DE1000869580939C0180919C019091F20417C09B
:10DE20008091EA0481508093EA048F3FA9F489E04D
:10DE30008093EA0480919C01813011F480E801C054
:10DE4000869580939C0180919C019091D4078923B1
:10DE500011F0439A01C04398429B04C08091D003C3
:10DE6000886003C08091D003877F8093D003439B59
:10DE700006C08091D00380618093D0030895809183
:10DE8000D0038F7E8093D00308950F931F93CF9379
:10DE9000DF93482FEB0180910904E42FFF27843B97
:10DEA000D8F08F010E0F1F1FF801E754F74F808144
:10DEB00091819B01281B390BC90163E070E00E942E
:10DEC000BD91CB01880F991F860F971F0351174FE4
:10DED000F8019183808306C0EE0FFF1FE351F74FD7
:10DEE00011821082E42FFF27EE0FFF1FE754F74F38
:10DEF000D183C083DF91CF911F910F9108954FB7C8
:10DF000024E130E0F8948091C9008F778093C900B4
:10DF10008091C9008F7B8093C9008091C9008F7D5B
:10DF20008093C9005A9A52985B9A539A832F9927E3
:10DF30008093CD002093CC008091C80082608093B4
:10DF4000C80080E18093C9008091CA008F778093D8
:10DF5000CA008091CA008F7B8093CA008091CA005A
:10DF60008F7D8093CA008091CA008F7E8093CA0003
:10DF70008091CA00877F8093CA008091C9008B7FFF
:10DF80008093C9008091CA0084608093CA00809108
:10DF9000CA0082608093CA008091C80087FF03C0D6
:10DFA0008091CE00F9CF8091C90080688093C9002C
:10DFB0004FBF0895EF92FF920F931F93CF93DF937C
:10DFC000482F00E010E080919E01813061F41092B2
:10DFD0009E0184E48093F8041092FA041092F904EC
:10DFE0001092FB04E6C18091F804882319F421E023
:10DFF00030E001C098019091F904992371F4232B2A
:10E0000011F081E010C084E48093F8049093FA0446
:10E010009093F9049093FB04B5C1913069F4232BDC
:10E0200009F0A6C182E08093F9048091FA048F5F21
:10E030008093FA0483E0A4C19230D1F4232B09F039
:10E0400097C183E08093F8044093FB049091FA0415
:10E05000923039F41092FC0447FF03C081E08093B2
:10E06000FC0483E08093F9049F5F9093FA048AC1D3
:10E07000933009F07DC1232B09F07AC19093F80405
:10E0800082E08093F9048091FA048F5F8093FA0410
:10E090002091FB04822F9927782F6627842F9927B8
:10E0A000682B792B8091AC07813051F47370CB01D0
:10E0B0008050924063E070E00E94BD91EB0119C076
:10E0C000823069F47770CB018050944066E070E054
:10E0D0000E94BD91EB012695269526950CC0EB017B
:10E0E000D370C856D140CE01D7FD0196EC01D5952D
:10E0F000C79526952695022F11270F7010700F5F78
:10E100001F4F0D30110508F02CC10230110519F414
:10E1100004E010E005C00430110511F402E010E045
:10E12000D801A00FB11FFD01E754F74F8081918105
:10E130009E01281B390BC90137FF03C090958195BB
:10E140009F4F069704F5E091EE07EE2351F0FF276D
:10E15000EE0FFF1FE754F74F8081918184369105C0
:10E1600094F480910904883C30F480910904865F1E
:10E170008093090408C088EC8093090480916F00A3
:10E180008F7D80936F00A754B74F8D919C91BC01F8
:10E19000660F771F680F791F6C0F7D1F77FF02C016
:10E1A0006D5F7F4F7B01F594E794F594E794CE0182
:10E1B00001968E159F0524F40894E108F10808C023
:10E1C000CE010197E816F9061CF40894E11CF11C35
:10E1D0000630110509F0ABC0C536D1050CF482C07C
:10E1E0009091F704E92FFF27E95FF54FE081ED37C4
:10E1F00029F48091F60480958093F604993009F013
:10E200006DC08091F604882319F4E33821F066C0CC
:10E21000ED3709F063C08091080A8D3739F4809199
:10E22000090A833899F463E87FEF0DC0833871F4ED
:10E230008091090A833819F460E070E004C08D37DA
:10E2400029F46DE770E085E00E94456F80910A0A2D
:10E250008D3739F480910D0A833899F46DE770E0B9
:10E260000DC0833871F480910D0A833819F460E091
:10E2700070E004C08D3729F463E87FEF86E00E94E8
:10E28000456F80910E0A8D3739F480910F0A8338DB
:10E2900099F463E87FEF0DC0833871F480910F0A21
:10E2A000833819F460E070E004C08D3729F46DE71D
:10E2B00070E089E00E94456F80910C0A992787FDE4
:10E2C0009095BC018AE00E94456F80910B0A9927C6
:10E2D00087FD9095BC018CE00E94456F1092F70479
:10E2E0001092F604CA30D1055CF48091F7048F5F78
:10E2F0008093F704E82FFF27E95FF54F83E88083D9
:10E300008091F7048A3011F41092F7043FEFCC3972
:10E31000D3076CF48091F704E82FFF27E95FF54FEE
:10E320008DE780838091F60480958093F604053014
:10E33000110518F4B701802F11C00730110519F429
:10E34000BE0187E00BC00530110519F4BE0188E05D
:10E3500005C008301105B1F4BE018BE00E94456F85
:10E3600011C00231110570F081E080939E010AC056
:10E3700081E080939E011092FA041092FC0484E4E0
:10E380008093F8048091FA04803198F08091FC0425
:10E39000882331F480919E01882311F480933A01FF
:10E3A0001092FA041092FC041092F90484E4809311
:10E3B000F804E6E0CDB7DEB70C943592CF93FC01BC
:10E3C00097FF05C0CFEFF095E195FF4F01C0C1E089
:10E3D00028E631E0CF01B9010E94BD91FC018B35E7
:10E3E000910554F08B5590408A35910538F484EBB3
:10E3F00090E08E1B9F0BFC0141E00DC0CF01855BBF
:10E4000090408A35910518F4E45BF04003C02E1B60
:10E410003F0BF9014FEFEE0FFF1FE85BF64F259121
:10E4200034918C2F992787FD9095289FB001299FC3
:10E43000700D389F700D1124842F992787FD9095BA
:10E44000689FA001699F500D789F500D1124CA014B
:10E45000CF9108952AE530E0281B390BC9010E94AD
:10E46000DE7108950895089508950895089580E04F
:10E4700090E008951092130A1092120A1092170A4F
:10E480001092160A1092150A1092140A1092180A85
:10E490008AE090E00E946F199093FE048093FD043F
:10E4A0000895CF93DF938091FD049091FE040E9424
:10E4B0007819882309F4AFC08091FD049091FE047F
:10E4C0000A969093FE048093FD04E0E0F0E09F0143
:10E4D00090E05FEFA8E5B8E04BE0ED018B8187FFAE
:10E4E0000BC09F5F8D81E80FF11D8981280F311DC1
:10E4F0008E81851708F4582F4150189647FFEDCFAD
:10E500005093180A232B41F52091030530910405FF
:10E510004091050550910605BB27A52F942F832F09
:10E520009093020580930105AA27BB27281B390B6E
:10E530004A0B5B0BCF01AA27BB27280F391F4A1FA5
:10E540005B1F20930305309304054093050550930A
:10E550000605E5E0F0E013C02091010530910205C9
:10E560002E173F0718F4E21BF30B02C0E0E0F0E0C7
:10E57000892F9927880F991FE80FF91F3596F09377
:10E58000130AE093120AEF3FF10578F480911F011E
:10E59000909120018E9F90018F9F300D9E9F300D96
:10E5A0001124C90164E670E013C0CF0196958795E8
:10E5B0009695879520911F0130912001289FA001F9
:10E5C000299F500D389F500D1124CA0169E170E058
:10E5D0000E94A9917093150A6093140A2091FF0478
:10E5E000309100052E0F3F1F309300052093FF044C
:10E5F0005EE02131350778F08091160A9091170A74
:10E6000001969093170A8093160A20513E4030934A
:10E6100000052093FF04DF91CF91089530911205FA
:10E62000E32FFF2783E0EE0FFF1F8A95E1F7E85AFB
:10E63000F74F2781422F552747FD509580911305AD
:10E640009927841795072CF420931305309315050B
:10E650000AC0222341F080911405992748175907D1
:10E6600014F420931405832F8F5F809312058D304F
:10E67000D0F010921205809114058F3F19F080930D
:10E68000080502C0109208058091130580930905C2
:10E6900080911505809307058FEF809314051092E4
:10E6A000130510921505089595E1899F802D112479
:10E6B0000E94BF8B8AE89CE09F938F9381E99BE83F
:10E6C0009F938F93E0913D05F0913E0509950F9042
:10E6D0000F900F900F900895CF93C0E020919F016D
:10E6E00020930C058091D10385FF02C0C0E123C0B7
:10E6F0009091E4049923B1F080910804882349F4AF
:10E70000E92FFF27EE0FFF1FE150F64F849188237A
:10E7100049F4E92FFF27EE0FFF1FE250F64FC49197
:10E72000CC2349F48091F40786FD03C010929F0129
:10E7300004C0C22F02C0C0930C05809116058C172F
:10E7400071F480911705909118050E94781988231B
:10E7500019F480E090E017C088E893E102C080EDF2
:10E7600097E00E946F199093180580931705CC23AA
:10E7700031F080919F01C81711F410929F01C0934E
:10E7800016058C2F9927CF91089540E050E030E096
:10E790008091E00999278A38910589F08B38910595
:10E7A00024F48938910541F013C08D38910569F042
:10E7B0008E38910539F00CC041E75AE008C049E4B1
:10E7C0005BE005C049E15AE002C045E45AE03CE2A2
:10E7D0009091D50920E08091D609281770F49317FD
:10E7E00060F4DA01A90FB11DE22FFF27EE53F64FB7
:10E7F00085898C939F5F2F5FEECF089520E335E7E7
:10E8000080913B018B3211F08D32F9F480919707A2
:10E81000282F33278091FD039091FE03829FA00152
:10E82000839F500D929F500D1124CA0163E070E048
:10E830000E94BD91CB019B01205D3A48C196C197D2
:10E8400008F03FC02EEF34E73CC0803229F58091BC
:10E85000D10381FF36C020910A0530910B05205D60
:10E860003A4855E72133350748F085E7243938071A
:10E8700018F420E335E702C02456304045E7203342
:10E880003407F8F454E72D3C350718F020E335E75A
:10E8900018C02C593F4F15C08E3549F49091F8039C
:10E8A0008AE0989F90011124205D3A480AC086377B
:10E8B00041F49091F8038AE0989FC0011124281B2D
:10E8C000390BC9010895EF92FF920F931F93992777
:10E8D0008A38910509F444C18B38910524F48938AC
:10E8E000910551F0DEC28D38910509F424C28E38AD
:10E8F000910509F486C1D5C2809103049091040466
:10E90000A0910504B0910604BC01CD0124E630E0DD
:10E9100040E050E00E94F291DA01C9018C509E4F14
:10E920009093770A8093760A0E94FE7390937D0AF3
:10E9300080937C0A90937F0A80937E0A9093810A49
:10E940008093800A2091760A3091770A80917A0A22
:10E9500090917B0A2817390724F430937B0A20937F
:10E960007A0A8091780A9091790A8217930724F4A1
:10E970003093790A2093780A1092730A81E79AE01B
:10E98000909329058093280580913B018093970AF5
:10E990008091D00380FF02C083E401C080E28093B5
:10E9A000980A2091E404222309F1822F6AE00E9450
:10E9B0009D91805D8093820A822F0E949D91892F74
:10E9C000805D8093830A8AE38093840A81E1289F93
:10E9D000F0011124A5E8BAE0E25CF54F9FE08491D4
:10E9E0008D939150319697FFFACF58C28091D10301
:10E9F00085FF0CC0A2E8BAE0EEE5FCE094E184916A
:10EA00008D939150319697FFFACF48C230911005FF
:10EA1000332309F499C087E58093820A80E58093C7
:10EA2000830A40E24093840A20911105822F6AE014
:10EA30000E949D91805D8093850A822F0E949D9106
:10EA4000892F805D8093860A8FE28093870A832FC7
:10EA50000E949D91805D8093880A832F0E949D91E2
:10EA6000892F805D8093890A40938A0A20910D0541
:10EA700030910E0583E0293E380780F0C90168EE29
:10EA800073E00E94A991CB01805D80938B0AC9013C
:10EA900068EE73E00E94A9919C0102C040938B0A2A
:10EAA0002536310580F0C90164E670E00E94A99125
:10EAB000CB01805D80938C0AC90164E670E00E94FE
:10EAC000A9919C0103C080E280938C0AC9016AE08D
:10EAD00070E00E94A991CB01805D80938D0AC901ED
:10EAE0006AE070E00E94A991805D80938E0A8DE6B5
:10EAF00080938F0A80E28093900A20910F0525363B
:10EB000060F0822F64E60E949D91805D8093910A5F
:10EB1000822F0E949D91292F02C08093910A822FFB
:10EB20006AE00E949D91805D8093920A822F0E94EC
:10EB30009D91892F805D8093930A83E78093940A47
:10EB400080E28093950AAAC1A2E8BAE0E4E7FCE07B
:10EB500094E184918D939150319697FFFACF9EC1A5
:10EB60008091030490910404A0910504B0910604DF
:10EB7000BC01CD0124E630E040E050E00E94F2917B
:10EB8000DA01C9018C509E4F90935F0B80935E0B0E
:10EB90000E94FE739093610B8093600B88E78093D3
:10EBA000620B80918E098093630B0E946C7380933B
:10EBB0004B0B80918D0981FF02C084E407C08091D6
:10EBC0008F09833011F480E201C081E28093640BED
:10EBD00089E49BE0909329058093280580918D011D
:10EBE0008093700B8091640B8093720B80919309DA
:10EBF0009091940997FD0196959587958093650B63
:10EC00004DC10E940E738091030490910404A09161
:10EC10000504B0910604BC01CD0124E630E040E0DB
:10EC200050E00E94F291DA01C9018C509E4F9093FE
:10EC3000340A8093330A80911F01909120019093B0
:10EC40002E0A80932D0A80911F01909120019093AC
:10EC5000300A80932F0A80912F099091300997FDF7
:10EC600001969595879580931F0A8093260A209197
:10EC700093093091940937FF02C02F5F3F4F3595BC
:10EC800027952093240A809191099091920964E13B
:10EC900070E00E94A9916093250A20932B0A60934B
:10ECA0002C0A0E94FE7390933C0A80933B0A88E7EB
:10ECB00080933D0A80911F01909120019093380A22
:10ECC0008093370A809108058C5E8093310A809189
:10ECD00009058C5E8093320A8091160A9091170A7A
:10ECE0006AE070E00E94A99170933A0A6093390A31
:10ECF00010921B0A8091120A9091130A9093360A7F
:10ED00008093350A89E19AE090932905809328053C
:10ED10002091D8023091D902C9016CE370E00E94C1
:10ED2000A9916093400AC9016CE370E00E94A99127
:10ED30008093410AB3C00E940E7380919109909113
:10ED4000920964E670E00E94A99170935B0A609357
:10ED50005A0A80912F099091300997FD0196959557
:10ED6000879580934B0A809193099091940997FD20
:10ED70000196959587958093500A80910001482FC0
:10ED800055279A012B5F3F4F80911F0190912001E1
:10ED90002817390784F480911F0190912001841B6A
:10EDA000950B9C01220F331F280F391F822F825190
:10EDB0008093570A02C01092570AE0900304F09023
:10EDC00004040091050410910604C801B70124E66B
:10EDD00030E040E050E00E94F2913093590A2093D5
:10EDE000580A37FF04C01092590A1092580AC801F5
:10EDF000B70124E630E040E050E00E94F291DA01F1
:10EE0000C9018C509E4F90935D0A80935C0A80915B
:10EE10001F01909120019093520A8093510A809192
:10EE20001F01909120019093540A8093530A0E94ED
:10EE3000FE7390935F0A80935E0A88E78093600A6E
:10EE400080911F01909120019093640A8093630A3E
:10EE5000809108058C5E8093550A809109058C5E2F
:10EE60008093560A8091160A9091170A6AE070E022
:10EE70000E94A9917093660A6093650A1092470AEE
:10EE80008091120A9091130A9093620A8093610A0A
:10EE900085E49AE090932905809328052CE230E0E0
:10EEA00002C020E030E0C9011F910F91FF90EF9068
:10EEB0000895EF92FF920F931F93CF93DF9380916A
:10EEC0000A0590910B059C0153E0220F331F5A95C0
:10EED000E1F7281B390B8091190390911A03280F31
:10EEE000391F37FF02C0295F3F4F43E03595279513
:10EEF0004A95E1F730930B0520930A0590911A0586
:10EF0000992309F020C380911905282F332744271E
:10EF100055278F5F80931905F9012131310508F0DC
:10EF20000FC3E857FF4F0C9444928091D10385FFA3
:10EF30002AC080E00E94BF8B80911F019091200128
:10EF40006AE070E00E94BD919F938F9380911F01B2
:10EF5000909120016AE070E00E94BD917F936F93D1
:10EF600080EA9CE09F938F9382EB9BE89F938F9323
:10EF7000E0913D05F0913E0509952DB73EB7285F1C
:10EF80003F4F2DBF28C080E00E94BF8B80911F01A2
:10EF9000909120016AE070E00E94BD919F938F9351
:10EFA00080911F01909120016AE070E00E94BD9164
:10EFB0007F936F938DEA9CE09F938F9381E99BE809
:10EFC0009F938F93E0913D05F0913E0509958DB794
:10EFD0009EB708968DBF8091720980FF39C08091DD
:10EFE00020048823E9F08AE00E94BF8B80913B01D6
:10EFF00099279F938F938091030490910404A0918B
:10F000000504B0910604BC01CD0124E630E040E0E7
:10F0100050E00E94F2913F932F938AEB9CE099C6B7
:10F020008AE00E94BF8B8091030490910404A09118
:10F030000504B0910604BC01CD0124E630E040E0B7
:10F0400050E00E94F2913F932F9386EC9CE0ADC775
:10F050008AE00E94BF8B81ED9CE09F938F9381E9B2
:10F060009BE80C9406818091D10385FF2AC085E13D
:10F070000E94BF8B8091D8029091D9026CE370E01E
:10F080000E94A9919F938F938091D8029091D90269
:10F090006CE370E00E94A9917F936F938BED9CE0ED
:10F0A0009F938F9382EB9BE89F938F93E0913D0515
:10F0B000F0913E0509952DB73EB7285F3F4F2DBF14
:10F0C00028C085E10E94BF8B8091D8029091D9021F
:10F0D0006CE370E00E94A9919F938F938091D80276
:10F0E0009091D9026CE370E00E94A9917F936F9395
:10F0F00088EE9CE09F938F9381E99BE89F938F9389
:10F10000E0913D05F0913E0509958DB79EB70896B3
:10F110008DBF8FE10E94BF8B80E690E09F938F931D
:10F1200080912F09909130099F938F9385EF9CE0F8
:10F130009F938F93C1E9DBE8DF93CF93E0913D0587
:10F14000F0913E0509958091D0032DB73EB7285F19
:10F150003F4F2DBF80FF06C089E20E94BF8B80E039
:10F160009DE073C389E20E94BF8B82E09DE0B9C637
:10F170008091D10385FF1BC08AE20E94BF8B8091E2
:10F18000160A9091170A9F938F9384E09DE09F93B6
:10F190008F9382EB9BE89F938F93E0913D05F091D5
:10F1A0003E0509958DB79EB706968DBF1BC08AE2B6
:10F1B0000E94BF8B8091160A9091170A9F938F939C
:10F1C0008CE09DE09F938F9381E99BE89F938F93C1
:10F1D000E0913D05F0913E0509952DB73EB72A5FB8
:10F1E0003F4F2DBF86E30E94BF8B8091120A909102
:10F1F000130A6AE070E00E94A9919F938F93809117
:10F20000120A9091130A6AE070E00E94A9917F931C
:10F210006F9384E19DE09F938F9381E99BE89F9397
:10F220008F93E0913D05F0913E0509958DB79EB70E
:10F230000896C9C689E00E94BF8B80E29DE09F933B
:10F240008F9301E91BE81F930F93E0913D05F09127
:10F250003E0509958EE10E94BF8B0F900F900F9095
:10F260000F9082E29DE09F938F931F930F93E09105
:10F270003D05F0913E05099583E30E94BF8B0F90F9
:10F280000F900F900F9084E29DE09F938F931F93B8
:10F290000F93E0913D05F0913E0509958FE30E94A3
:10F2A000BF8B0F900F900F900F9086E29DE09F9381
:10F2B0008F931F930F93E0913D05F0913E050995C3
:10F2C0008EE70E94BF8B0F900F900F900F908CE3F2
:10F2D0009DE09F938F931F930F939AC780919901FD
:10F2E000882309F462C08DE50E94BF8B82E59DE012
:10F2F0009F938F93C1E9DBE8DF93CF93E0913D05C6
:10F30000F0913E05099584E50E94BF8B0F900F9008
:10F310000F900F9080918E0999279F938F9384E58A
:10F320009DE09F938F93DF93CF93E0913D05F09104
:10F330003E0509958EE50E94BF8B2DB73EB72A5F2B
:10F340003F4F2DBF80919109909192096AE070E042
:10F350000E94A9917F936F938DE59DE09F938F937A
:10F36000DF93CF93E0913D05F0913E0509958DB770
:10F370009EB706968DBF80918F09833081F480916E
:10F380008D0981FF06C08BE50E94BF8B87E69DE05B
:10F39000A8C58BE50E94BF8B8AE69DE0A2C58BE5E0
:10F3A0000E94BF8B8DE69DE02DC784E0D3C3809182
:10F3B0009901882309F47AC080911C0591E9E92E0E
:10F3C0009BE8F92E882309F44BC089E60E94BF8B85
:10F3D0008091E30499279F938F9380E79DE09F930B
:10F3E0008F93FF92EF92E0913D05F0913E050995D4
:10F3F00085E70E94BF8B2DB73EB72A5F3F4F2DBFD9
:10F4000080918D0199279F938F9300E610E01F93C1
:10F410000F9380919309909194099F938F938BE719
:10F420009DE09F938F93FF92EF92E0913D05F091C5
:10F430003E05099582E70E94BF8B8DB79EB70A965D
:10F440008DBF8091E10499279F938F931F930F9312
:10F450008091E20499279F938F9387E89DE073C67C
:10F4600089E60E94BF8B80918D0199279F938F938E
:10F4700080E690E09F938F938091930990919409F7
:10F480009F938F938091900999279F938F9387E9FA
:10F490009DE09F938F93FF92EF92E0913D05F09155
:10F4A0003E0509958DB79EB70C968DC585E052C374
:10F4B0009091E4049923D1F080912505882381F06F
:10F4C000903270F487E00E94547383E90E94BF8BEE
:10F4D0008091E40499279F938F9380EB9DE0A4C3D0
:10F4E00083E90E94BF8B8BEB9DE0B3C38091D10376
:10F4F00001E9E02E0BE8F02E85FF06C084E90E94AA
:10F50000BF8B81EC9DE0DAC383E90E94BF8B84ED61
:10F510009DE0D4C38091AE0B863059F480911C05D8
:10F52000882319F010921C059AC681E080931C056F
:10F5300096C6883009F093C60E94C48B81E0DBC375
:10F540009093190594C6913009F0E0C38091190594
:10F55000282F3327442755278F5F80931905F901FA
:10F560002131310508F07EC6E756FF4F0C944492D6
:10F570008091D10385FF43C080E00E94BF8B8091C2
:10F58000160A9091170A9F938F9380911F01909173
:10F5900020016AE070E00E94BD919F938F9380915B
:10F5A0001F01909120016AE070E00E94BD917F935D
:10F5B0006F938091D8029091D9026CE370E00E9421
:10F5C000A9919F938F938091D8029091D9026CE377
:10F5D00070E00E94A9917F936F938AEE9DE09F93C4
:10F5E0008F9382EB9BE89F938F93E0913D05F09181
:10F5F0003E0509952DB73EB7225F3F4FB1C580E06C
:10F600000E94BF8B8091160A9091170A9F938F9347
:10F6100080911F01909120016AE070E00E94BD91ED
:10F620009F938F9380911F01909120016AE070E079
:10F630000E94BD917F936F938091D8029091D902DF
:10F640006CE370E00E94A9919F938F938091D80200
:10F650009091D9026CE370E00E94A9917F936F931F
:10F6600085E09EE0C2C285E10E94BF8B80E690E00B
:10F670009F938F9380918A0190918B019F938F9399
:10F6800080E29EE09F938F93C1E9DBE8DF93CF9305
:10F69000E0913D05F0913E050995809172092DB7E5
:10F6A0003EB7285F3F4F2DBF80FF51C0809120049F
:10F6B000882339F18FE10E94BF8B809103049091E0
:10F6C0000404A0910504B0910604BC01CD0124E618
:10F6D00030E040E050E00E94F2913F932F938AE2A5
:10F6E0009EE09F938F9381EA9BE89F938F93E09195
:10F6F0003D05F0913E0509958DB79EB706968DBFE5
:10F7000038C08FE10E94BF8B809103049091040464
:10F71000A0910504B0910604BC01CD0124E630E0BF
:10F7200040E050E00E94F2913F932F9383E39EE0EC
:10F730009F938F93DF93CF93E0913D05F0913E052A
:10F7400009952DB73EB72A5F3F4F2DBF12C08FE1FD
:10F750000E94BF8B8CE39EE09F938F93DF93CF93A8
:10F76000E0913D05F0913E0509950F900F900F90A7
:10F770000F9089E20E94BF8B80913B0199279F9354
:10F780008F9386E49EE09F938F93DF93CF9313C470
:10F79000809199018823F9F08BE20E94BF8B8091C0
:10F7A0008D0199279F938F93809191099091920950
:10F7B0006AE070E00E94A9917F936F9380E690E0E9
:10F7C0009F938F9380919309909194099F938F9326
:10F7D00089E49EE058C182E0BDC18FE30E94BF8BE7
:10F7E0008091140A9091150A9F938F938091120A29
:10F7F0009091130A6AE070E00E94A9919F938F9301
:10F800008091120A9091130A6AE070E00E94A99117
:10F810007F936F9380E69EE09F938F93C1E9DBE82F
:10F82000DF93CF93E0913D05F0913E0509958091DE
:10F83000D0032DB73EB7265F3F4F2DBF80FF0AC0D4
:10F8400082E50E94BF8B84E79EE09F938F9381EABD
:10F850009BE8DCC482E50E94BF8B87E79EE041C342
:10F860008091990111E9E12E1BE8F12E882309F41A
:10F8700049C084E50E94BF8B80918E0999279F9390
:10F880008F938091900999279F938F938AE79EE0A9
:10F890009F938F93E701FF92EF92E0913D05F091E6
:10F8A0003E0509958DB79EB708968DBF80918F094B
:10F8B000833051F484E60E94BF8B8DE89EE09F93D5
:10F8C0008F93FF92EF920BC084E60E94BF8B83E977
:10F8D0009EE09F938F9382EB9BE89F938F93E091A1
:10F8E0003D05F0913E0509950F900F900F900F90F8
:10F8F00080918D0981FFBBC484E60E94BF8B89E99A
:10F900009EE0EFC284E50E94BF8B8FE99EE0D6C1E6
:10F9100080911B05C1E9EC2ECBE8FC2E882309F46D
:10F9200050C089E60E94BF8B809175086AE00E94F2
:10F930009D91892F99279F938F93809175080E949D
:10F940009D9199279F938F9380916D080E949D911F
:10F95000892F99279F938F9380916D080E949D9185
:10F9600099279F938F93809165080E949D91892F7D
:10F9700099279F938F93809165080E949D91992765
:10F980009F938F9380915D080E949D91892F992765
:10F990009F938F9380915D080E949D9199279F93DB
:10F9A0008F9385EB9EE09F938F93FF92EF92E09170
:10F9B0003D05F0913E0509952DB73EB72C5E3F4FB2
:10F9C000CFC389E60E94BF8B80E690E09F938F9320
:10F9D00080917708992787FD90959F938F938091C9
:10F9E0006F08992787FD90959F938F938091670863
:10F9F000992787FD90959F938F9380915F08992712
:10FA000087FD90959F938F9382ED9EE09F938F93B8
:10FA1000FF92EF92E0913D05F0913E0509958DB77B
:10FA20009EB70E96D0C280911B05909184078823C3
:10FA300009F48DC0943009F48CC09630A1F58EE79E
:10FA40000E94BF8B809185086AE00E949D91892F5A
:10FA500099279F938F93809185080E949D91992764
:10FA60009F938F9380917D080E949D91892F992764
:10FA70009F938F9380917D080E949D9199279F93DA
:10FA80008F9385EE9EE09F938F9381E99BE89F93F0
:10FA90008F93E0913D05F0913E0509952DB73EB756
:10FAA000245F3F4F5DC3973008F4E1C38EE70E94A7
:10FAB000BF8B809195086AE00E949D91892F9927BC
:10FAC0009F938F93809195080E949D9199279F9372
:10FAD0008F9380918D080E949D91892F99279F93E4
:10FAE0008F9380918D080E949D9199279F938F936A
:10FAF000809185080E949D91892F99279F938F93CC
:10FB0000809185080E949D9199279F938F93809162
:10FB10007D080E949D91892F99279F938F938091B3
:10FB20007D080E949D9199279F938F9384EF9EE07B
:10FB30009F938F9381E99BE89F938F93E0913D057D
:10FB4000F0913E0509958DB79EB744963CC294301E
:10FB500021F486E00E9454738AC39630F1F48EE754
:10FB60000E94BF8B80E690E09F938F9380918708DF
:10FB7000992787FD90959F938F9380917F08992770
:10FB800087FD90959F938F9381E19FE09F938F9343
:10FB900081E99BE89F938F93DAC2973008F467C39B
:10FBA0008EE70E94BF8B80E690E09F938F938091B9
:10FBB0009708992787FD90959F938F9380918F0841
:10FBC000992787FD90959F938F9380918708992718
:10FBD00087FD90959F938F9380917F08992787FD4C
:10FBE00090959F938F9384E29FE09F938F9381E9F9
:10FBF0009BE89F938F930ECF9091E404992309F48F
:10FC00004AC0809125058823F9F09032E8F487E016
:10FC10000E94547383E90E94BF8B8091E40499276A
:10FC20009F938F9387E39FE09F938F9381EA9BE855
:10FC30009F938F93E0913D05F0913E0509952DB777
:10FC40003EB72A5F3F4F8CC283E90E94BF8B82E49C
:10FC50009FE09F938F9301E91BE81F930F93E0911F
:10FC60003D05F0913E0509951F921F929091E40485
:10FC700081E1989FC0011124825C954F9F938F93DF
:10FC80001F930F93E0913D05F0913E0509958DB7C7
:10FC90009EB70A9698C18091D103B1E9EB2EBBE8DB
:10FCA000FB2E85FF06C084E90E94BF8B88E49FE09D
:10FCB00005C083E90E94BF8B8BE59FE09F938F93E4
:10FCC000FF92EF92A5C28091AE0B863079F48091BD
:10FCD0001B05882319F010921B0503C081E0809357
:10FCE0001B0585E00E94547386E0AEC2883031F473
:10FCF0000E94C48B82E080931A05AFC2813009F064
:10FD0000AEC20E94C48B10921A05A7C2923009F0AD
:10FD1000ACC280911905282F3327442755278F5FC0
:10FD200080931905F9012131310508F09BC2E65590
:10FD3000FF4F0C94449280E00E94BF8B85EF97E0C8
:10FD40009F938F930E94633099279F938F9381E7AE
:10FD50009FE09F938F9381EA9BE89F938F93E0911D
:10FD60003D05F0913E0509952DB73EB7285F3F4F01
:10FD7000F7C185E10E94BF8B83E098E09F938F934A
:10FD8000809100016AE00E949D91892F99279F939D
:10FD90008F93809100010E949D9199279F938F934B
:10FDA00080E89FE09F938F9381E99BE89F938F93D7
:10FDB000E0913D05F0913E05099569CF8AE20E94E8
:10FDC000BF8B81E99FE09F938F93C1E9DBE8DF93CD
:10FDD000CF93E0913D05F0913E0509958091720920
:10FDE0000F900F900F900F9080FF41C0809192076D
:10FDF0009091750181FD0BC0892F99279F938F9357
:10FE000086E99FE09F938F93DF93CF9313CFE09189
:10FE10003D05F0913E05933318F080EA9FE002C063
:10FE200087EA9FE09F938F93DF93CF9309950F907D
:10FE30000F900F900F9080915609E0913D05F09141
:10FE40003E059091750180FF0BC0892F99279F93E4
:10FE50008F938EEA9FE09F938F93DF93CF93AFC0F2
:10FE6000892F99279F938F9384EB9FE0CFC08AEBD4
:10FE70009FE037C08FE30E94BF8B83EC9FE09F938E
:10FE80008F93C1E9DBE8DF93CF93E0913D05F091DB
:10FE90003E0509950F900F900F900F908091E80705
:10FEA000882319F487EC9FE01CC08091DE03E09169
:10FEB0003D05F0913E05882319F080ED9FE002C0DA
:10FEC00087ED9FE09F938F93DF93CF9309950F90DA
:10FED0000F900F900F908091F30786FFC8C18EEDB1
:10FEE0009FE09F938F93DF93CF9392C184E50E940D
:10FEF000BF8B85EE9FE09F938F93C1E9DBE8DF9393
:10FF0000CF93E0913D05F0913E05099580917209EE
:10FF10000F900F900F900F9085FD03C08AEE9FE029
:10FF200011C08091D607883F10F4E82F07C0EFEF8B
:10FF3000F0E0E81BF109E65FFB4FE081E23358F4A3
:10FF400083EF9FE09F938F93DF93CF93E0913D05E5
:10FF5000F0913E0516C0E43B18F08AEF9FE0F2CF27
:10FF60008091F307E0913D05F0913E0585FF03C0C8
:10FF700081E090E102C088E090E19F938F93DF934E
:10FF8000CF9309950F900F900F900F908091EC07F1
:10FF9000882309F46CC18EE50E94BF8B8091EC0729
:10FFA00099279F938F938FE090E19F938F9381E99F
:10FFB0009BE89F938F93E0913D05F0913E05099555
:10FFC0008DB79EB706968DBF52C189E60E94BF8B42
:10FFD0008AE190E19F938F93C1E9DBE8DF93CF93B0
:10FFE000E0913D05F0913E0509950F900F900F901F
:10FFF0000F908091EB07E0913D05F0913E0588233D
:020000021000EC
:1000000051F099279F938F9384E290E19F938F9370
:10001000DF93CF9313CE88E290E19F938F93DF938A
:10002000CF93FAC080911D05A1E9EA2EABE8FA2E24
:10003000882309F053C08EE70E94BF8B809169012D
:1000400099279F938F9380918707E82FFF27EE0FC3
:10005000FF1FE754F74F808191819F938F93809189
:100060008607E82FFF27EE0FFF1FE754F74F808129
:1000700091819F938F938EE290E19F938F93FF9254
:10008000EF92E0913D05F0913E05099583E90E94CC
:10009000BF8B8DB79EB70A968DBF80918907E82FD9
:1000A000FF27EE0FFF1FE754F74F808191819F9349
:1000B0008F9380918807E82FFF27EE0FFF1FE754EB
:1000C000F74F8081918181589F4F9F938F9382E456
:1000D00090E19F938F93FF92EF9241CE8EE70E9423
:1000E000BF8B80910C0499279F938F9380910B0471
:1000F00099279F938F9380910A0499279F938F93B9
:1001000081E590E19F938F93FF92EF92E0913D05FF
:10011000F0913E05099583E90E94BF8B8DB79EB78C
:100120000A968DBF80910F0499279F938F9380919A
:100130000E0499279F938F9380910D0499279F9385
:100140008F9385E690E19F938F93FF92EF92E091DA
:100150003D05F0913E0509952DB73EB7265F3F4F0F
:100160002DBF85C080912505882309F480C08EE7C6
:100170000E94BF8B8091720986FD11C089E790E1D2
:100180009F938F9382EB9BE89F938F93E0913D0524
:10019000F0913E0509950F900F900F900F90809170
:1001A000F10799278F709070892B89F088E890E18A
:1001B0009F938F9382EB9BE89F938F93E0913D05F4
:1001C000F0913E0509950F900F900F900F90809140
:1001D000720982FF11C082E990E19F938F9382EBB5
:1001E0009BE89F938F93E0913D05F0913E05099523
:1001F0000F900F900F900F908091720983FD37C080
:1002000087E990E19F938F9382EB9BE89F938F9375
:10021000E0913D05F0913E0509950F900F900F90EC
:100220000F9025C00091AE0B063089F480911D051A
:10023000882319F010921D0503C081E080931D05ED
:1002400086E00E94547387E00E94547308C0013016
:1002500031F40E94C48B00931A0510921905109274
:10026000AE0B05C01092190502C010921A05E6E007
:10027000CDB7DEB70C9435924FB728E130E0F89453
:100280008091C9008F778093C9008091C9008F7BCE
:100290008093C9008091C9008F7D8093C9005A9ACC
:1002A00052985B9A539A832F99278093CD0020937D
:1002B000CC008091C80082608093C80080E1809368
:1002C000C9008091CA008F778093CA008091CA00CC
:1002D0008F7B8093CA008091CA008091CA008F7E74
:1002E0008093CA008091CA0088608093CA00809180
:1002F000C9008B7F8093C9008091CA00846080937D
:10030000CA008091CA0082608093CA008091C800B0
:1003100087FF03C08091CE00F9CF8091C90080682B
:100320008093C90080918C0B846080938C0B4FBFAD
:1003300008959091F804992341F48F3031F490930B
:100340001F0580E58093F8040895E0911F05EF5F95
:10035000E0931F05E83121F481E080931E050895A4
:10036000E93120F089E180931F050895FF27EB58BC
:10037000F44F80830895A0E0B0E0E1ECF1E80C9444
:10038000159291E0D92E82E0A82EBD2CE12C01E03F
:10039000F02E80918C0B82FDB5C080916F008F7D17
:1003A00080936F00E091EE07EE2351F0FF27EE0FF0
:1003B000FF1FE754F74F80819181843691055CF4EB
:1003C00080910904883C20F4809109048C5E01C06E
:1003D00088EC809309048091760B682F77278091B1
:1003E00020058150809320058F3F31F41CE7C12EFA
:1003F00082E08093200502C0C4E2CC2E40E04C1580
:1004000008F07EC0EA2DFF27EB58F44F80818D2144
:1004100011F06E297F298D2D9927880F991FD82ECD
:10042000882319F4B1E0DB2EAD0CEE0CFF1C20E0AC
:10043000E21628E0F20609F061C0A1E0EA2EF12CF4
:10044000CB018050944065E070E00E94BD91AB2DDF
:10045000BB27FD01EA0FFB1FE754F74F8081918115
:100460009C01220F331F280F391F260F371F37FF1C
:1004700002C02D5F3F4FE901D595C795D595C7952A
:10048000CB0101968C179D0714F4219706C061508B
:100490007040C617D7070CF4219680910904833C5D
:1004A000D8F08D010A0F1B1FF801E754F74F808128
:1004B0009181FE01E81BF90BCF0163E070E00E941F
:1004C000BD91CB01880F991F860F971F0351174FBE
:1004D000F8019183808307C0AA0FBB1FA351B74FB8
:1004E00011961C921E92EB2DFF27EE0FFF1FE75473
:1004F000F74FD183C08360E070E0B3944F5F7FCF4C
:1005000010923A0110921E05EAE0CDB7DEB70C94C6
:1005100031920895089540E050E080912105909136
:1005200022059C01220F331F280F391F80911903C8
:1005300090911A03280F391F37FF02C02D5F3F4FDC
:1005400035952795359527953093220520932105DC
:1005500080913B018B32D9F480919707282F332764
:100560008091FD039091FE03829FA001839F500D17
:10057000929F500D1124CA0157FD4F96AC0125E002
:10058000559547952A95E1F74B5F5F4F3DC08D32FA
:10059000D9F480919707282F33278091FD039091FC
:1005A000FE03829FA001839F500D929F500D112446
:1005B000CA0157FD4F96AC0195E0559547959A9520
:1005C000E1F74550504020C0803271F48091D10352
:1005D00081FF1AC0C90137FD4F96AC0185E05595E2
:1005E00047958A95E1F710C08E3529F48091F8037C
:1005F000482F552709C0863739F48091F803992789
:1006000044275527481B590BCA01AA2797FDA095D7
:10061000BA2F8093920290939302A0939402B09386
:10062000950208950F931F930E940E7380911F01EE
:1006300090912001AA2797FDA095BA2F8093C10120
:100640009093C201A093C301B093C4018091120A98
:100650009091130AAA27BB278093D4019093D501C8
:10066000A093D601B093D7010AE010E08091160A5A
:100670009091170AB8010E94A991CB01AA27BB2724
:100680008093E7019093E801A093E901B093EA0118
:100690008091030490910404A0910504B091060494
:1006A000BC01CD0124E630E040E050E00E94F29130
:1006B0002093FA013093FB014093FC015093FD011C
:1006C00080918A0190918B01AA2797FDA095BA2F5E
:1006D00080930D0290930E02A0930F02B09310022C
:1006E00080918E099927AA27BB2780932002909397
:1006F0002102A0932202B0932302809190099927AE
:10070000AA27BB278093330290933402A09335022B
:10071000B09336028091910990919209B8010E949C
:10072000A991CB01AA27BB27809346029093470249
:10073000A0934802B0934902809193099091940943
:10074000AA2797FDA095BA2F8093590290935A0239
:10075000A0935B02B0935C02809109059927AA27B8
:10076000BB2780936C0290936D02A0936E02B093AE
:100770006F028091E3049927AA27BB2780937F0209
:1007800090938002A0938102B09382028091E4044E
:100790009927AA27BB278093A5029093A602A0932E
:1007A000A702B093A8021F910F9108950024222759
:1007B0003327442751E0BB27EE27FF27A0E1660F30
:1007C000771F881F991F001C221F331F441F660FAD
:1007D000771F881F991F001C221F331F441F2AF4F4
:1007E000050E2B1F3E1F4F1F04C0051A2B0B3E0B7F
:1007F0004F0B550FBB1FEE1F587F556047FD5250E2
:10080000AA95E9F6E695B7955795E695B795579564
:10081000852F9B2F08952227332741E0552768E035
:10082000880F991F221F331F880F991F221F331F04
:100830001AF4240F351F02C0241B350B440F551F1B
:10084000487F456037FD42506A9551F75695479568
:1008500056954795842F0895AA2797FF04C0809541
:1008600090958A1F9A1F77FF04C0609570956A1F44
:100870007A1F669F9001779FA001679F300D411DF1
:100880005A1F300D411D5A1F889FF001999F2E0F4E
:100890003F1F401D511D899F300D411D5A1F300DB6
:1008A000411D5A1FCA01B901112480CF4FB720E45E
:1008B00030E0F8948091C9008F778093C9008091CF
:1008C000C9008F7B8093C9008091C9008F7D809380
:1008D000C9005A9A52985B9A539A832F992780930A
:1008E000CD002093CC008091C80082608093C80026
:1008F00088E18093C9008091CA008F778093CA00F5
:100900008091CA008F7B8093CA008091CA008F7D3E
:100910008093CA008091CA008F7E8093CA00809124
:10092000CA00877F8093CA008091C9008B7F809323
:10093000C9008091CA0084608093CA008091CA0077
:1009400082608093CA008091C80087FF03C08091B5
:10095000CE00F9CF8091C90080688093C9004FBF55
:1009600008950F931F93CF93DF93482F4F5F8931E3
:1009700008F08BC08091B808841720F44F5F409333
:10098000B8084150CB0183539B4268E170E00E945C
:10099000BD91A42FBB27FD01EA0FFB1FE754F74FC2
:1009A000808191819B01281B390BC90137FF03C04E
:1009B000909581959F4F069794F480910904883C07
:1009C00030F480910904865F8093090408C088ECA4
:1009D0008093090480916F008F7D80936F00FD01EB
:1009E000EA0FFB1FE754F74F808191819C01220F92
:1009F000331F280F391F260F371F37FF02C02D5F07
:100A00003F4FE901D595C795D595C795CB0101967F
:100A10008C179D0714F4219706C061507040C617CB
:100A2000D7070CF4219680910904843BD8F08D01FE
:100A30000A0F1B1FF801E754F74F80819181FE01D7
:100A4000E81BF90BCF0163E070E00E94BD91CB0180
:100A5000880F991F860F971F0351174FF801918335
:100A6000808307C0AA0FBB1FA351B74F11961C92DA
:100A70001E92E42FFF27EE0FFF1FE754F74FD1839D
:100A8000C083443011F410923A01DF91CF911F914D
:100A90000F910895CF93DF932091AF0B822F992769
:100AA000807F9070409709F06CC02F3109F046C0EC
:100AB0008091B00B80932C052091B20B20932E05D2
:100AC0008091B30B80932D05822F99279093BA08BC
:100AD0008093B908222309F054C080918607282FFB
:100AE0003327220F331FF901E351F74F1182108290
:100AF00080918707A82FBB27AA0FBB1FFD01E351D9
:100B0000F74F1182108280918907E82FFF27EE0F9F
:100B1000FF1FCF018351974FEC0119821882275490
:100B2000374FE90119821882A754B74F11961C92CA
:100B30001E92E754F74F1182108223C0C22FCF704C
:100B4000CA30F8F48091B00B8093DB0B8091B10B2D
:100B50008093DA0B8091B20B8093DD0B8091B30B05
:100B60008093DC0B6091DA0B7091DB0B8C2F0E9471
:100B7000B1846091DC0B7091DD0B8C2F8F5F0E9434
:100B8000B184DF91CF910895CF93C82F8F3F49F45F
:100B900080912F058F3F29F4109231051092300576
:100BA00032C020913105222339F4CF3111F485E090
:100BB00001C084E080933205809132059091300528
:100BC0008217A0F4892F8095809330058F3F19F408
:100BD0008EEF8093300580913005C81711F40E9484
:100BE0004A8510923105109230050BC0E22FFF2785
:100BF000E155F44FC0832F5F209331059C0F9093F4
:100C00003005C0932F05CF91089590912B05933215
:100C100040F4E92FFF27E954F44F80839F5F9093BE
:100C20002B050895833218F48D5F80932B0508956A
:100C300090E2EAEBFBE08FE19193815087FFFCCFDC
:100C40000895CF93CFB723E031E0F8948091C900A5
:100C50008F778093C9008091C9008F7B8093C900F2
:100C60008091C9008F7D8093C9005A9A52985B9AEF
:100C7000539A832F99278093CD002093CC008091A5
:100C8000C80082608093C80088E18093C900809189
:100C9000CA008F778093CA008091CA008F7B8093AF
:100CA000CA008091CA0080628093CA008091CA0005
:100CB00080618093CA008091CA0088608093CA00D6
:100CC0008091C90084608093C9008091CA008460CB
:100CD0008093CA008091CA0082608093CA0080918C
:100CE000C80087FF03C08091CE00F9CF8091C90072
:100CF00080688093C9008091C90080648093C90096
:100D00000E941886CFBFCF910895282F99278F7002
:100D10009070892B31F4209580912A05822B809345
:100D20002A0508951F920F920FB60F9211248F93E8
:100D3000EF93FF938091D202882309F068C0E0917D
:100D40003405EE2389F480913305882369F480917A
:100D5000B70B882321F081E08093350505C0809191
:100D6000C90081608093C90080913505882379F49A
:100D7000EF5FE093340580918E0B8E1720F481E0B5
:100D8000809335051CC0FF27E257F44F3CC080918B
:100D90003305882361F48091B70B882311F483E035
:100DA00003C0813999F481E0809333050FC083300B
:100DB00099F48091B70B882349F01092B70B80917A
:100DC000C9008E7F8093C9008EEF1EC08091C9003C
:100DD00081608093C9000EC0833261F48091C900A4
:100DE0008E7F8093C9008FEF8093CE0081E0809347
:100DF000D20218C080913305E82FFF27E954F44F41
:100E00008F5F8093330580818093CE000BC010925A
:100E1000330510923405109235058091C900806128
:100E20008093C900FF91EF918F910F900FBE0F90AB
:100E30001F901895682727E0322F67FF06C0862F7E
:100E40009927880F991F832702C0862F880F682F44
:100E5000215027FFF2CF992708950F931F93CF9327
:100E6000DF93062F60E0162F601740F4EC018991A4
:100E70000E941A87682F1F5F1017C8F3862F9927C3
:100E8000DF91CF911F910F910895DC0190E09617AB
:100E900058F48C91803241F09F5F961728F4FD0141
:100EA000E90FF11D8081F6CF892F99270895A0E0E1
:100EB000B0E0EDE5F7E80C9416928FE980938F0B84
:100EC00080E18093910B84EA8093920B85E5809377
:100ED000930B8DE58093940B1092950B80913705C1
:100EE000882309F06AC08091360513E1819FC00113
:100EF000112463E086559E4F0E944587082F8091FC
:100F00003605819FC00111246AE080569E4F0E94E1
:100F10004587982F800F865F80938E0B4EEFB42EFF
:100F2000B80EB092900B209136052093960BE92EC7
:100F3000FF24C70133E0880F991F3A95E1F7802B12
:100F40008093970B822F992723E1C22ED12C8C9D61
:100F500090018D9D300D9C9D300D1124C90180564E
:100F60009E4FA701BC0188E99BE00E94DE8F1127FC
:100F70008091360599278C9DE0018D9DD00D9C9D1B
:100F8000D00D1124CE0186559E4FA801BC01C7018A
:100F90008856944F0E94DE8F0257144F0E0D1F1D6E
:100FA0006B2D80E99BE00E942D87F801828780915C
:100FB00037058F5F8093370570C01091950B0E94A5
:100FC00012834091D3024031C8F563E170E0812F74
:100FD0009927DC01AA0FBB1FA80FB91FA257B44F56
:100FE000842F9927869FF001879FF00D969FF00D23
:100FF0001124E056FE4F2585C4E0880F991FCA953D
:10100000E1F7282BED012887268537853F798289EE
:101010009927982F88279295990F907E282B392B06
:101020002987832F99278A87842F8F5F1F5F163028
:1010300018F4482F803158F28093D30283E0189F30
:1010400090011124822F885F80938E0B825C8093A5
:10105000900B812F99278C01000F111F080F191F6A
:101060000257144F822F8A5F682F80E99BE00E940D
:101070002D87F80180878091D302803170F081E064
:101080008093D30210923705809136058F5F80934D
:101090003605803110F010923605E9E0CDB7DEB7A5
:1010A0000C9432928091D202882309F447C0809137
:1010B000D10385FD04C08091D602882381F082E9A6
:1010C0008093B70B83E28093B80B8091D60288237C
:1010D00009F485E58093B90B1092D60202C0809383
:1010E000B70B8091D4028F3071F480912A050E9451
:1010F0003772882341F081E98093B70B8093B80B56
:1011000081E38093B90B1092D2028091C80085FFD1
:10111000FCCF8091C9008F7E8093C9008091C90067
:101120008E7F8093C9000E9457878EE78093CE0000
:1011300080912A058093D40210922A050895EF9297
:10114000FF920F931F93CF93DF937C018B01EA01F2
:10115000452B39F0F80181918F01F701099521970D
:10116000C9F7E6E0CDB7DEB70C943592EF92FF9267
:101170000F931F93CF93DF937C018B01EA01452BE3
:1011800041F0F8010F5F1F4F8491F70109952197F6
:10119000C1F7E6E0CDB7DEB70C9435920F931F93FD
:1011A000CF938C01C62F161634F480E2F80109950E
:1011B000C1501C16D4F3CF911F910F9108950F9336
:1011C0001F93CF938C01C62F161634F480E3F801D9
:1011D0000995C1501C16D4F3CF911F910F9108951A
:1011E000A5E3B0E0E6EFF8E80C940D922E96EEAD94
:1011F000FFAD2E97882499245401809124058823DB
:1012000021F42C961FAE1EAE2C97AEE44A2E512C24
:101210004C0E5D1E6F01B60105C0153239F0089401
:10122000C11CD11CF60114911123B9F7A601461B6C
:10123000570B31F02C968EAD9FAD2C970E94B6883F
:10124000112309F46AC20894C11CD11CFF24FDA615
:10125000FCA6FFEFEF2EF9A6F6010894C11CD11CE5
:101260001491153721F0812F80628837B1F4F0FE98
:101270000AC0F20124E030E0420E531E80809180CB
:10128000A280B3800AC0F20142E050E0440E551E35
:10129000808191814C01AA24BB24103221F489A5BC
:1012A0008823D1F61DC0133219F458E0F52AD4CFA3
:1012B0001A3211F01D3291F41A3259F4F20182E01F
:1012C00090E0480E591EE081ECA7EE232CF6E19544
:1012D000ECA790E1F92AAFEDFA22BECF1B3211F450
:1012E00019A7BACF1E32C1F5F6010894C11CD11C52
:1012F00014911A3279F4F20122E030E0420E531ECA
:10130000408151813FEF4F3F530714F44FEF5FEFA0
:10131000E42EA2CF40E050E0812F80538A30A0F429
:10132000CA01E3E0880F991FEA95E1F7840F951F42
:10133000480F591F410F511D40535040F60108946A
:10134000C11CD11C1491E8CF8FEF4F3F580714F404
:101350004FEF5FEFE42E85CF103329F4F4FC7CCF00
:1013600090E2F92A79CF812F81538930D8F440E077
:1013700050E0CA0173E0880F991F7A95E1F7840F56
:10138000951F480F591F410F511D40535040F60102
:101390000894C11CD11C1491812F80538A3048F3CA
:1013A0004CA75FCF183619F4A4E0FA2A55CF1C36A3
:1013B00019F4B1E0FB2A50CF133661F43E010894D2
:1013C000611C711CF20122E030E0420E531E80814C
:1013D00089833CC1143421F0143611F0193651F5CB
:1013E000143411F431E0F32AF0FE0AC0F20144E0B3
:1013F00050E0440E551E80809180A280B3800CC0C6
:10140000F20182E090E0480E591E808191814C01EA
:10141000AA2497FCA094BA2CB7FE0AC0B094A0945A
:1014200090948094811C911CA11CB11C8DE289A711
:101430000AE06FC01F3411F01F3631F41F3411F46D
:1014400091E0F92A08E064C0103779F4F201A2E0D3
:10145000B0E04A0E5B1E808191814C01AA24BB241E
:1014600000E1B0E4FB2A18E753C01337C1F5F201DD
:1014700022E030E0420E531E6080718061147104DE
:1014800089F43E010894611C711C88E289838EE610
:10149000F301818385E78B838CE68C838D8389E2DE
:1014A0008E831F82E7FC13C08E2D992787FD9095B0
:1014B000AC0160E070E0C3010E94D18F009729F079
:1014C000382E3618E3140CF0C3C03E2CC1C0F30113
:1014D00001900020E9F731973E2E3618B9C0153536
:1014E00011F0153731F4153511F4F1E0FF2A0AE057
:1014F0000FC0183519F0183709F0A0C000E1F3FE4D
:1015000007C081149104A104B10411F020E4F22A6F
:1015100019A6EDA6E7FC02C03FEDF32269E2662EB4
:10152000712C6C0E7D1E81149104A104B10421F470
:101530004DA5442309F47BC0802F9927AA27BB27F8
:101540008EA79FA7A8ABB9AB202E332490E08916B5
:1015500090E0990691E0A90690E0B90648F0C5012F
:10156000B4012EA53FA548A959A90E94D09117C042
:10157000AFEF8A169104A104B10449F040F0C40110
:10158000B1010E94A9919B014427552708C0882DCD
:10159000602F0E949D91282F3327442755272AAB7F
:1015A0003BAB4CAB5DAB0A3059F48AA9880F880F6E
:1015B000880F9AA9990F890F382D381B832F10C0D7
:1015C000003139F48AA98295807F482D481B842FE9
:1015D00007C08AA9880F880F880F582D581B852FA0
:1015E00090E02EA53FA548A959A982169306A40606
:1015F000B50608F091E08AA89BA8ACA8BDA88A30DF
:1016000010F4805D04C0895A183509F48F7DD30128
:101610008E933D01992309F099CF083041F4F3FEF0
:1016200006C0803321F080E3FD0182933F01CE01AB
:101630000196382E3618F8E23F0E0BC0112309F43C
:101640006CC03E010894611C711C198351E0352E59
:1016500019A6032D2DA4231827FC222489A588234D
:1016600011F00F5F02C0F6FC0E5F020DEF2CFF249D
:10167000C70180739070892B49F48CA5801B682F5B
:101680002C968EAD9FAD2C970E94CE8889A588237D
:1016900031F041E050E0BE01675D7F4F0AC0E6FED9
:1016A0000EC080E38AA71BA742E050E0BE01665D42
:1016B0007F4F2C968EAD9FAD2C970E949F88C701BF
:1016C00080739070809749F48CA5801B682F2C96AE
:1016D0008EAD9FAD2C970E94DF88622D2C968EAD2B
:1016E0009FAD2C970E94DF88832D992787FD9095C9
:1016F000AC01B3012C968EAD9FAD2C970E949F88B4
:10170000E4FE89CD2CA5201B2CA7622F2C968EAD34
:101710009FAD2C970E94CE887ECDE2E1CB5C0C94ED
:101720002992982F8091B60B883A50F48091B60B8D
:10173000E82FFF27E356F54F93838F5F8093B60B17
:101740000895982F8091B60B883A58F48091B60B83
:10175000E82FFF27E356F54F906893838F5F8093C0
:10176000B60B0895982F80912505882321F0892FA5
:101770000E94A18B0895892F0E94918B0895883A29
:1017800010F48093B60B089580E090E2E0EAFAE06E
:1017900091938F5F883AE0F308954FB721E830E0E6
:1017A000F8948091C9008F778093C9008091C90017
:1017B0008F7B8093C9008091C9008F7D8093C90081
:1017C0005A9A52985B9A539A832F99278093CD0007
:1017D0002093CC008091C80082608093C80088E18B
:1017E0008093C9008091CA008F778093CA0080914E
:1017F000CA008F7B8093CA008091CA008F7D80933E
:10180000CA008091CA008F7E8093CA008091CA006E
:10181000877F8093CA008091C90084608093C9004B
:101820008091CA0084608093CA008091CA0082605F
:101830008093CA008091C90081608093C900809123
:10184000C80087FF03C08091CE00F9CF8091C90006
:1018500080688093C9004FBF3CE73093190A2DE799
:101860002093440A8EE880931A0A1092360A109246
:10187000350A10921F0A80EE80931C0A3093710A79
:1018800020939C0A10927D0A10927C0A10927F0A83
:1018900010927E0A1092810A1092800A84EF91E0E1
:1018A00090937B0A80937A0A9093790A8093780ABE
:1018B0009093770A8093760A1092730A89E880934E
:1018C000720A10929A0A10929B0A80E98093740A15
:1018D0003093490B2093740B10924B0B8AE8809342
:1018E0004A0B1092510B1092500B10924F0B10920A
:1018F000530B1092540B1092550B1092560B1092E2
:10190000580B1092590B10925A0B10925B0B1092BD
:101910005F0B10925E0B10925D0B10925C0B80EAD5
:1019200080934C0B3093450A2093700A1092470A1B
:101930008DE88093460A10926F0A80ED8093480AE2
:101940008BE780939D0A80E880939E0A10929F0AFD
:1019500080911F0A90E2E0EAFAE091938F5F883A63
:10196000E0F38DE78093480B0895CF93C82F8091C3
:101970003805803879F48C2F0E9463748093270592
:1019800080912705882331F1C093B50B80912705FD
:101990008F5F16C08F37F1F48091AE0B882329F446
:1019A0008C2F80958F708093AE0B0E946C73809308
:1019B0009F0A8DE99AE090932905809328058DEA86
:1019C000809327058091C9008F7E8093C90082E0B3
:1019D00080932605C0933805CF9108953091260550
:1019E000332331F080912605815080932605089598
:1019F00080912705882381F1409127059091390531
:101A0000413091F4292F309339058091C9008061CC
:101A10008093C90080912505882319F0309325050E
:101A200010C0409325050DC0E0912805F0912905CF
:101A30008191F0932905E0932805282F980F909322
:101A400039058091C80085FFFCCF2093CE0080919E
:101A5000270581508093270508952FB740E0F8941B
:101A6000E0E0F0E081E2809357009491E2E0F0E062
:101A7000809357003491E4E0F0E080935700849124
:101A80002FBF9E3199F4363941F4893011F441E089
:101A90000DC08A3059F442E009C0373939F4863034
:101AA00011F443E003C0853009F444E0842F992702
:101AB00008959FB7F8948091C900877F8093C900EB
:101AC0008091C9008F7E8093C9008091C9008F7773
:101AD0008093C9008091C9008F7B8093C900809159
:101AE000C9008F7D8093C90052985A9A53985B9A87
:101AF0009FBF08951F93CF93DF93182F80912405E4
:101B0000882309F4A7C08091D102181709F4A2C054
:101B100080912305882321F40E942D8D8093230535
:101B200082ED91E0909339018093380189E791E14A
:101B30009F938F93C0E6D5E1DF93CF93E0913D056E
:101B4000F0913E0509950F900F900F900F90812F07
:101B50009927AA27BB27FC01099778F5E554FF4F81
:101B600020913D0530913E050C94449285E791E12A
:101B700002C08CE691E19F938F93DF93CF93F9019D
:101B8000099527C087E691E1F6CF8FE591E1F3CF84
:101B900087E591E19F938F93DF93CF93F9010995A7
:101BA00088ED91E0909339018093380112C082E56D
:101BB00091E1E1CF86E891E1DECF8CE891E19F935E
:101BC0008F93DF93CF93E0913D05F0913E0509950A
:101BD00010E00F900F900F900F90809123058430AC
:101BE00011F0823011F50E94598D812F8150833080
:101BF00018F40E947F6F2CC0143019F40E942186C3
:101C000027C0183019F40E94898222C0153019F4B7
